:020000040800F2
:10000000B05C00201F0500088D040008110F0008D7
:100010009104000893040008950400080000000003
:10002000000000000000000000000000970400082D
:1000300099040008000000009B0400089D040008CB
:100040009F040008A1040008A3040008A5040008F8
:10005000A7040008A9040008AB040008AD040008C8
:10006000AF040008B1040008B3040008B504000898
:10007000B7040008B9040008BB040008BD04000868
:10008000BF040008C1040008C3040008C504000838
:10009000C7040008C9040008CB040008CD04000808
:1000A000CF040008D1040008D3040008D5040008D8
:1000B000D7040008D9040008DB040008DD040008A8
:1000C000DF040008E1040008E3040008E504000878
:1000D000E7040008E9040008EB040008ED04000848
:1000E000EF040008F1040008F3040008F504000818
:1000F000F7040008F90400080000000000000000F8
:100100000000000000000000FB040008FD040008DF
:100110000000000000000000FF04000801050008C6
:100120000305000805050008070500080905000883
:100130000B0500080D0500080F0500081105000853
:10014000130500080000000000000000000000008F
:10015000000000000000000000000000000000009F
:100160000000000000000000150500081705000849
:1001700019050008000000001B0500080000000031
:08018000000000001D0500084D
:10020000DECEA5ED02003078463337320000000024
:100210000000000000004457325F313530370000E5
:100220000000000000004170706C69636174696FC8
:100230006E00000000000000000000000000000050
:100240000000000000000405C500DAF7DECEA5EDD1
:100250000200307846333732000000000000000012
:10026000000053504C6174436F6E74726F6C6C6518
:1002700072004170706C69636174696F6E00000098
:10028000000000000000000000000000000000006E
:0802900000000000FE00DAF797
:10029800790B000818000000B10D000803000000E9
:1002A800ED1300080600000095160008090000007C
:1002B800FD18000802000000F119000810000000F5
:1002C800AD1B0008FF000000991E00080C0000008C
:1002D8005920000800000000A521000805000000C2
:1002E800FD3F000812000000E94300080A00000072
:1002F8001D4800080A0000004550000814000000CE
:10030800D154000808000000E95B0008070000005D
:1003180091620008100000007966000813000000D0
:10032800217800081300000031A50008160000001D
:1003380079090108160000007D0B0108170000006C
:100348001144010816000000E144010817000000EC
:08035800A55601081500000084
:100360002F49072291438D462E492F480A1A06D05D
:100370000722914381F30988022282F314882B48D3
:100380002B492C4A00F039F82B482C492C4A00F014
:1003900034F82C482C492D4A00F02FF82C482D49D0
:1003A0002D4A00F02AF82D482D492E4A00F025F854
:1003B0002D482E492E4A00F020F82E482E490022C2
:1003C00000F026F82D482E49091A082903DB0022DF
:1003D0000260043001601F481F49884205D002684E
:1003E000043003B4904703BCF7E700208646EC4690
:1003F00000200021234A9047FEE7884207D0521A86
:1004000005D0037801300B700131013AF9D1704702
:10041000884202D002700130FAE770471A487047EC
:10042000B05C0020B0640020B05C002078B7010808
:1004300088010020200200207805000878050008C7
:100440005888010810B80108B0640020B06400208A
:100450007805000878050008780500087805000888
:1004600078050008780500085888010858880108B0
:1004700078B701082002002064590020B0590020FC
:10048000B0590020552E0008FFFFFFFFFEE7FEE7F2
:10049000FEE7FEE7FEE7FEE7FEE7FEE7FEE7FEE734
:1004A000FEE7FEE7FEE7FEE7FEE7FEE7FEE7FEE724
:1004B000FEE7FEE7FEE7FEE7FEE7FEE7FEE7FEE714
:1004C000FEE7FEE7FEE7FEE7FEE7FEE7FEE7FEE704
:1004D000FEE7FEE7FEE7FEE7FEE7FEE7FEE7FEE7F4
:1004E000FEE7FEE7FEE7FEE7FEE7FEE7FEE7FEE7E4
:1004F000FEE7FEE7FEE7FEE7FEE7FEE7FEE7FEE7D4
:10050000FEE7FEE7FEE7FEE7FEE7FEE7FEE7FEE7C3
:10051000FEE7FEE7FEE7FEE7FEE7FEE7FEE713483D
:10052000854600F022F84EF68850CEF200000168B1
:1005300051F47001016000BF00BF00BFF1EE100A6E
:1005400050F04070E1EE100A4FF0000080F3148884
:100550004EF63C71CEF20001086850F04070086021
:10056000034804490160FFF7FBBE7047008000208C
:0805700008ED00E000000008A6
:10057800F8B5044601F024FB06F052F8064640F2AE
:100588002025C2F200054FF000072B689869042C5B
:1005980017D8DFE804F0030609101300C0F340027F
:1005A80010E0C0F380120DE000F01102012A14BF20
:1005B8000022012206E0C0F3800203E0C0F34012EB
:1005C80000E03A4672B910F4807F0ED100F01001B5
:1005D800CBB26BB906F024F8801B0528D5D94FF0AB
:1005E8000000F8BD4FF00100F8BD4FF00000F8BD65
:1005F8004FF00000F8BD00BFF8B540F22024C2F269
:10060800000426684FF0FF35F561FF2B34BF1D4607
:10061800FF254FF000044FF0540767F3090461F316
:100628008A2465F31744FF2B94BF0023012363F347
:10063800186462F3596460F34D347460002914BF80
:1006480003200020FFF794FF002814BF284600204D
:10065800F8BD00BF2DE9F04F83B004468946154622
:10066800002A72D040F22023C2F200031868026800
:1006780042F0010101604FF001004FF000010A460D
:100688000346FFF7B9FF002848D040F22023C2F202
:100698000003186884624FF00100FFF769FF002823
:1006A8003FD04FF001004FF0030740F22028C2F27C
:1006B800000800E035464FF001010A462B46FFF7D7
:1006C8009BFF824680B3CB462E4600F1FF3202F0F4
:1006D800010101913846FFF74BFF00283AD126E087
:1006E8003846FFF745FF10B3D8F80020516AA146F5
:1006F80009F8011B06F1FF363846FFF739FF0028D5
:100708004DD114E04FF00400FFF732FF90B14FF0E5
:100718000000002ECED14FF001000DE04FF0000098
:100728000AE04FF0000007E04FF0000004E04FF04F
:10073800000001E04FF0000040F22021C2F2000169
:100748000B684FF000021A6001E04FF0010003B09F
:10075800BDE8F08FD8F80040636A89F8003009F1E5
:100768000104A14605F1FF360AEB0600A842C9D0EC
:10077800019A002AB4D03846FFF7FAFE0028D6D0EE
:10078800D8F800104B6A8BF8013004F10104A14637
:1007980006F1FF360AEB0600A842A1D1B2E7D8F865
:1007A8000030586A607009F10104A14606F1FF366D
:1007B8000AEB0602AA4293D1A4E700BF10B582B0A3
:1007C8001446B9BB4FF0120001A94FF00302FFF71E
:1007D80041FF90B39DF804309DF805004FEA0021D1
:1007E80041EA03409DF80620104313F0800F18BF1C
:1007F80040F07F4000280FDB14F0AEFF4FF040427E
:100808004FF6FF73C4F25F1315F0B8FA15F07EF8CF
:1008180020604FF0000012E014F09EFF4FF000023D
:100828004FF07A5315F0F4F915F070F820604FF096
:10083800000004E04FF0140001E04FF0180002B08F
:1008480010BD00BF08B51F290AD8084611464FF049
:100858000102FFF7FFFE00280CBF1820002008BD8A
:100868004FF0140008BD00BF2DE9F04F87B001918B
:100878009A468DF817204FF001038AF800301F2997
:100888005CD840F22021C2F200010C68226842F0D4
:10089800010626600DF117094FF0020B4FF0010415
:1008A80040F22026C2F200065F46CDF810A000E014
:1008B800D34620464FF000014FF001025B46FFF798
:1008C8009BFE8046002849D07CB9CDF80890444664
:1008D80008F1FF3101F0010203923846FFF748FEA4
:1008E800002855D1DDF810A043E0336801989862DC
:1008F8000BF1FF3BB8F1010808BFDA4613D0E4E773
:100908003846FFF735FE60B33168A94619F8013B50
:100918008B6204F1FF343846FFF72AFE00285FD1C6
:10092800DDF810A025E04FF00400FFF721FED8B154
:100938004FF00004BAF1000FBAD106E04FF0000002
:100948008AF800004FF014001FE040F22021C2F2A4
:1009580000010B684FF00000186016E0DDF810A0E9
:1009680007E0DDF810A004E0DDF810A001E0DDF8F4
:1009780010A040F22020C2F2000002684FF00001EF
:1009880011608AF800104FF0180007B0BDE8F08F2A
:10099800336899F80000029D05F101059862A9469F
:1009A80008F1FF340BEB040AC8EB0A0A002CBAD092
:1009B80003990029A4D03846FFF7DAFD0028D6D0DD
:1009C8003368029A507805F101059862A94604F146
:1009D800FF340BEB040CC8EB0C0A002C90D1A2E7F7
:1009E80030686A7809F101058262A94604F1FF348A
:1009F8000BEB040EC8EB0E0A002C81D193E700BF65
:100A0800F0B585B00C460B2800F2A1800B2900F246
:100A1800A18000EB800248F65C03C0F6010303EBFB
:100A280082010A7C002A40F0988004EB840148F691
:100A38005C03C0F6010303EB8102117C012940F03D
:100A48008F8048F65C03C0F6010300EB800253F880
:100A5800222004EB840153F821309A4240F083802D
:100A6800012A02D0022A33D119E041F21C06C4F24D
:100A78000206376847F40011316041F23003C4F2CE
:100A880002031A686FF304121A6040F22025C2F2BA
:100A9800000545F20046C4F200062E6018E041F257
:100AA8001C05C4F202052E6846F480072F6041F247
:100AB8003001C4F202010A686FF345120A6040F27D
:100AC8002023C2F2000345F60005C4F200051D60AC
:100AD80048F65C07C0F6010700EB800007EB8003CF
:100AE800187999684FF0000600964FF001050195B6
:100AF800DA6802924FF003022B4600F0D3FD04EBB4
:100B0800840407EB84042079A16800960195E368C2
:100B180002934FF003022B4600F0C4FD40F220215F
:100B2800C2F20001086848F65802C0F601021368CC
:100B3800036141F2020040F28811C2F2000140F262
:100B48002422C2F2000208F0A9FC28460DE04FF06A
:100B580000000AE04FF0000007E04FF0000004E05A
:100B68004FF0000001E04FF0000005B0F0BD00BFFD
:100B780000B583B04FF003004FF0000140F601428A
:100B8800C0F6000202F0DAFC4FF0010040F6114115
:100B9800C0F6000140F6F132C0F6000202F0CEFCC9
:100BA8004FF004004FF0050102460FF00BFE4FF026
:100BB800000000904FF0FF0301934FF00A014FF03F
:100BC8000B024FF0010301F087FE4FF004004FF0D5
:100BD8000501FFF715FF48F68410C0F6010005F07F
:100BE800D3FF03B000BD00BF08B519B94FF003002B
:100BF80014F01EFD08BD00BF08B5012903D14FF050
:100C0800010014F015FD08BD08B54FF0070000F00D
:100C1800E7FD08BD08B501464FF0080000F0E0FD0B
:100C280008BD00BF48F6A013C0F601031A684EF6C7
:100C38000C50CEF200000260FEE700BF08B5FFF7D7
:100C4800F1FF00BF51E8002FBFF35F8F41E80003B9
:100C5800012B3FF4F7AF1046704700BF13461A4602
:100C68002DE9F00F092AC0F00980B1E8F80FA0E8D3
:100C7800F80FA2F10902092ABFF4F7AF4FF00C03ED
:100C880003FB02F21D4B1A44974600F032B800BF2E
:100C980000BF00BF00BF0B68036000F02AB800BFA8
:100CA80000BF91E8180080E8180000F022B891E829
:100CB800380080E8380000F01CB891E8780080E837
:100CC800780000F016B891E8F80080E8F80000F025
:100CD80010B891E8F80180E8F80100F00AB891E846
:100CE800F80380E8F80300F004B891E8F80780E812
:100CF800F807BDE8F00F704713460000920C000893
:100D080013461A462DE9F00F0B460C460D460E46C3
:100D18000F46884689468A468B46092AC0F00780CE
:100D2800A0E8F80FA2F10902092ABFF4F9AF4FF0C1
:100D3800080303FB02F2144B1A44974600F020B84C
:100D480000BF00BF046000F01BB800BF80E830009F
:100D580000F016B880E8700000F012B880E8F000E3
:100D680000F00EB880E8F00100F00AB880E8F0035F
:100D780000F006B880E8F00700F002B880E8F00F4D
:100D8800BDE8F00F70471346440D0008EFF31180DB
:100D98004FF0800181F3118870474FF0000000BFC9
:100DA80080F31188704700BF30B440F20003C0F6EA
:100DB800000340F28812C0F60002D01A4FEAA001E0
:100DC800B1F5C47F04D81346264A9A4201D324E0D9
:100DD800FEE7254D254C601B20F003054FF000036E
:100DE80040F20002C2F2000240F20001C0F6000127
:100DF80005F10400C5F380045D589D5003F1040318
:100E0800834226D109E05C589C5003F104035C58E6
:100E1800D45003F104038342F5D14EF60853CEF2C1
:100E2800000340F20002C2F200021A604FF0B5015E
:100E3800CBF26B1145F6B010C2F2000001604EF61D
:100E48001453CEF200031A6842F01001196030BC46
:100E58007047002CD7D05C589C5003F104038342A0
:100E6800D1D1DAE700000008040000088B0100086F
:100E780010B4034600283ED002F1100440F20000EE
:100E8800C2F2000040F82430002A0ADA12F10C0FEE
:100E980035DB02F10C024EF61850CEF20000115468
:100EA8002DE04EF20014CEF200040F299CBF090178
:100EB800C9B24EF20043CEF20003D1541146002AC3
:100EC800B8BF02F11F014FEA611004EB80014FF037
:100ED8001F03C8F200031340002B05DA03F1FF32A9
:100EE80062F01F0303F1010358B24FF0010202FA46
:100EF80000F30B6003E0002AC8DB024CD5E710BC06
:100F0800704700BF80E100E01EF0040F0CBFEFF354
:100F18000880EFF3098020E9F00F00F001B800BF66
:100F280010B5026845F66413C2F200031A604168FE
:100F3800596082689A60C168D96002691A6141691A
:100F4800596182699A61C169D961026A1A62416A02
:100F58005962826A9A62C16AD962026B1A63416BEA
:100F68005963826B9A63C16BD96300F140001864BE
:100F78004EF62850CEF2000002685A6417F028FC9A
:100F8800002800F0FB8148F6A410C0F6010017F015
:100F980025FC4EF62C54CEF200042368002B05DA0B
:100FA80048F6B410C0F6010017F018FC4EF62C51A4
:100FB800CEF20001086810F0020F05D048F6C41000
:100FC800C0F6010017F00AFC4EF62852CEF20002D5
:100FD8005478002C72D048F6DC10C0F6010017F0E7
:100FE800FDFB4EF62853CEF20003597811F0010F9D
:100FF80005D048F6EC10C0F6010017F0EFFB4EF6EE
:101008002850CEF20000427802F00204E3B22BB17D
:1010180048F60C20C0F6010017F0E0FB4EF6285108
:10102800CEF20001487800F00402D4B22CB148F6A0
:101038003020C0F6010017F0D1FB4EF62853CEF24F
:101048000003597801F00800C2B22AB148F65420CA
:10105800C0F6010017F0C2FB4EF62854CEF2000489
:10106800637803F01001C8B228B148F67420C0F6BE
:10107800010017F0B3FB4EF62852CEF20002547866
:1010880004F02003D9B229B148F69420C0F6010033
:1010980017F0A4FB4EF62850CEF20000427802F07A
:1010A8008004E3B253B14EF63851CEF2000109681C
:1010B80048F6B420C0F6010017F090FB4EF6285011
:1010C800CEF20000428894B2002C5ED048F6D420BC
:1010D800C0F6010017F082FB4EF62853CEF200034B
:1010E800598811F0010F05D048F6E420C0F6010038
:1010F80017F074FB4EF62850CEF20000428802F03A
:101108000204A3B22BB148F61030C0F6010017F064
:1011180065FB4EF62851CEF20001488800F0040223
:1011280094B22CB148F63430C0F6010017F056FBE3
:101138004EF62853CEF20003598801F0080082B217
:101148002AB148F67430C0F6010017F047FB4EF696
:101158002854CEF20004638803F4807188B228B161
:1011680048F6A430C0F6010017F038FB4EF62852B6
:10117800CEF20002548804F4007399B229B148F6FB
:10118800C030C0F6010017F029FB4EF62850CEF209
:1011980000000278002A63D048F6D830C0F6010073
:1011A80017F01CFB4EF62854CEF20004237813F0F7
:1011B800010F05D048F6E830C0F6010017F00EFB25
:1011C8004EF62851CEF20001087800F00202D4B29F
:1011D8002CB148F60840C0F6010017F0FFFA4EF6A9
:1011E8002853CEF20003197801F00800C2B22AB1E0
:1011F80048F62040C0F6010017F0F0FA4EF62854E1
:10120800CEF20004237803F01001C8B228B148F6E2
:101218004440C0F6010017F0E1FA4EF62852CEF22B
:101228000002147804F02003D9B229B148F66840C6
:10123800C0F6010017F0D2FA4EF62850CEF20000A0
:10124800027802F08004E3B253B14EF63451CEF284
:101258000001096848F68840C0F6010017F0BEFA98
:1012680045F66414C2F20004216A48F6B440C0F698
:10127800010017F0B3FA616A48F6C840C0F60100E9
:1012880017F0ACFAA16A48F6DC40C0F6010017F086
:10129800A5FAE16A48F6F040C0F6010017F09EFA98
:1012A800216848F60450C0F6010017F097FA616803
:1012B80048F61850C0F6010017F090FAA16848F6F1
:1012C8002C50C0F6010017F089FAE16848F6405042
:1012D800C0F6010017F082FA216948F65450C0F6AA
:1012E800010017F07BFA616948F66850C0F6010002
:1012F80017F074FAA16948F67C50C0F6010017F09F
:101308006DFAE16948F69050C0F6010017F066FAE8
:10131800216B48F6A450C0F6010017F05FFA216C63
:1013280048F6B850C0F6010017F058FA616B48F655
:10133800CC50C0F6010017F051FAA16B48F6F050F6
:10134800C0F6010017F04AFA45F6AC10C2F20000E8
:10135800026848F61460C0F601001146126817F0DA
:101368003DFA40F2C073C2F200031A6848F62C60D6
:10137800C0F601001146126817F030FAFFF75EFC5C
:1013880010BD00BF00B504F045FE002808BF5DF899
:1013980004FBEFF30981EFF3118221E9F40F5DF803
:1013A80004EB1EF0100F08BF21ED108A41F804ED80
:1013B8000B4C2268002A18BF516004F09DFE226879
:1013C800516851F804EB1EF0100F08BFB1EC108AF9
:1013D800B1E8F40F82F3118881F30988704700009F
:1013E800AC59002008B541F28D30C0F600004FF02E
:1013F800FF016FF00102FFF73BFD08BDF8B5074696
:101408000C461E460799089D14F0030F00D0FEE70E
:1014180022B1A4EB8500A0F1480401E004F14800E2
:10142800012D01D8A16205E02A46FFF717FCA7EBBA
:101438008507A7624FF0000363604FF01130E06248
:101448004FF0223121634FF0333262634FF044335F
:10145800A3604FF05530E0604FF0663121614FF0E6
:10146800773262614FF08833A3614FF09930E061C1
:101478004FF0AA3121624FF0BB3262624FF0CC3399
:10148800A363E663069820644FF0807161646FF08F
:101498000202226005F11200F8BD00BF62B64EF6E6
:1014A8000453CEF200031A6842F08050186000BF5F
:1014B80010B540F20403C4F600031C6848F66C61DA
:1014C800C0F601010A6824EA020448F62872C0F648
:1014D8000102106804431C6040F20443C4F6000390
:1014E8001868496820EA0100526840EA02041C6052
:1014F80040F60403C4F600031868186040F6044177
:10150800C4F600010A680A6041F20404C4F6000443
:101518002368236041F20440C4F6000001680160BA
:1015280040F20C01C4F600010C6848F6AC62C0F643
:101538000102136824EA030448F6DC63C0F60103D9
:10154800186804430C6040F20C41C4F600010C68B2
:10155800506824EA0004586804430C6040F60C0103
:10156800C4F600010C68906824EA000498680443F3
:101578000C6040F60C41C4F600010C68D06824EAFF
:101588000004D86804430C6041F20C01C4F6000161
:101598000868126920EA02001B6940EA03040C602B
:1015A80041F20C41C4F600010868086048F69873D7
:1015B800C0F601031A6840F21404C4F6000422605D
:1015C800596840F21440C4F6000001604FF000036F
:1015D80040F61402C4F60002136040F61444C4F640
:1015E8000004236041F21401C4F600010B6041F2CB
:1015F8001440C4F60000036040F20001C4F6000184
:101608000C6848F6C072C0F60102136824EA0304A5
:1016180048F6C463C0F60103186804430C6040F23E
:101628000041C4F600010C68506824EA00045868B8
:1016380004430C6040F60001C4F600010C68906891
:1016480024EA0004986804430C6040F60041C4F69C
:1016580000010C68D06824EA0004D86820430860B8
:1016680041F20001C4F600010868126920EA02008C
:101678001B691843086041F20041C4F600010A687A
:101688000A604FF0010002F0D9FD10BD08B541F223
:101698001403C4F202031A6842F4FC001860FFF74E
:1016A80007FF08BD2DE9F0019DF814709DF818603A
:1016B800079D48F60074C0F6010454F820004FEA6C
:1016C8004104FF2F12D0D0F80C8048F6F46CC0F615
:1016D800010C5CF8277007FA04FC4FF0030707FABF
:1016E80004F728EA07074CEA0707C760FF2B11D061
:1016F800D0F804C048F64077C0F6010757F82370C1
:1017080007FA01F74FF0010303FA01F32CEA030388
:101718003B434360FF2E10D0876848F6B073C0F68D
:10172800010353F8266006FA04F64FF0030303FAA0
:1017380004F327EA030333438360B5F1FF3F16D070
:101748004FEAD10303F1080350F8236001F00701C1
:101758004FEA810105F00F0505FA01F54FF00F0773
:1017680007FA01F126EA0101294340F82310FF2A6C
:1017780010D001684FF0030303FA04F321EA0303CE
:1017880048F61871C0F6010151F8222002FA04F453
:101798001C430460BDE8F001704700BF48F6487379
:1017A800C0F6010353F820100A6848F67073C0F6B3
:1017B800010353F820100A4048F6D873C0F6010315
:1017C80053F82000824214BF00200120704700BF58
:1017D80048F60073C0F6010353F82000006970470B
:1017E80048F67073C0F6010353F820307BB139B165
:1017F80048F68461C0F6010151F820201360704753
:1018080048F64462C0F6010252F8200003607047AF
:1018180040F23023C2F200031B689BB1A8B91A68D2
:101828006FF300021A604FF00000586240F2342152
:10183800C2F2000108801A6842F0010018604FF0F7
:10184800010070474FF0000070474FF000007047EC
:1018580010B483B040F23023C2F200031B6803B314
:1018680010BB40F23422C2F20002586A148840EADF
:101878000440019000BF00BF00BF00BF00BF586A0E
:10188800148840EA04400090019C00988442ECD1FE
:10189800DDED017AB8EEE70A81ED000A4FF00100AC
:1018A80004E04FF0000001E04FF0000003B010BC6E
:1018B800704700BF40F23023C2F200031B689BB19F
:1018C800A8B91A686FF300021A6059624FEA114109
:1018D80040F23420C2F2000001801A6842F001018F
:1018E80019604FF0010070474FF0000070474FF04B
:1018F8000000704741F22403C4F20203186847F25B
:101908000402C4F20002136840F23622C2F2000256
:101918004FF00001117013F0010F03D04FF00400D5
:10192800107032E04FEA106212F0600F07D040F2F8
:101938003621C2F200014FF020020A7025E002F0C1
:101948000401C9B239B140F23623C2F200034FF0A4
:101958004000187019E0C3F3400343EAD06010F068
:10196800010F07D040F23621C2F200014FF0800289
:101978000A700AE002F01002D1B231B140F2362307
:10198800C2F200034FF00100187041F22401C4F2C2
:1019980002010A6842F080730B6047F20000C4F24B
:1019A8000000016841F00802026045F6AC13C2F27B
:1019B8000003186840F23821C2F20001086070473D
:1019C80040F23623C2F200031878704708B54FF288
:1019D800AC71C1F6FF714FF00C0215F017F94FF01A
:1019E8000C0008BD0000000010B542F20803CEF25A
:1019F80004031A6842F01000186041F6A920C0F6E6
:101A080000004FF00F014FF03602FFF731FA41F2B4
:101A18001C01C4F202010C6844F010030B6041F28F
:101A28000004C4F2000449F22C62C0F601021068F6
:101A3800206049F61C01C0F60101886913F0A4FE74
:101A480015A3D3E9002314F0E3F84FF000024FF098
:101A58000003C3F6F07313F095FF13F001FF41F292
:101A68002C03C4F20003188041F22800C4F20000DD
:101A78004FF00002028049F23061C0F601010868A7
:101A880041F20C03C4F200031860228842F00101FD
:101A9800218010BDAFF300802D431CEBE2362A3FB6
:101AA800684620F007018D4601B541F21003C4F2E3
:101AB80000034FF000021A6004F0BCFDBDE80140CD
:101AC8008546704770B50446B0F5CC7F2FD940F2F3
:101AD8003233984216D940F26560844215D940F6EF
:101AE800CB418C4214D941F69712944213D943F250
:101AF8002F36B44212D946F25F639C4298BF06253E
:101B08000ED90FE04FF001050AE04FF0020507E09B
:101B18004FF0030504E04FF0040501E04FF0050520
:101B2800072D06D1FFF78AF84FF0070501E04FF0BF
:101B38000005FFF72BF9064604EB84044FEAC400BE
:101B480049F23461C0F6010151F83520B0FBF2F3D7
:101B58009CB2012C05D9B4F5805F04D3FFF76EF869
:101B680001E04FF0020443F20000C4F2000045F225
:101B78005551016049F23462C0F6010202EBC50515
:101B88006B6843F20401C4F200010B6043F20802DF
:101B9800C4F2000214604AF6AA2303603046FFF735
:101BA800FFF870BD08B543F20003C4F200034CF619
:101BB800CC421A604FF0C800FFF784FF08BD00BF91
:101BC80043F20003C4F200034AF6AA221A607047DF
:101BD80010B5044643F20C03C4F20003186810F071
:101BE800010F74D04FF0320005F0DCFF43F20C0116
:101BF800C4F200010A6812F0010F68D04FF03200F9
:101C080005F0D0FF43F20C03C4F20003186810F08B
:101C1800010F5CD04FF0320005F0C4FF43F20C0115
:101C2800C4F200010A6812F0010F50D04FF03200E0
:101C380005F0B8FF43F20C03C4F20003186810F073
:101C4800010F44D04FF0320005F0ACFF43F20C0115
:101C5800C4F200010A6812F0010F38D04FF03200C8
:101C680005F0A0FF43F20C03C4F20003186810F05B
:101C7800010F2CD04FF0320005F094FF43F20C0115
:101C8800C4F200010A6812F0010F20D04FF03200B0
:101C980005F088FF43F20C03C4F20003186810F043
:101CA800010F14D04FF0320005F07CFF43F20C0115
:101CB800C4F200010A6812F0010F08D04FF0320098
:101CC80005F070FF43F20C03C4F200031B682046C2
:101CD800FFF7F8FE10BD00BF02469CF8043043B180
:101CE800DCF8000040B140F26421C2F2000141F882
:101CF8002200DCF8000050B940F26423C2F200036D
:101D080053F8220049F64042002808BF10467047A1
:101D18004FF00000704700BF40F20C03C4F6000308
:101D28001A681A6040F20C40C4F6000001680160AD
:101D380040F60C03C4F600031A681A6040F60C401B
:101D4800C4F600000168016041F20C03C4F6000308
:101D58001A681A6041F20C40C4F60000016801607C
:101D680040F20003C4F600031A681A6040F200400B
:101D7800C4F600000168016040F60003C4F60003E1
:101D88001A681A6040F60040C4F600000168016055
:101D980041F20003C4F600031A681A6041F20040D9
:101DA800C4F6000001680160704700BF38B50D46F1
:101DB800044600B3132801D9FEF740FF49F61C0377
:101DC800C0F6010353F8240055B1B0FBF5F14FEA12
:101DD800114202F10103B0FBF3F0B0FBF5F502E0AC
:101DE8004FF000052A4649F2CC71C0F6010151F8BE
:101DF80024309A62DD6238BD30B583B000918DF829
:101E080004200346B0B94FF000042046FFF780FFD6
:101E180038B1EC462046FFF75FFF01462046FFF742
:101E2800C5FF04F1010425462046FFF771FF00288D
:101E380029D020E049F26C62C0F6010212F82000B5
:101E4800012816D149F26C61C0F6010101EB830447
:101E5800637803EB830049F20002C0F6010252F8EE
:101E68002040EC462046FFF737FF01462046FFF7A3
:101E78009DFF03B030BDEC462046FFF72DFF01461D
:101E88002046FFF793FF04F10104142CBDD1F0E7BD
:101E980070B54FF0000001460246FFF7ADFF49F26A
:101EA800CC75C0F601054FF0010449F28066C0F612
:101EB80001062046FFF72CFFB0B112E02046FFF7DD
:101EC80027FF10B168683168016004F101042046F9
:101ED80005F10405FFF71CFF70B10AE0FFF71CFFCE
:101EE80070BD6B6832681A6004F1010405F10405DD
:101EF800E4E76B6832681A6004F1010405F104052F
:101F0800142CDBD1EAE700BF38B52DED028B05466E
:101F180041F21803C4F20203186810F4007F57D185
:101F280040F23C20C2F2000049F27861C0F601019B
:101F380003F0EEFA41F20404C4F2020422684FF0FE
:101F4800020161F38F32226041F21803C4F20203E6
:101F5800186840F400741C601A6842F001011960A6
:101F680042F20443C4F201034FF00000186049F242
:101F78007C64C0F60104226842F20C41C4F20101FB
:101F88000A6049F26C63C0F60103186842F2104413
:101F9800C4F20104206049F27062C0F601021168BF
:101FA80042F22C43C4F20103196049F27460C0F68E
:101FB8000100046842F20841C4F201010C600A6899
:101FC80042F004030B600846046814F0040FFBD1C8
:101FD80040F23C20C2F200004FF0000103F0B0FADA
:101FE80042F20044C4F20104616B4FF0110262F343
:101FF80004016163E36C4FF0050005F0D3FDA368AD
:1020080043F48000A06021460A6812F0020FFBD05A
:1020180042F20043C4F2010393ED138A40F23C20DC
:10202800C2F2000003F09AFB4FF2BA70C1F6FF70DB
:10203800018807EE901AB8EE670AF8EE480A80EEB3
:10204800208A85ED008A4FF00100BDEC028B38BD77
:1020580008B572B649F28C63C0F601031A684EF6E9
:102068003470CEF20000026049F29C61C0F60101B2
:102078000A684EF68853CEF200031A6049F294605B
:10208800C0F60100016842F20802CEF204021160B3
:1020980049F28863C0F60103186842F20C01CEF2D7
:1020A8000401086041F20003C4F202031A6842F412
:1020B8008030186019460B6813F4003FFBD049F2D2
:1020C8008462C0F60102106841F20401C4F2020100
:1020D800086049F29863C0F601031A6842F20000EA
:1020E800C4F20200026041F20001C4F202010B686E
:1020F80043F080720A600846016811F0007FFBD047
:1021080041F20403C4F202031A684FF0020060F3BC
:1021180001021A6019460B6803F00C02082AFAD16A
:1021280041F21800C4F20200016841F001030360A3
:1021380042F21C02C4F20202106848F66411C0F6AA
:1021480001010A6849F29063C0F601031B68504018
:10215800184222D048F66411C0F60101087800F050
:102168000401C8B2C8B942F21C01C4F202010868ED
:1021780020EA0300134018434FF60003C1F6FF732B
:102188005A68D1B261F317405B68C3F3074262F340
:102198001F604FF0FF3100F0A3F908BD41F21403AE
:1021A800C4F202031A6842F001001860704700BFC9
:1021B80070B41646002A47D040F20802C4F2020260
:1021C800146814F0010F06D040F20C05C4F20205A1
:1021D8002A68002AFCD140F20804C4F202044FF035
:1021E8000005256049F2A062C0F60102156840F2B8
:1021F8000402C4F20202156040F21002C4F20202A4
:10220800116040F21401C4F20201086040F20C00AF
:10221800C4F20200066049F2A462C0F60102116825
:102228002160206840F0010222606BB140F20C018D
:10223800C4F202010B68002BFCD140F20800C4F282
:1022480002004FF00002026070BC704742F21003B7
:10225800C4F20203186810F0800F0DD042F2040196
:10226800C4F2020140F22312C4F267520A6048F62F
:10227800AB13CCF6EF530B6042F21000C4F202002D
:10228800016801F08002002A14BF02200020704774
:1022980042F21003C4F20203186810F0800F07D14D
:1022A80042F21001C4F202010A6842F080030B6096
:1022B800704700BF40F20003C0F60003984208D3FD
:1022C80040F20001C0F6040188422CBF0020012022
:1022D80070474FF0000070472DE9F04706460D465D
:1022E800FFF7E8FF002855D02846FFF7E3FF00284E
:1022F80053D0AE4254D8FEF749FD8246FFF7A6FFF9
:102308000446B8BB41F28830FFF762FC49F2AC637F
:10231800C0F601031A6842F21000C4F2020002601B
:1023280042F21409C4F20209804642F20C07C4F2D0
:102338000207FFF745FCC9F80060D8F8001041F023
:102348004003C8F8003006F500663A6812F0010F3D
:10235800FBD1386810F0200F0AD0396841F020030B
:102368003B60B542E5D24FF06400FFF731FC01E075
:102378004FF0020449F2B062C0F60102106842F25E
:102388001001C4F202010860FFF782FF5046FEF711
:1023980007FD07E04FF0020404E04FF0020401E0FB
:1023A8004FF002042046BDE8F08700BFF8B50746A5
:1023B8000C4616460846FFF77DFF002800F0898086
:1023C80006F1FF302018FFF775FF002800F0848021
:1023D80040F2D073C2F2000353E8002F02F1010269
:1023E80043E800210129F7D0FFF730FF0546002810
:1023F8004BD149F2B461C0F601010A6842F21000FB
:10240800C4F20200026014F0010F09D037F8013C51
:1024180024F8013C04F1010407F1010706F1FF3635
:10242800012E25D904F1020207F10200A6F1020CDF
:102438004FEA5C0C04F1040E0EEB4C0E42F20C0158
:10244800C4F202010B6813F0010FFBD130F8023C13
:1024580022F8023C02F1020200F102007245F1D1B9
:102468000CF101024FEA420024183F1806F0010659
:102478000EB13978218049F2B864C0F601042268A7
:1024880042F21003C4F202031A60FFF701FF40F2A0
:10249800D073C2F2000353E8002FA2F1010243E80F
:1024A8000024012CF7D053E8002FB2F1004F0DD1D2
:1024B8004FF0000243E80024012CF4D04EF60450FB
:1024C800CEF20000016841F080510160BFF32F8F08
:1024D80004E04FF0020501E04FF002052846F8BD80
:1024E80030B585B004460D4668464FF0FF014FF001
:1024F800100214F0AFFBE3B203F00402D0B20028DC
:1025080040F0B58003F00201CBB223B14FF01100C7
:102518008DF8000003E06FF055028DF80020C4F339
:1025280007218DF80210C4F307438DF804304FEAF1
:1025380014648DF806408DF80850FEF727FC054610
:10254800FFF784FE002840F0868042F20800C4F2BB
:10255800020040F22312C4F26752026048F6AB113F
:10256800CCF6EF51016042F21003C4F202031C687A
:1025780014F4007F6FD049F2A860C0F60100026829
:1025880042F21001C4F202010A600B6843F04004F1
:102598000C6042F20C00C4F20200026812F0010F53
:1025A800FBD142F21003C4F202034FF0000119609C
:1025B80042F20804C4F2020440F22310C4F2675045
:1025C800206048F6AB12CCF6EF5222601B6813F479
:1025D800007F40D049F2BC61C0F601010C6842F2AC
:1025E8001000C4F20200046042F20802C4F20202BF
:1025F80040F22313C4F26753136048F6AB11CCF6CC
:10260800EF511160046814F4007F24D04FF60003E2
:10261800C1F6FF7303F11000834213D24FF0100488
:102628004FF00001184642F20C02C4F202023DF8D3
:1026380001300B52136813F0010FFBD101F10201B5
:10264800A142F4D142F21004C4F202044FF0000196
:102658002160FFF71DFE4FF0000442F21000C4F2A3
:10266800020004602846FEF79BFB204601E04FF07D
:10267800020005B030BD00BF40F2B423C2F200032F
:102688001868704770B48568C668446806FB0540DA
:102698004118196040F2B420C2F20000006881427B
:1026A8000CD2521890420CD340F2B820C2F200006B
:1026B8000268891819604FF0010004E04FF000002B
:1026C80001E04FF0000070BC704700BF2DE9F041F9
:1026D8000546FFF775FA4FF01E0440F2BC26C2F219
:1026E80000064FF000084FF0010733689869042D81
:1026F80017D8DFE805F0030609101300C0F34002FD
:1027080010E0C0F380120DE000F01102012A14BF9E
:102718000022012206E0C0F3800203E0C0F3401269
:1027280000E04246AAB9C0F3072111F0010F14D105
:1027380000F01003D8B2A0B901F00202D1B2A1B9D9
:10274800384605F02FFA013CCFD14FF00000BDE824
:10275800F0814FF00100BDE8F0814FF00000BDE8C6
:10276800F0814FF00000BDE8F0814FF00000BDE8B7
:10277800F08100BFF8B540F2BC24C2F2000425681D
:102788004FF0FF36EE61FF2B34BF1E46FF264FF099
:1027980000044FF0A00767F3090461F38A2466F385
:1027A8001744FF2B94BF0023012363F3186462F3DB
:1027B80059646C6060F34D346C60002914BF0320C9
:1027C8000020FFF783FF002814BF30460020F8BD23
:1027D8002DE9F04180460F4616461D46FFF7CAFF11
:1027E8000446002874D14FF0050003F09FFA4046D4
:1027F800394632462B46FFF7BDFF0446002867D10D
:102808004FF0050003F092FA4046394632462B460F
:10281800FFF7B0FF044600285AD14FF0050003F037
:1028280085FA4046394632462B46FFF7A3FF044651
:1028380000284DD14FF0050003F078FA404639469C
:1028480032462B46FFF796FF0446002840D14FF04A
:10285800050003F06BFA4046394632462B46FFF72F
:1028680089FF0446002833D14FF0050003F05EFAD3
:102878004046394632462B46FFF77CFF044638BBB4
:102888004FF0050003F052FA4046394632462B46CF
:10289800FFF770FF0446D8B94FF0050003F046FA79
:1028A8004046394632462B46FFF764FF044678B95E
:1028B8004FF0050003F03AFA4046394632462B46B7
:1028C800FFF758FF044618B94FF0050003F02EFA39
:1028D8002046BDE8F08100BF2DE9F04184B01446E0
:1028E8001D460B2900F2A4800B2A00F2A48001EBFC
:1028F800810249F2C463C0F6010303EB8202137C30
:10290800002B40F09B8004EB840249F2C463C0F6BC
:10291800010303EB8202137C012B40F0928049F201
:10292800C463C0F6010301EB810653F8262004EBCB
:10293800840653F826309A4240F0868040F2C02739
:10294800C2F200073870012A02D0022A23D111E00E
:1029580041F21C00C4F20200066846F4001202604C
:1029680040F2BC23C2F2000345F20047C4F200075C
:102978001F6010E041F21C00C4F20200066846F431
:102988008002026040F2BC23C2F2000345F6000751
:10299800C4F200071F6049F2C468C0F6010801EBE1
:1029A800810108EB8102107991684FF000060096CA
:1029B8004FF001070197D36802934FF003023346A3
:1029C800FEF770FE04EB840408EB84042079A16808
:1029D80000960197E26802924FF003023B46FEF729
:1029E80061FE40F2BC20C2F2000001680E6049F2AC
:1029F800C063C0F601031A680A6145B340F2B82003
:102A0800C2F200000A99016040F2B422C2F2000248
:102A18000B9B136040F2C420C2F2000049F2C0715F
:102A2800C0F601012A46334606F0FEFD384610E09E
:102A38004FF000000DE04FF000000AE04FF00000FA
:102A480007E04FF0000004E04FF0000001E04FF015
:102A5800010004B0BDE8F0812DE9F04F83B0914644
:102A68000D46002900F09C8040F2BC23C2F200030E
:102A780019680A6842F001040C60044640F2C02A52
:102A8800C2F2000A49F2B47BC0F6010B40F2BC273F
:102A9800C2F200079AF800005BF8206006F1FF33E5
:102AA80009EA0301731A00F1FF3202F0FF0001285E
:102AB8008CBF012602264FF001004FF000010246AC
:102AC800AB4294BFF3187319FFF782FE064600283D
:102AD80052D09AF8001001F1FF33DAB2012A0BD86C
:102AE8003868C9F30721816206F1FF364FF002000A
:102AF800FFF7ECFD002842D03B685FFA89F29A6242
:102B0800013E26D04FF0020806F1FF3000F0010127
:102B180001914046FFF7DAFD002846D132E04046F1
:102B2800FFF7D4FD70B334B1386814F8012B6FEA9D
:102B38000201816203E039684FF0FF038B6206F1FE
:102B4800FF3605F1FF354046FFF7C0FD002855D197
:102B580018E09AF800005BF820108944C1F10002DF
:102B680009EA02094FF00400FFF7B0FD68B1002D33
:102B780090D14FF001000AE04FF0000007E04FF05D
:102B8800000004E04FF0000001E04FF0000040F2C8
:102B9800BC23C2F2000319684FF000020A6001E08A
:102BA8004FF0010003B0BDE8F08F24B93B684FF047
:102BB800FF029A6205E0386814F8011B6FEA010306
:102BC800836205F1FF35013EC3D0019A002AA6D0E1
:102BD8004046FFF77BFD0028D4D024B938684FF071
:102BE800FF01816205E03B6814F8012B6FEA0200DF
:102BF800986205F1FF35013E91D1AAE724B93B68F7
:102C08004FF0FF00986205E0396814F8012B6FEA6D
:102C180002038B6205F1FF35013E80D199E700BFC1
:102C280030B583B015461C461A4601ABFFF72AFD9E
:102C380048B128462146019AFFF70EFF00280CBF2D
:102C48001820002001E04FF01F0003B030BD00BF86
:102C58002DE9F04F83B0044689461646002A00F055
:102C68009E8040F2C023C2F20003187800F1FF31C1
:102C780001F0FF0340F2BC22C2F2000211680868AA
:102C880040F001020A604FF001004FF000010A46CF
:102C980083428CBF03460223FFF79AFD002864D0C5
:102CA80040F2C023C2F20003197801F1FF30C2B22A
:102CB800012A0DD840F2BC23C2F200031968C4F3FC
:102CC800072088624FF00200FFF700FD00284FD070
:102CD80040F2BC22C2F200021368E4B29C624FF0D8
:102CE8000100FFF7F3FC002845D04FF001004FF03A
:102CF800030740F2BC28C2F2000800E02E464FF05D
:102D080001010A463346FFF735FD8246002835D0D3
:102D1800CB46354600F1FF3101F0010001903846FD
:102D2800FFF7D4FC00283FD12BE03846FFF7CEFC54
:102D380038B3D8F80020536A6FEA0301A14609F8AE
:102D4800011B05F1FF353846FFF7C0FC002854D1B8
:102D580017E04FF00400FFF7B9FCA8B14FF00000EE
:102D6800002DCBD14FF0010010E04FF000000DE036
:102D78004FF000000AE04FF0000007E04FF00000BD
:102D880004E04FF0000001E04FF0000040F2BC22E8
:102D9800C2F2000213684FF00001196001E04FF021
:102DA800010003B0BDE8F08FD8F80040626A6FEA0E
:102DB800020389F8003009F10104A14606F1FF3544
:102DC8000AEB0501B142C4D001980028ADD03846BD
:102DD800FFF77CFC0028D4D0D8F80020536A6FEAAB
:102DE80003018BF8011004F10104A14605F1FF3538
:102DF8000AEB0500B04298D1ABE7D8F80000426A68
:102E08006FEA0203637009F10104A14605F1FF3579
:102E18000AEB0501B14288D19BE700BF30B583B00A
:102E280015461C461A4601ABFFF72CFC48B1019821
:102E380029462246FFF70CFF00280CBF1820002067
:102E480001E04FF01F0003B030BD00BF08B545F6E4
:102E5800B010C2F2000045F6B042C2F20002131AE6
:102E68004FF0FF314FEAA302FDF74AFF01F044FF9C
:102E7800FEF714FB4FF0000008BD00BFBFF36F8FD3
:102E8800704700BF49F66C03C0F60103185C00EBFD
:102E9800400149F68812C0F6010252F821305B6AF7
:102EA800704700BF38B549F66C03C0F601031B5CD8
:102EB80003EBC30440F2D422C2F2000202EB840204
:102EC80082F8211014693CB140F2D425C2F2000501
:102ED8001346D2699B69A04738BD00BFF8B50646BE
:102EE8000F4649F66C03C0F601031D5C05EBC500EF
:102EF80040F2D424C2F2000404EB8004D4F810C0D9
:102F0800BCF1000F07D0E2698A4204D030464FF086
:102F18000001A369E047E76163695BB105EBC500A0
:102F280040F2D422C2F2000202EB80023046394657
:102F38009269984794F8201079B127696FB105EB29
:102F4800C50540F2D423C2F2000303EB85053046E1
:102F580094F82110E269AB69B847F8BD49F66C03EB
:102F6800C0F60103185C00EB400149F68812C0F670
:102F7800010252F82130186840F08001196070474A
:102F880049F66C03C0F60103185C00EB400149F6F2
:102F98008812C0F6010252F82130986940F0020107
:102FA80099611A6842F0800018607047F8B50446C5
:102FB80000EB400249F68813C0F6010353F822607B
:102FC800F569356205F0010215F0020F1CBF42F0E9
:102FD8000202D2B215F0040F18BF42F0080215F031
:102FE800080F18BF42F0040215F4807F05D07068FE
:102FF80010F4804F18BF42F0100215F0200F00D1D6
:10300800E2B104EBC40140F2D427C2F2000707EB97
:1030180081039F688FB1716A04EBC40040F2D42326
:10302800C2F2000303EB800349F65810C0F6010012
:10303800005DC9B29B69B84700E0736A326812F054
:10304800800F1CD015F0800F19D031686FF3C711AD
:10305800316004EBC40040F2D423C2F2000353F8F9
:10306800203063B140F2D422C2F2000202EB8002A7
:1030780049F65810C0F60100005D9169984715F0AF
:10308800400F17D004EBC40140F2D423C2F200036E
:1030980003EB810253686BB1084640F2D421C2F2B7
:1030A800000101EB800249F65810C0F60100005DEE
:1030B80091699847F8BD00BF684620F007018D4622
:1030C80001B54FF00300FFF771FFBDE801408546E9
:1030D800704700BF684620F007018D4601B54FF0E4
:1030E8000200FFF763FFBDE801408546704700BF57
:1030F800684620F007018D4601B54FF00100FFF743
:1031080055FFBDE801408546704700BF10B582B045
:103118008DF8071049F66C03C0F60103185C00EB44
:10312800400249F68811C0F6010151F82240E369CE
:1031380013F0800FFBD002A911F8012DA26200EB59
:10314800C00040F2D424C2F2000404EB8004608C76
:103158004FF0010204F03EFD608404F1200402B047
:1031680010BD00BF70B582B08DF8071049F66C032A
:10317800C0F60103185C00EB400149F68812C0F65E
:10318800010252F82140E56915F0800F1DBF9DF836
:103198000750A5620126002600EBC00340F2D420A8
:1031A800C2F2000000EB8305688C0DF107014FF0B7
:1031B800010204F00FFD688405F12005216841F043
:1031C80080022260304602B070BD00BF2DE9F04396
:1031D80085B016461F4649F66C03C0F601031C5C11
:1031E80004EB440249F68815C0F6010555F822405B
:1031F80049F68413C0F60103185C00EB400249F657
:103208007005C0F6010505EBC2058846002956D0B1
:10321800002E57D0287B29699DF8342000924FF062
:10322800010301936A6902924FF003023B46FEF7DD
:1032380039FA40F2D073C2F2000353E8002F02F1CA
:10324800010243E800210129F7D021684FF000006E
:103258002060012E14BF00260126626866F3CF3273
:10326800626049F66C10C0F601000268B8F1010FFF
:1032780014BF4FF000084FF0010868F3C302A260C2
:10328800216053E8002FA2F1010243E80024012C39
:10329800F7D053E8002FB2F1004F0DD14FF00002E4
:1032A80043E80024012CF4D04EF60450CEF200007E
:1032B800016841F080510160BFF32F8F17E04FF094
:1032C800010901E04FF00009287869689DF830305D
:1032D80000934FF001020192AB6802934FF0030292
:1032E8003B46FEF7DFF9B9F1000FA2D092E705B02F
:1032F800BDE8F0832DE9F84F81468B4690461E467F
:103308009DF828A049F66C03C0F601031D5C05EB87
:10331800450249F68810C0F6010050F822409DF891
:103328002C70012F14BF00270127082E06D0072E66
:1033380002D1B8F1000F01D1FDF780FC0AF1FF318D
:10334800CBB2012B01D9FDF779FC49F65C12C0F626
:10335800010252F82500B0FBFBF1E1604FF02002BA
:1033680067F38612BAF1010F04D0002F0CBF0223B5
:10337800002301E04FF0000363F30D3267F38E3250
:103388006068C0F3C03363F3CF3262604FF06D0101
:10339800B8F1020F14BF0023012363F3492118F188
:1033A800000818BF4FF0010868F38A21082E18BFDB
:1033B8004FF0000868F30C3121604846FFF762FDC2
:1033C800BDE8F88F2DE9F843054649F66C03C0F6C9
:1033D8000103185C00EBC00240F2D424C2F20004DE
:1033E80004EB820449F68811C0F6010100EB40069F
:1033F8004FEA860301EB030851F80390FDF7C6FC7A
:10340800064694F82000B8B14FF00007C9F80070DC
:103418003846394698F90420FDF72AFD28463946EA
:10342800FFF740FDE3681BB12846E169A2699847A8
:103438004FF0000284F820203046FDF7B1FCBDE8CB
:10344800F88300BF2DE9F04F85B005468B469246BC
:10345800994649F66C03C0F601031E5C40F2D42875
:10346800C2F2000806EBC6074FEA870708EB070415
:1034780006EB460049F68811C0F6010101EB80060B
:10348800FDF784FC039041F21C03C4F202031868A0
:1034980049F65011C0F601010A6820EA020E49F601
:1034A8004812C0F6010210684EEA0000186041F2A6
:1034B8001803C4F202031868496820EA0100526838
:1034C8001043186049F67011C0F6010105EB850339
:1034D800C818C95C4278837890F803C0CDF800C05A
:1034E800007901902846FFF771FE9DF83820009278
:1034F8009DF83C1001912846594652464B46FFF725
:10350800F9FE109B48F807301298A060119A626083
:103518001399E160149BA361B0684FF00F0196F90D
:103528000420FDF7A5FC4FF0010084F82000039863
:10353800FDF736FC05B0BDE8F08F00BF49F66C0317
:10354800C0F60103185C00EBC00340F2D420C2F2BD
:10355800000000EB830319615A61704749F6841330
:10356800C0F60103185C00EB400149F6B802C0F64A
:10357800010202EB01107047032812D849F66C03C8
:10358800C0F60103185C00EBC00140F2D422C2F27D
:10359800000202EB81034FF6FF7058844FF00100E0
:1035A80070474FF00000704703280ED849F66C03A7
:1035B800C0F60103185C00EBC00140F2D422C2F24D
:1035C800000202EB8103588C70474FF000007047EF
:1035D800F8B54FF04C0404FB00F440F6CC21C2F2DD
:1035E8000001621846F20003C4F2000303EB001363
:1035F80045F60045C4F2000505EB80006558002D2E
:1036080074D094680CB1968801E04FF000061F68EA
:1036180066F30F071F6059686FF309015960D16895
:1036280019B15668A719BFB201E04FF000079E68AC
:1036380067F30F069E603E2994BF00270127DE68C6
:1036480067F3CF36DE60DE6816F4004F1DBF4F0902
:1036580007F1FF3707F01F07C1F34407DE6867F378
:103668008E26DE600368166A66F303032E7A49F62F
:10367800CC15C0F6010555F8265065F34A236FF3BB
:103688000823C3F30115002C14BF022400246C4046
:1036980064F30513C3F30134002914BF0321002187
:1036A800614061F30D336FF3CF336FF3C7130360DA
:1036B80040F6C450C2F200000378191F18BF012158
:1036C80051624FF0010090624FF00003D362136320
:1036D800536340F27C30C2F20000018801F101011D
:1036E8008BB2038002F1100000F050FDF8BD00BF5E
:1036F800F8B545F64443C4F200031C6840F2643050
:10370800C2F20000028802F1010291B2018014F4B1
:10371800004F00F0948045F64445C4F200052E6839
:1037280006F00F0340F6CC27C2F200074FF04C001A
:1037380000FB037545F60042C4F2000202EB830762
:1037480040F27E31C2F200010E8806F10106B0B2E5
:10375800088052F82360C6F3C032EB6A1343EB6269
:10376800C6F3C021286B08432863C6F3C0126B6BED
:1037780013436B63C6F3072101F00800C2B25AB1C4
:103788004FF00003EB6340F28A31C2F2000108886F
:1037980000F1010082B20A80EB6B93B126F07F0141
:1037A800C8B270B140F28033C2F200031A8802F145
:1037B800010291B219804FF000016963286A03F091
:1037C80047FCE86A18B96B6B0BB92A6B7AB340F2FD
:1037D8008231C2F20001088800F1010083B20B8037
:1037E80005F1100000F0D2FC08BB40F29032C2F2A2
:1037F8000002108840F26431C2F200010B8840F2E6
:103808006832C2F2000222F8103000F1010080B2E2
:10381800092805D840F29031C2F20001088006E07C
:1038280040F29033C2F200034FF000021A8049F6CA
:10383800C810C0F60100016826EA01063E6014F4CB
:10384800806F16D040F28433C2F200031A8802F166
:10385800010290B2188040F6A251C2F200014FF066
:1038680001030B7040F69852C2F20002106802F091
:10387800C7F814F4006F25D040F28630C2F2000079
:10388800018801F101018BB2038045F64040C4F282
:103898000000026842F00801016040F62C53C2F2B1
:1038A80000034FF00100187040F6A151C2F2000168
:1038B8004FF000020A7040F69853C2F200031868ED
:1038C80002F09EF814F4805F25D040F28830C2F2EE
:1038D8000000018801F101018AB2028045F64043E7
:1038E800C4F2000318686FF3C300186040F62C5147
:1038F800C2F200014FF000020A7040F6A153C2F272
:1039080000034FF00100187040F69851C2F2000110
:10391800086802F075F86FEA040445F64442C4F2F8
:1039280000021460F8BD00BF684620F007018D460C
:1039380089B500AFFFF7DCFEBD46BDE88940854686
:10394800704700BF45F64043C4F200031A6860F3AD
:10395800CF321A60704700BF40F6C853C2F2000366
:103968001A5C45F60040C4F2000049B150F8220044
:10397800C0F3011149F6E413C0F60103585C70471F
:1039880050F82210C1F3013349F6E412C0F60102DF
:10399800D05C704740F6C853C2F200031A7845F667
:1039A8000043C4F2000353F8221049F6BC10C0F6D5
:1039B8000100006821EA000181F0100141F48070E3
:1039C80043F8220040F28C33C2F200031A8802F155
:1039D800010291B2198070472DE9F00340F6C853EF
:1039E800C2F20003185C45F6004CC4F2000C0CEB64
:1039F800800C4FEA001346F20007C4F2000703EBFD
:103A08000708D85983B207EB4307012A31D901F1D6
:103A18000204A2F102094FEA590901F1040606EB72
:103A28004906351BA5F10205C5F3400534F8024CDB
:103A3800384620F8044B01F10403B34238D10FE0B3
:103A480033F8025C044624F8045B03F1020333F8FC
:103A5800025C858004F1040003F10203B342EFD154
:103A680002F0010009F1010901EB490107EB89079F
:103A780000E0104608B109783980D8F8040062F3EC
:103A88000900C8F80400DCF8003049F6C012C0F696
:103A98000102116823EA01000346C0F3011282F013
:103AA800030161F30513CCF80030BDE8F00370475B
:103AB800002DC5D033F8024C20F8044B03F1020363
:103AC800B342BDD1CCE700BF2DE9F00140F6C853A1
:103AD800C2F200031C5C45F6004CC4F2000C0CEB6F
:103AE800840C46F20000C4F2000000EB0414A36842
:103AF8009BB200EB4300E3684FEA83534FEA9353CA
:103B0800934204D2E2684FEA82534FEA9352012A61
:103B180031D901F10203A2F102084FEA580801F174
:103B2800040707EB4807FD1AA5F10205C5F340068F
:103B3800044634F8045B23F8025C01F10403BB4239
:103B480034D10FE0254635F8046B23F8026C03F1F5
:103B58000203A48823F8024C05F1040403F10203CC
:103B6800BB42EFD102F0010308F1010801EB480163
:103B780000EB880000E013460BB103880B70DCF8FB
:103B8800000049F6C411C0F601010B6820EA0300E1
:103B98000346C0F3013181F0030060F30D339BB29B
:103BA800CCF800301046BDE8F0017047002EC9D0AF
:103BB80034F8045B23F8025C03F10203BB42C1D171
:103BC800D0E700BF08B545F64043C4F200031A68C1
:103BD8006FF3C3021A604FF00000FFF7F9FC4FF0D3
:103BE8000100FFF7F5FC4FF00200FFF7F1FC4FF082
:103BF8000300FFF7EDFC4FF00400FFF7E9FC4FF07E
:103C08000500FFF7E5FC4FF00600FFF7E1FC4FF079
:103C18000700FFF7DDFC49F6DC10C0F6010001687B
:103C280045F64C43C4F20003196008BD2DE9F04184
:103C3800074640F6CC23C2F200031868002800F0BB
:103C4800118140F6CC21C2F200014A683F2A08D906
:103C580040F6CC24C2F20004A5685619E368F518AA
:103C680001E04FF0400540F6CC20C2F20000C16CE4
:103C7800002900F0008140F6CC22C2F20002146D47
:103C8800A54207D840F6CC26C2F20006756D601929
:103C9800B36DC51840F6CC21C2F20001D1F89820C6
:103CA800002A00F0EC8040F6CC24C2F20004D4F8DC
:103CB8009C60B54209D840F6CC20C2F20000D0F88A
:103CC800A0507119D0F8A430CD1840F6CC22C2F219
:103CD8000002D2F8E440002C00F0D58040F6CC2653
:103CE800C2F20006D6F8E800854209D840F6CC2191
:103CF800C2F20001D1F8EC504219D1F8F030D518D1
:103D080040F6CC24C2F20004D4F83061002E00F052
:103D1800BE8040F6CC20C2F20000D0F834118D42AB
:103D280009D840F6CC22C2F20002D2F838514C1918
:103D3800D2F83C31E51840F6CC26C2F20006D6F897
:103D48007C01002800F0A78040F6CC21C2F20001D7
:103D5800D1F88021954209D840F6CC24C2F200045B
:103D6800D4F884515619D4F88831F51840F6CC2087
:103D7800C2F20000D0F8C811002900F0908040F687
:103D8800CC22C2F20002D2F8CC41A54209D840F6B2
:103D9800CC26C2F20006D6F8D0516019D6F8D43134
:103DA800C51840F6CC21C2F20001D1F81422002A2D
:103DB80079D040F6CC24C2F20004D4F81862B54297
:103DC80009D840F6CC20C2F20000D0F81C52711974
:103DD800D0F82032CD1840F6CC22C2F20002D2F838
:103DE8006042002C63D0454E4FF00808FCF726FFD0
:103DF800387A88B140F28E31C2F200010A8812F096
:103E0800020F0CD04FF0010404F1010442FA04F34C
:103E180013F0010FF8D104E04FF0000401E04FF077
:103E2800010440F28E30C2F200004FF0010202FAA3
:103E380004F201880A4302807889B060BB89F36084
:103E48003F2B99BF013323F001031F3323F01F03D6
:103E5800F360F26881184819B0F5E07F2ED9FCF7B5
:103E6800EDFE2BE040F6CC26C2F200064FF000082B
:103E78004FF040051EE0224E4FF001081AE0214E97
:103E88004FF0020816E0204E4FF0030812E01F4ED4
:103E98004FF004080EE01E4E4FF005080AE01D4ED4
:103EA8004FF0060806E01C4E4FF0070802E0134EDC
:103EB8004FF00808B8F1070F9AD997E740F6C853AA
:103EC800C2F2000303F804803760756006F120052C
:103ED80028464FF000014FF01C0212F0BBFE34627E
:103EE8007A68B26306F110004FF006013A682B4673
:103EF80000F02CF92046BDE8F08100BF2C0D002011
:103F0800180B0020640B0020B00B0020FC0B0020D5
:103F1800480C0020940C0020E00C0020032907D155
:103F280045F64C43C4F200031A6860F306021A60AF
:103F3800704700BFF0B585B00646002842D041F270
:103F48001C01C4F202010C6844F400050D604FF036
:103F5800000400944FF0030501954FF00E070297F7
:103F680020464FF00B012A462346FDF79BFB0094A1
:103F78000195029720464FF00C012A462346FDF78B
:103F880091FB49F6E013C0F601031A6845F640476D
:103F9800C4F200073A60284603F004FE3C6043F68A
:103FA8003110C0F600004FF00F014FF04B02FCF744
:103FB8005FFF45F64440C4F2000004604FF41C4122
:103FC800396011E04FF000004FF00F014FF04B0245
:103FD800FCF74EFF49F6B813C0F601031A6845F618
:103FE8004040C4F2000002603046FCF713FE05B002
:103FF800F0BD00BF2DE9F04182B049F6E817C0F6E0
:10400800010744F2DD06C0F6000640F2BC15C2F214
:1040180000054FF00408CDF8008038464FF08001C5
:1040280032462B4601F038FE40F2C434C2F2000496
:104038002060CDF8008038464FF08101324605EB0C
:10404800080301F029FE6060CDF8008038464FF083
:104058008201324605F1080301F01EFEA060CDF88A
:10406800008038464FF08301324605F10C0301F019
:1040780013FEE060CDF8008038464FF084013246E8
:1040880005F1100301F008FE2061CDF800803846E4
:104098004FF08501324605F1140301F0FDFD606122
:1040A800CDF8008038464FF08601324605F11803F6
:1040B80001F0F2FDA061CDF8008038464FF087018D
:1040C800324605F11C0301F0E7FDE06102B0BDE8EE
:1040D800F08100BF80B505464FF0000640F29C39DC
:1040E800C2F2000940F2E438C2F2000840F2963702
:1040F800C2F200071FE0FCF749FE2C6861682960DE
:104108004FF000026260237B062B0ED1216849F82C
:104118002610092E9CBF0136F6B2012E03D93A8823
:1041280002F101023A8088F80060FCF739FE236842
:104138000BB1A06898472B6803F1FF3010F1030F0B
:10414800D9D901F02BFC4FF00006F4E70260B3F177
:10415800FF3F18BF8360FF290ED145F6AC13C2F2AA
:1041680000031A6822B192F829304FEA530101E09E
:104178004FF007010173704701F07F010173704729
:1041880010B14FF000020260704700BF38B5044616
:10419800FCF7FCFD054640F2E633C2F200031A883C
:1041A80002F101021A80002C35D06368EBB940F2A5
:1041B800E830C2F20000028802F101020280207B8E
:1041C80040F2BC13C2F2000353F82010616043F8B8
:1041D8002040247B40F2C432C2F2000252F824008C
:1041E80001F00EFC4FF0010422E040F29230C2F2DE
:1041F8000000028802F101020280247B062C15D1FE
:1042080040F29831C2F200010B8803F101030B80E0
:104218004FF000040CE040F29430C2F20000018834
:1042280001F1010101804FF0000401E04FF00004AA
:104238002846FCF7B5FD204638BD00BF10B504463A
:1042480040F2A450C2F200004FF000014FF01802F3
:1042580012F000FDD4B140F20840C2F200004FF065
:1042680000014FF0300212F0F5FC40F28440C2F237
:1042780000004FF000014FF0180212F0EBFC40F282
:104288007C43C2F200034FF002021A7010BD00BF57
:1042980038B549F60C23C0F6010353F8205040F214
:1042A8003C41C2F2000151F8204049F63C22C0F6D8
:1042B8000102105CFDF78CFA2840A04214BF0020D0
:1042C800012038BD49F63C23C0F601031A5C40F2D0
:1042D8008441C2F2000151F8222049F60C23C0F6AD
:1042E800010353F8200002420CBF00200120704750
:1042F80070B440F2D073C2F2000353E8002F02F109
:10430800010243E800210129F7D049F63C22C0F612
:104318000102155C40F2A451C2F2000151F8254097
:1043280049F60C26C0F6010656F8202024EA0200B9
:1043380041F8250053E8005FA5F1010543E8005660
:10434800012EF7D053E8005FB5F1004F0DD14FF0C3
:10435800000543E80056012EF4D04EF60450CEF284
:104368000000016841F080510160BFF32F8F1442B3
:104378000CBF0020012070BC704700BF49F64823DD
:10438800C0F60103185C704710B50446FDF720FA23
:1043980040F2DC13C2F2000353F82410484010BD69
:1043A80010B504464FF00100FFF748FF40F23843CC
:1043B800C2F200031C7049F65420C0F6010050F800
:1043C800342040F28041C2F200010A6000EBC404CC
:1043D800606840F29C43C2F20003186010BD00BF41
:1043E80000B585B04FF00000FFF7DAFF4FF000038B
:1043F800009340F2A042C2F2000201924FF0400046
:10440800029049F63020C0F601004FF0020144F254
:10441800BD42C0F6000201F02BFB40F2A053C2F2ED
:104428000003186005B000BD2DE9F00180460028A2
:104438003CD04FF000034FEA8302086850F823404D
:104448004D6855F8236086EA0407886850F82350B9
:1044580084EA050C4CEA07076FEA070CC86850F8AD
:10446800235026EA050707EA0C0705EA0C0C66EA5A
:104478000C06354040F82350CD6855F823003843E2
:1044880045F823000D6955F82300384345F8230003
:104498004D690DB145F8237048688558886885507E
:1044A8004868845003F101034345C4D1BDE8F001D5
:1044B800704700BF2DE9F84340F28048C2F2000877
:1044C80040F2EC36C2F2000640F2F034C2F20004C8
:1044D8004FF0000540F29C47C2F20007D8F80000F0
:1044E80000EB800001F022FC3368002B40F0538180
:1044F800204629464FF0180212F0ACFB4BE14FF072
:10450800060049F6F411C0F60101FFF78DFF40F2ED
:104518007C41C2F200010A785AB102F1FF3040F240
:104528007C43C2F20003187040F2A451C2F20001A9
:104538000D6040F27842C2F200021068E8B940F219
:104548007843C2F200031D6040F23941C2F2000113
:104558000A784AB940F27842C2F20002106860B1A3
:1045680028460CF047F808E040F27840C2F2000014
:10457800036843F000610160ECE740F27C43C2F25B
:104588000003197859B101F1FF3040F27C42C2F2C0
:104598000002107040F2A453C2F200035D6040F2C2
:1045A8007841C2F200010868E8B940F27842C2F2E4
:1045B8000002156040F23943C2F20003197849B984
:1045C80040F27841C2F20001086860B128460CF058
:1045D80011F808E040F27840C2F20000026842F0A8
:1045E80000630360ECE740F27C42C2F200021378F9
:1045F8005BB103F1FF3140F27C40C2F20000017070
:1046080040F2A452C2F20002956040F27843C2F22E
:1046180000031968E9B940F27840C2F20000056069
:1046280040F23942C2F2000213784BB940F27843A3
:10463800C2F20003196861B128460BF0DBFF08E0FD
:1046480040F27841C2F20001086840F000620A6056
:10465800ECE740F27C40C2F2000002785AB102F165
:10466800FF3340F27C41C2F200010B7040F2A450CB
:10467800C2F20000C56040F27842C2F2000213683C
:10468800EBB940F27841C2F200010D6040F23940C6
:10469800C2F2000002784AB940F27842C2F200023F
:1046A800136863B128460BF0A5FF08E040F2784391
:1046B800C2F20003196841F000601860ECE740F2AC
:1046C8007C41C2F20001087858B100F1FF3340F292
:1046D8007C42C2F20002137040F2A451C2F20001FF
:1046E8000D6140F27840C2F200000368EBB940F275
:1046F8007842C2F20002156040F23941C2F200016C
:10470800087848B940F27840C2F20000036863B103
:1047180028460BF06FFF08E040F27843C2F200032E
:104728001A6842F000611960ECE740F27C42C2F27C
:104738000002117859B101F1FF3040F27C43C2F216
:104748000003187040F2A452C2F20002556140F210
:104758007841C2F200010868D8B940F27843C2F241
:1047680000031D6040F23942C2F20002117839B1EB
:1047780040F27840C2F20000036843F00062026031
:1047880040F27841C2F20001086810B128460BF0E7
:1047980031FF3560A2E6D4F800902846FFF7F4FD13
:1047A80040EA09012160D4F804904FF00100FFF7B6
:1047B800EBFD40EA09026260D4F808904FF002006D
:1047C800FFF7E2FD40EA0900A060D4F80C904FF032
:1047D8000300FFF7D9FD40EA0903E360D4F810901D
:1047E8004FF00400FFF7D0FD40EA09012161D4F839
:1047F80014904FF00500FFF7C7FD40EA0902626117
:10480800306800F1010030603B689842FFF466AE02
:1048180075E600BF00B585B04FF00003009340F285
:10482800E852C2F2000201924FF04000029049F6AD
:104838008430C0F601004FF0060144F65D02C0F670
:10484800000201F015F940F2BC53C2F200031860EF
:1048580005B000BD2DE9F04F85B040F234731F4616
:10486800C2F2000740F204700646C2F2000640F2A7
:10487800D051C2F20001029101F090F83A68002A82
:10488800FAD014E1A359002B51D02846FFF77CFD3C
:10489800029962586050904349D0A35910EA030224
:1048A80045D0039991F800E049F68C39C0F6010922
:1048B8004FEA451840F2C051C2F200014FF6FF7CA2
:1048C80049F6842AC0F6010A40F2EC6BC2F2000BEA
:1048D800204674468646C2F10003134022EA0302CA
:1048E8001CB95EF80B0003421ED1180E04D01AF84A
:1048F800003003F118030DE0180C04D01AF800304A
:1049080003F1100306E0180A1ABF1AF8003008333A
:104918001AF80330434419F8033031F8130060459E
:104928001CBF013021F81300002AD4D1744605F1C8
:10493800010504F10404062DA4D1019D6A1E01920B
:1049480040F0AC8003990C7804F10104E3B20B70D9
:104958000B2B03D14FF000050D7002E0002B40F047
:104968009A8040F21C72C2F20002116891B16FEA9B
:10497800010433682340336040F2EC60C2F2000067
:1049880005682C40046040F21C71C2F200014FF02F
:1049980000020A6040F21C74C2F20004636893B11A
:1049A8006FEA030075680540756040F2EC62C2F278
:1049B800000251680840506040F21C74C2F20004C2
:1049C8004FF00003636040F21C70C2F2000085687B
:1049D80095B16FEA0504B2682240B26040F2EC6318
:1049E800C2F2000399680C409C6040F21C70C2F24D
:1049F80000004FF00005856040F21C74C2F200040C
:104A0800E26892B16FEA0203F1681940F16040F27E
:104A1800EC60C2F20000C5682B40C36040F21C7411
:104A2800C2F200044FF00002E26040F21C73C2F2CE
:104A38000003196991B16FEA0100356905403561D4
:104A480040F2EC64C2F2000422691040206140F296
:104A58001C73C2F200034FF00001196140F21C7090
:104A6800C2F20000456995B16FEA050472692240F7
:104A7800726140F2EC63C2F2000359690C405C6158
:104A880040F21C70C2F200004FF0000545614FF47F
:104A9800FA74019402E04FF4FA7001904FF00100AB
:104AA80001F044F93A68002A3FF4E6AE07E04FF413
:104AB800FA74019440F2E865C2F2000503954FF0DC
:104AC80000042546DEE600BF10B54FF0000440F2B2
:104AD8003473C2F200031C6040F2EC60C2F20000C2
:104AE80021464FF00602FCF70BF940F20470C2F2BF
:104AF800000021464FF00602FCF702F940F21C7054
:104B0800C2F2000021464FF00602FCF7F9F840F225
:104B1800D050C2F2000021464FF00602FCF7F0F830
:104B280040F2C050C2F2000021464FF0100212F0CD
:104B380091F840F2E860C2F20000047010BD00BFB6
:104B480070B549F63C23C0F601031B5C49F60C22FC
:104B5800C0F6010252F8202040F23470C2F2000080
:104B6800046840F20475C2F2000555F823001042AB
:104B780006D104F1010640F23475C2F200052E6038
:104B880049B140F2EC61C2F2000151F823501543DB
:104B980041F8235009E040F2EC61C2F2000151F8FB
:104BA800235025EA020541F82350104340F20471CE
:104BB800C2F2000141F8230040F21C71C2F2000168
:104BC80051F8230020EA020241F8232034B940F2C8
:104BD800BC53C2F20003186800F012FF70BD00BF9A
:104BE80030B449F63C23C0F601031B5C49F60C229D
:104BF800C0F6010252F8202040F20470C2F2000010
:104C080050F82300104229D040F23474C2F2000454
:104C1800256805F10105256071B140F21C71C2F2E9
:104C2800000151F82340144341F8234040F2E86161
:104C3800C2F20001097889B96FEA020240F2EC6118
:104C4800C2F2000151F82340144041F823400240C9
:104C580040F20470C2F2000040F8232030BC7047D4
:104C680030B4034640F2D072C2F2000252E8000F9C
:104C780000F1010042E80004012CF7D040F2C050D6
:104C8800C2F2000030F8132039B140F2C051C2F22C
:104C980000014FF0000421F8134040F2D073C2F233
:104CA800000353E8004FA4F1010443E80045012D37
:104CB800F7D053E8004FB4F1004F0DD14FF0000486
:104CC80043E80045012DF4D04EF60450CEF2000022
:104CD800016841F080510160BFF32F8F104630BC4E
:104CE800704700BF40F2E863C2F200031878D0F1C1
:104CF800010038BF002070472DE9F84FDFF83481F4
:104D08004B4FC8EB07004FEAD00707F101074FF0F8
:104D1800000540F2982AC0F6000A40F26039C0F651
:104D2800000931E044464FF000066FEA060B0BEB32
:104D3800070101F0010B58F8043CAB4229D135E0DA
:104D480054F8043CAB4205D154F8080C8047FCF7F2
:104D580037FF0BE0FF2B09D9FF2D07D154F8040CBE
:104D68004FF0070154F8082C00F0A2FF06F10106E5
:104D780004F1080454F8041CA94240D14CE005F1A0
:104D88000105B5F5807F02D0CA45CBD3F7E7BDE86A
:104D9800F88FFF2B0FD9FF2D0DD158F8040C4FF0C9
:104DA800070158F8082C00F083FF04E058F8082C95
:104DB8009047FCF705FF06F1010604F10804BE421E
:104DC800DDD0BBF1000FBBD054F8040CA8420AD0C8
:104DD800FF280DD9FF2D0BD14FF0070154F8082CEF
:104DE80000F066FF04E054F8081C8847FCF7E8FE6A
:104DF80006F1010604F10804BE42A1D1BFE7FF296C
:104E08000FD9FF2D0DD154F8040C4FF0070154F8B9
:104E1800082C00F04DFF04E054F8082C9047FCF7EC
:104E2800CFFE06F1010604F10804BE4288D1A6E7C8
:104E380067030008A0020008027840F29D73C2F2DE
:104E480000031B789A4206D34FF0000202700878DC
:104E580000F1010008700A7840F29E73C2F2000364
:104E68001878824224BF00200870704710B5A0F15E
:104E78000803052B3DD8DFE803F01F3C2C3C038AD0
:104E880040F23C70C2F200004FF020014FF0540293
:104E980011F0E0FE40F29070C2F200004FF0FF31D6
:104EA8004FF00C0211F0D6FE40F2A470C2F20000DE
:104EB800026802F1010202604FF0000140F238730B
:104EC800C2F20003197040F23970C2F2000001709A
:104ED8005DE040F23871C2F200014FF000030B7040
:104EE80040F23970C2F20000027802F10102027049
:104EF80043E040F23872C2F20002127840F239718F
:104F0800C2F200010B7840F29D71C2F200010978EB
:104F180001FB032340F23C71C2F20001C95C8142EB
:104F280006D140F2A071C2F20001097806291DD10C
:104F380040F23C74C2F20004E0544FEA531040F2CD
:104F48009071C2F2000103F01F034FF0010404FA4C
:104F580003F351F820401C4341F8204040F2A4706C
:104F6800C2F20000016801F10101016002F10102D1
:104F780040F23873C2F200031A7040F23870C2F27D
:104F8800000040F23971C2F20001FFF755FF4FF0FF
:104F9800000010BD70B4039D049C064628B140F281
:104FA800A070C2F200000078307029B140F2A870F9
:104FB800C2F20000007808702AB140F29C71C2F277
:104FC8000001087810702BB140F2A972C2F20002F9
:104FD800117819702DB140F23873C2F200031878B5
:104FE80028702CB140F23972C2F200021178217097
:104FF80070BC704707281DD8002808BF052040F25C
:10500800A073C2F20003187049F64C43C0F60103BE
:1050180013F8101040F29D72C2F20002117003EBF7
:105028004000417840F29E73C2F2000319704FF0BD
:10503800010070474FF00000704700BF08B540F20C
:10504800A873C2F200034FF001021A704FF0050076
:10505800FFF7D0FF4FF00C004FF00001FFF706FFFD
:1050680008BD00BF08B540F23872C2F200021070E5
:1050780040F23973C2F20003197010461946FFF75F
:10508800DBFE08BD034628B140F29D70C2F2000065
:105098000078187029B140F29E73C2F200031878A4
:1050A80008702AB140F2A471C2F200010B681360C3
:1050B80040F23C70C2F20000704700BF2DE9F001D9
:1050C80040F23C77C2F200073F1853284BD8002A19
:1050D80049D03B4607F1010702F1FF3257FA82F740
:1050E8004FF0000640F29074C2F200044FF0010540
:1050F8006FEA030C0CEB070202EA050C13F8018BAC
:1051080001F1FF3111F8012F90452FD13DE013F83F
:1051180001CB01F1010049788C450ED003F8011C40
:105128004FEA521102F01F0605FA06FC54F82160F6
:105138004CEA060644F821602E4602F10102D2B27A
:10514800542A07D013F801CB00F1010140788445B7
:1051580042D150E03EB140F2A473C2F20003196894
:1051680001F101011960BDE8F001704703F8012C55
:105178004FEA501600F01F0805FA08F854F82620E0
:1051880048EA020244F826202E4600F10100C2B285
:10519800542ADFD0BB42DDD0BCF1000FB7D013F8E2
:1051A80001CB11F8010F84450ED003F8010C4FEA2A
:1051B800521002F01F0605FA06FC54F820604CEA6B
:1051C800060644F820602E4602F10102D2B2542AA3
:1051D800C0D0BB429BD1BDE703F8010C4FEA521087
:1051E80002F01F0605FA06FC54F820604CEA060691
:1051F80044F820602E4602F10102D2B2542AA9D006
:10520800BB4284D1A6E700BF003018BF012040F29E
:10521800A873C2F200031870003118BF012140F2D0
:105228009C70C2F200000170003218BF012240F2E7
:10523800A973C2F200031A70704700BF40F29F734F
:10524800C2F200034FF000021A7070474FF054008A
:10525800704700BF40F29F73C2F200034FF0010293
:105268001A707047034628B10868834214BF0020AB
:10527800012070474FF00000704700BF10B440F2A3
:10528800D073C2F2000353E8002F02F1010243E891
:1052980000210129F7D00468C4B16268824202D1B2
:1052A8009268626002E0436881689960236883427B
:1052B80002D15B68236002E0826841685160A2689D
:1052C80002F1FF31A1604FF00004046040F2D07396
:1052D800C2F2000353E8002FA2F1010243E80024C0
:1052E800012CF7D053E8002FB2F1004F0DD14FF049
:1052F800000243E80024012CF4D04EF60450CEF20C
:105308000000016841F080510160BFF32F8F10BC8D
:10531800704700BF38B504460D464FF000014FF006
:10532800100211F097FCE56038BD00BFF8B50446DF
:105338000F46C6688D192946FFF794FF00283CD10F
:1053480040F2D073C2F2000353E8002F02F10102C9
:1053580043E800210129F7D04FF000006860616838
:10536800A96001B14D60226802B925606560BC5131
:10537800A36803F10103A36040F2D073C2F20003F3
:1053880053E8002FA2F1010243E80024012CF7D0D2
:1053980053E8002FB2F1004F0DD14FF0000243E85F
:1053A8000024012CF4D04EF60450CEF2000001681F
:1053B80041F080510160BFF32F8FF8BD2DE9F04116
:1053C80004468846C6688D199719C2B940F2D07349
:1053D800C2F2000353E8002F02F1010243E8002162
:1053E8000129F7D002686A6005604FF00000A860E4
:1053F800616809B9656020E06B689D601DE0394609
:10540800FFF730FF00283FD02846FFF737FF40F26C
:10541800D073C2F2000353E8002F02F1010243E8FF
:1054280000210129F7D0B868A8606F60BD602168C5
:10543800B9420EBF2560A9684D6048F80640A268C9
:1054480002F10102A26040F2D073C2F2000353E8F5
:10545800002FA2F1010243E80024012CF7D053E801
:10546800002FB2F1004F0DD14FF0000243E80024A5
:10547800012CF4D04EF60450CEF20000016841F041
:1054880080510160BFF32F8FBDE8F081C368C91850
:10549800486808B1C01A70474FF00000704700BF55
:1054A800036813B1C068181A70474FF000007047BE
:1054B80008B5C368C918FFF7D5FE08BD08B5C068A8
:1054C8000818FFF7DBFE08BD08B540F2AC70C2F261
:1054D80000004FF01C01FFF71DFF08BD70B5054621
:1054E80000F108063046FFF7DBFF0446686050B15C
:1054F80030462146FFF7E2FF4FF00100A861204641
:1055080000F07EFA70BD4FF00003AB6170BD00BFC4
:1055180038B504460D464FF000014FF0280211F04F
:1055280099FB204640F8085B4FF01C01FFF7F2FE9C
:1055380040F2AC70C2F200002146FFF7F7FE38BD1A
:105548002DE9F0410746884645F6AC13C2F2000340
:105558001868002800F0FE8040F2D074C2F20004FF
:1055680054E8002F02F1010244E800210129F7D094
:10557800796831B145F6AC12C2F20002136899425B
:105588002ED145F6AC10C2F2000004687C60B969FF
:1055980001F10101B96140F2D073C2F2000353E88E
:1055A800002FA2F1010243E80024012CF7D053E8B0
:1055B800002FB2F1004F0DD14FF0000243E8002454
:1055C800012CF4D04EF60450CEF20000016841F0F0
:1055D80080510160BFF32F8F4FF00100BDE8F081CB
:1055E800B8F1FF3F24D140F2D073C2F2000353E870
:1055F800002FA2F1010243E80024012CF7D053E860
:10560800002FB2F1004F0DD14FF0000243E8002403
:10561800012CF4D04EF60450CEF20000016841F09F
:1056280080510160BFF32F8F4FF00000BDE8F0817B
:1056380007F108052846FFF733FF0246F0B145F6A3
:10564800AC16C2F20006306892F8294090F829108A
:105658008C4208D912E0336892F8290093F829405F
:10566800A04204D90AE045F6AC16C2F20006284664
:105678001146FFF70BFF02460028ECD1284645F6F5
:10568800AC11C2F200010968FFF798FE40F2D0762B
:10569800C2F2000656E8002FA2F1010246E80024F3
:1056A800012CF7D056E8002FB2F1004F0DD14FF082
:1056B800000246E80024012CF4D04EF60450CEF245
:1056C8000000016841F080510160BFF32F8FB8F1ED
:1056D800000F04D008EB880000F028FB01E000F080
:1056E8005DF940F2D074C2F2000454E8003F03F1BF
:1056F800010344E80032012AF7D045F6AC16C2F29D
:10570800000628463168FFF7D9FE54E8003FA3F1A8
:10571800010344E80032012AF7D054E8003FB3F10E
:10572800004F0DD14FF0000344E80032012AF4D0B5
:105738004EF60450CEF20000016841F0805101603D
:10574800BFF32F8F78683268904214BF0020012081
:10575800BDE8F0814FF00100BDE8F08110B50446C6
:1057680045F6AC13C2F200031868002860D06268DE
:10577800904201D0FBF762FA40F2D073C2F2000304
:1057880053E8002F02F1010243E800210129F7D074
:10579800A16901F1FF30A06118B340F2D073C2F2E1
:1057A800000353E8002FA2F1010243E80024012C72
:1057B800F7D053E8002FB2F1004F0DD14FF000029F
:1057C80043E80024012CF4D04EF60450CEF2000039
:1057D800016841F080510160BFF32F8F4FF0000046
:1057E80010BD2046FFF77AFE40F2D073C2F20003E4
:1057F80053E8002FA2F1010243E80024012CF7D05E
:1058080053E8002FB2F1004F0DD14FF0000243E8EA
:105818000024012CF4D04EF60450CEF200000168AA
:1058280041F080510160BFF32F8F4FF0010010BD90
:105838004FF0010010BD00BFF8B5054640F2D07327
:10584800C2F2000353E8002F02F1010243E80021ED
:105858000129F7D040F2AC70C2F20000FFF720FE39
:105868000446E0B140F2AC77C2F200076068A84293
:1058780003D12046FFF732FE0AE004F1080630465D
:105888002946FFF715FE18B130462946FFF716FEE0
:1058980038462146FFF7FAFD04460028E6D140F2D3
:1058A800D073C2F2000353E8002FA2F1010243E8CB
:1058B8000024012CF7D053E8002FB2F1004F0DD18E
:1058C8004FF0000243E80024012CF4D04EF60450B7
:1058D800CEF20000016841F080510160BFF32F8FC4
:1058E800F8BD00BF08B549F65C43C0F60103195C72
:1058F800012906D011B102290BD105E0FDF72EFED2
:1059080008BD02F00FF908BDFBF798F94FF0000049
:1059180008BD4FF0000008BD4EF60453CEF2000358
:105928001A6842F080501860704700BF4FF00102BB
:1059380080F8282040F2CC73C2F2000390F82910B6
:1059480002FA01F2188802431A80704710B440F234
:10595800C873C2F200031A68C2B1904213D104E0BE
:1059680088420FD102F1140203E040F2C872C2F279
:10597800000243691BB19C69816961189961436997
:10598800136003E00A4651690029E9D14FF000028B
:1059980082614FF0FF31416110BC704710B5FBF7D1
:1059A800F5F9044645F6AC13C2F20003186890F8FE
:1059B8002820032A1BD0FBF7E9F945F6AC13C2F2FD
:1059C800000319684FF0000281F8282091F8292077
:1059D800096940F6BC03C2F2000343F82210FBF742
:1059E800DFF92046FBF7DCF9FFF796FF10BD4FF013
:1059F800020180F828102046FBF7D2F910BD00BF3D
:105A080038B5044690B3036883B3FBF7BFF905467E
:105A180094F8280010BB2046FFF788FF45F6AC1124
:105A2800C2F200010B6843B194F8292093F82900C9
:105A380020F00101531A002B15DA40F2D072C2F29D
:105A48000002106838B140F0004140F2D073C2F251
:105A58000003196007E0FFF75FFF04E0022804BFB6
:105A6800032084F828002846FBF79AF938BD00BFC0
:105A78002DE9F04F85B006460F46934698460F9D90
:105A8800DDF84090FBF782F9824640F61403C2F233
:105A980000031968504881420FD248F20002C2F24E
:105AA800000252F82C4C54B14C4B1C468B4207D97F
:105AB80053F82C090028F8D102E0474C00E0464C86
:105AC800A14206D1A1F12C0140F61402C2F2000253
:105AD800116020464FF000014FF02C0211F0BAF887
:105AE8004FF0FF3161611EB949F66056C0F60106F4
:105AF8002660B8F1000F08D00E9B042B08D9184671
:105B080000F103004FEA900604E04FF0000601E0C0
:105B18004FF000060DBB46F2B049C2F2000940F250
:105B2800BC75C2F20005296845F69570C0F60000FC
:105B38000090CDF80480029648464FF000025B467C
:105B4800FBF75CFC2A68A260E0604FEA800153180A
:105B58002B60C1EB0900606020E028464FF0FF3160
:105B68004A46FBF7CDF84AF2ED52CDF6CE622A60EE
:105B7800E56005EB8905656045F69571C0F600019D
:105B88000091CDF804800296284629464FF001027C
:105B98005B46FBF733FCA5EB800363606FEA070203
:105BA800C2F3C01101EB470707F0FF0784F829701B
:105BB80040F2D473C2F2000353F82700206143F87F
:105BC80027405046FBF7ECF82046FFF719FF204620
:105BD80005B0BDE8F08F00BFD47F0020A87F00206B
:105BE80030B585B04FF0000145F6AC13C2F20003A2
:105BF8001960284C48F20005C2F200052A1B20460D
:105C08004FEAA202FBF77CF840F2BC70C2F2000037
:105C18000460A5F12C0540F61401C2F200010D60E4
:105C280045F6B043C2F200034FF0B504CBF26B1453
:105C38001C6003F14C004FF0FF3243F8042F43F887
:105C4800042F43F8042F8342F9D14FF00004009445
:105C580040F61801C2F2000101914FF028030293A7
:105C680049F66C50C0F601004FF0070145F6155291
:105C7800C0F600022346FFF7FBFE40F6B802C2F268
:105C88000002106040F2D470C2F20000C46305B094
:105C980030BD00BFB464002010B584B0069C0094E9
:105CA8004FF0000401940294FFF7E2FE04B010BD27
:105CB80000B585B04FF00003009301930293FFF7FE
:105CC800D7FE05B000BD00BF38B545F6AC13C2F22B
:105CD80000031868C0B1FBF759F8054645F6AC143F
:105CE800C2F200042068FFF721FE216891F82920FC
:105CF800086940F6BC03C2F2000343F822002846B4
:105D0800FBF74EF8FFF708FE38BD00BF38B545F67B
:105D1800AC15C2F2000540F2D474C2F200042B683C
:105D280022681A61FFF7D0FFF9E700BF38B545F6DA
:105D3800AC13C2F200031968002900F0918020B961
:105D4800FFF7C2FF4FF001029AE0B0F1FF3F04D124
:105D5800FFF724FE4FF0000292E040F2D074C2F246
:105D6800000454E8002F02F1010244E8002101294F
:105D7800F7D040F2C872C2F200021568002D7AD03E
:105D8800AB6998426FD3C01A05F114016D691DB152
:105D9800AB698342F7D96AE045F6AC15C2F2000553
:105DA8002B689861086858611846FAF74BFF40F26B
:105DB800D074C2F2000454E8003FA3F1010344E8A0
:105DC8000032012AF7D054E8003FB3F1004F0DD15B
:105DD8004FF0000344E80032012AF4D04EF6045094
:105DE800CEF20000016841F080510160BFF32F8FAF
:105DF800FFF7D4FD54E8003F03F1010344E8003203
:105E0800012AF7D028684169B1F1FF3F04D0FFF7B4
:105E18009DFD4FF0000201E04FF0010240F2D07307
:105E2800C2F2000353E8004FA4F1010443E800451F
:105E3800012DF7D053E8004FB4F1004F0DD14FF0CA
:105E4800000443E80045012DF4D04EF60450CEF28C
:105E58000000016841F080510160BFF32F8F0FE00F
:105E68004FF001020CE040F2C871C2F20001AC69C7
:105E7800221AAA6190E740F2C871C2F200018BE7CA
:105E8800104638BDF8B5044600287AD0FAF77EFFE8
:105E9800064640F61403C2F20003196839488142E5
:105EA80011D248F20002C2F2000252F81C5CA5426C
:105EB80063D0354B1D468B4205D9A3F12C03D86B13
:105EC800A042F7D15AE094F8293040F2D472C2F2D5
:105ED800000252F82300A04206D1016940F2D472B0
:105EE800C2F2000242F823102046FFF72FFD204699
:105EF800FFF7A2FC94F82900236940F6BC01C2F21E
:105F0800000141F8203045F6AC12C2F200021068D8
:105F1800A04229D0A06838B3E76800EB870540F2B3
:105F2800BC77C2F200073B685A1B29464FEAA20217
:105F38004FF00003FCF73CF9E1683868A0EB8103F7
:105F48003B6040F61402C2F2000211680D4B994200
:105F58000AD29A68954203D8E068A2EB80029A6058
:105F6800A3F12C038B42F4D84FF00001216084F890
:105F780028103046FAF714FFF8BD024D216929614F
:105F8800A1E7F8BDD47F0020A87F002000BFF0471C
:105F980072B645F6AC14C2F200042068FFF772FF2F
:105FA8004FF000032360FBF779FA00BF40F2C87393
:105FB800C2F20003196849B1886950B100F1FF3293
:105FC8008A61D2F1010038BF002070474FF000000D
:105FD80070474FF00000704770B540F2C873C2F2C6
:105FE80000031C68A4B1A06990B940F2C875C2F258
:105FF80000054FF0FF3660692946FAF723FE66610F
:106008002046FFF7FDFC2C6814B1A1690029F2D0E5
:1060180070BD00BFF0B472B640F2CC73C2F2000398
:106028001C882CB940F6B803C2F2000318685FE078
:1060380049F6604CC0F6010C40F6BC05C2F20005FA
:1060480040F2D476C2F20006C4F1000323401A0AD3
:106058001ABF1CF8021008311CF8031011F0010FC8
:106068000AD141F0010055F8200038B190F82820F5
:10607800012A38D81F4602E01F4600E01F4655F89F
:106088002120B2B192F828307BB140F2CC70C2F234
:106098000000048010462BE090F8283033B140F21D
:1060A800CC72C2F20002148022E010460069002877
:1060B800F2D156F82100824207D1BC43C4D140F244
:1060C800CC71C2F200010C80ACE745F8210011F058
:1060D800010FD4D114EA4703D1D04FEA4707BFB222
:1060E80041F00101CBE740F2CC71C2F200010C8013
:1060F80062B6F0BC704700BF70B545F6AC13C2F28B
:1061080000031B6883420FD193F82820012A9CBF03
:10611800022283F8282093F8291040F6BC00C2F226
:10612800000040F8213070BD40F2C072C2F2000297
:10613800136045F6AC11C2F20001086090F82920FE
:1061480040F6BC03C2F2000343F8220090F828107E
:1061580001299CBF022180F828108268AAB9C16869
:106168004AF2ED53CDF6CE630868984201D0FAF7AB
:1061780065FD45F6AC12C2F2000211684868CB68AA
:1061880098427ED2FAF75AFD70BD40F2C473C2F24B
:1061980000031B68984274D093B3586846F2B04421
:1061A800C2F20004251A4FEAA501D96045F6B042AB
:1061B800C2F2000290420AD34FF0B503CBF26B1340
:1061C80045F6B040C2F2000004689C4201D0FAF7DC
:1061D80035FD40F2C475C2F200052A6840F2BC746D
:1061E800C2F2000420685168D2684FF00003FBF740
:1061F800DFFF296823688B60C86803EB8002226090
:1062080045F6AC11C2F200010B6840F2C470C2F24C
:1062180000000360DA68002A33D0586899684FF0A4
:106228000103FBF7C5FF45F6AC16C2F20006356858
:10623800A868EC6800EB840440F2BC76C2F2000661
:106248003268131B21464FEAA3024FF00003FBF705
:10625800AFFFE9683068A0EB8102326040F61403B2
:10626800C2F200031968074B99420AD29A6894420D
:1062780003D8E868A2EB80029A60A3F12C038B4252
:10628800F4D870BDD47F002000B585B040F6582002
:10629800C2F200004FF00001FFF73CF840F6001092
:1062A800C2F200004FF00001FFF734F84FF000038E
:1062B800009340F61812C2F2000201924FF050000B
:1062C800029049F67450C0F60100194646F2E552AC
:1062D800C0F60002FFF7CCFB40F6FC03C2F2000355
:1062E800186005B000BD00BF08B5FFF7D9F8034630
:1062F80048B1C06850B100F1FF31D960D1F1010057
:1063080038BF002008BD4FF0000008BD4FF0000066
:1063180008BD00BF70B505460E46144640F2D0735E
:10632800C2F2000353E8002F02F1010243E8002102
:106338000129F7D0FFF7B4F80246002839D0C06821
:1063480084422DD3241A28461146FFF79FF80246A7
:1063580000282ED0C068A042F4D921E040F2D073C2
:10636800C2F2000353E8002FA2F1010243E800241F
:10637800012CF7D053E8002FB2F1004F0DD14FF0A8
:10638800000243E80024012CF4D04EF60450CEF26B
:106398000000016841F080510160BFF32F8F70BD8C
:1063A800F460D1680B1BD36028463146FFF706F826
:1063B800D4E7F46028463146FEF7B8FFCEE700BFC1
:1063C800F8B50646FFF76CF80446F8B1C368EBB9B0
:1063D80030462146FFF75AF80546FAF7D7FC074634
:1063E80030462146FFF76AF83846FAF7D9FC2269A1
:1063F8001AB130462146FFF78DFF04F11400FDF76E
:10640800C5FE1DB12C46E8680028E1D0F8BD00BFE4
:1064180008B540F61413C2F200031A6802F101022B
:106428001A6040F60010C2F20000FFF75DFF28B1C5
:1064380040F60010C2F20000FFF7C2FF08BD00BF1F
:1064480008B5014640F65820C2F20000FFF730F8C0
:1064580020B140F65820C2F2000008BD40F60010F6
:10646800C2F2000008BD00BF70B5044640F2D07308
:10647800C2F2000353E8002F02F1010243E80021B1
:106488000129F7D0FFF7DCFF05462146FFF710F892
:10649800002845D040F2D070C2F2000050E8002F2A
:1064A80002F1010240E800210129F7D028462146DF
:1064B800FEF7ECFF18B1C168E2688B18C360FAF701
:1064C80065FC064628462146FEF7F8FF3046FAF7EF
:1064D80067FC4FF0FF35E56040F2D073C2F200036D
:1064E80053E8002FA2F1010243E80025012DF7D05F
:1064F80053E8002FB2F1004F0DD14FF0000243E8EE
:106508000025012DF4D04EF60450CEF200000168AB
:1065180041F080510160BFF32F8F4FF0010501E07A
:106528004FF0000504F11400FDF72AFE40F2D07385
:10653800C2F2000353E8002FA2F1010243E800244D
:10654800012CF7D053E8002FB2F1004F0DD14FF0D6
:10655800000243E80024012CF4D04EF60450CEF299
:106568000000016841F080510160BFF32F8F284679
:1065780070BD00BF2DE9F04105460F461446984608
:10658800FFF772FF064694B19DF82030002B14BF28
:1065980020460020286105F114004146069A079B11
:1065A800FDF7D4FD384629462246FFF7B3FE3046AC
:1065B800BDE8F08170B584B00E4615460093089C7E
:1065C80001949DF82430029340F65821C2F200014C
:1065D80032462B46FFF7CEFF04B070BD00B583B03E
:1065E8004FF0000300934FF00100019040F668203F
:1065F800C2F2000041F288314FF0FF0246F219431F
:10660800C0F60003FFF7D6FF40F65824C2F2000494
:10661800FFF7E2FC2046FFF7D3FEFFF7BFF9F7E7E5
:1066280040F61013C2F2000318681A689042FBD1B2
:10663800704700BF10B540F61013C2F200031A6885
:1066480002F101021A60FFF7B1FC044640F6582037
:10665800C2F20000FFF748FE204310F0FF0F06D0FB
:1066680040F6FC00C2F200000068FFF7C9F910BD4F
:1066780008B549F68050C0F601004FF0060146F60D
:10668800B522C0F60002FFF713FB40F69853C2F29A
:106698000003186008BD00BF38B504460D4640F633
:1066A800CC23C2F20003586AA0420AD040F6CC219B
:1066B800C2F200014C620A681AB115B14948FDF7E7
:1066C80065FD40F6CC23C2F20003186F84420AD05D
:1066D80040F6CC21C2F200010C67CA6C1AB115B1A0
:1066E8004148FDF753FD40F6CC23C2F20003D3F82E
:1066F800BC0084420CD040F6CC21C2F20001C1F8A3
:10670800BC40D1F898201AB115B13848FDF73EFDC4
:1067180040F6CC23C2F20003D3F8080184420CD01F
:1067280040F6CC21C2F20001C1F80841D1F8E420BA
:106738001AB115B12E48FDF729FD40F6CC23C2F257
:106748000003D3F8540184420CD040F6CC21C2F2A5
:106758000001C1F85441D1F830211AB115B12548CA
:10676800FDF714FD40F6CC23C2F20003D3F8A001D4
:1067780084420CD040F6CC21C2F20001C1F8A041FD
:10678800D1F87C211AB115B11B48FDF7FFFC40F682
:10679800CC23C2F20003D3F8EC0184420CD040F6BB
:1067A800CC21C2F20001C1F8EC41D1F8C8211AB1DC
:1067B80015B11248FDF7EAFC40F6CC23C2F20003FB
:1067C800D3F83802A0420CD040F6CC21C2F2000126
:1067D800C1F83842D1F814221AB115B10848FDF7AA
:1067E800D5FC38BDDC0A0020280B0020740B0020E3
:1067F800C00B00200C0C0020580C0020A40C00201A
:10680800F00C00202DE9F04707460D469146089800
:10681800DDF828800C683E68D8F800108A19944280
:1068280002D80219964203D304192C60BDE8F087F8
:10683800341B061BB14234BF8A46B246099931B1AE
:10684800D9F8000008181919524610F0DFF9D8F8DD
:106858000030CAEB0302C8F800203E6806EB0A01C4
:106868003960D9F8000000EB0A03C9F800302E6837
:10687800A41954442C60BDE8F08700BF70B584B0FB
:106888009CF81960157A947B4FF007038CF8103048
:106898004FF005028CF8112006F00F0260F3C712C2
:1068A8008CF812204FF0000065F301008CF81300FB
:1068B8004FF0000261F30A02ACF814208CF816407D
:1068C800DCF80C100093DCF804300193CDF808C014
:1068D80001F104000CF108020CF11003FFF792FF1C
:1068E80004B070BD2DE9F04F8FB0074605911446EE
:1068F8004FF000030793136012896068131A8B42E4
:1069080038BF05930599002900F0AA8040F69C55E8
:10691800C2F200052D6815B34FEAC5054FF0000215
:106928004FF0FF01134640F6A450C2F20000A5F153
:106938000806C6F3C00E1658F6798E4240F09580C8
:1069480096E01658F6798E421CBF0133314602F1A3
:1069580008028658F6798E4240F09F80A0E04FF0FA
:10696800000303EB43024FEAC20000F11000089055
:106978004FF48071ADF824104FF00402ADF82620D2
:106988008DF828300DF129004FF000014FF0070273
:1069980010F060F904F1040B04944FF01003009315
:1069A800019705A802905846214607AA08ABFFF7A9
:1069B80029FF0599002951D04FF001028DF82120B7
:1069C8000DF132004FF000014FF0060210F042F9CD
:1069D80040F69C53C2F20003186800283ED04FF0DE
:1069E800FF014FF0000440F6A459C2F2000949F62D
:1069F8009058C0F6010840F69C5AC2F2000A59F8AD
:106A08003450ED798D4223D08DF820404FEA051699
:106A18000DF1220008EB06014FF0080210F0F6F81D
:106A280006F108010DF12A0041444FF0080210F068
:106A3800EDF84FF018020092019705AB0293584603
:106A4800049907AA08ABFFF7DDFE059830B129467F
:106A580004F10104DAF80020A242D0D8079801E036
:106A68004FF0FF300FB0BDE8F08F03F1010331465E
:106A780002F10802AA423FF474AFBEF1000F3FF4DE
:106A880060AF1658F6798E421CBF0133314602F1C9
:106A98000802AA427FF455AF63E703F101033146C8
:106AA80002F10802AA427FF44CAF5AE72DE9F041FF
:106AB8004FF00100FDF73EFA49F61460C0F60100F8
:106AC800FDF7B4F840F6C453C2F200034FF00102D8
:106AD8001A7040F69450C2F20000016841B940F6BD
:106AE8009454C2F20004FEF759FF2568002DFAD02D
:106AF80040F6A257C2F2000740F6C454C2F200049E
:106B080040F62C56C2F2000640F6A155C2F2000526
:106B180040F69058C2F200083B783BB14FF00002B3
:106B28003A704FF002002070FDF74CF8317859B1F7
:106B38004FF000033370227862F07F0020704FF02E
:106B480001000146FFF7A8FD297851B14FF0000078
:106B58002870237803F07F0222704FF00101FFF7BD
:106B68009BFD98F8000010B9FEF718FFD4E740F62F
:106B7800C451C2F200014FF002030B704FF0000045
:106B8800FDF7D8F9BDE8F08108B540F69453C2F294
:106B98000003186040F69850C2F200000068FEF743
:106BA8002FFF08BD70B505460E4640F6E453C2F205
:106BB80000031868032801D9FAF740F840F6E452B0
:106BC800C2F20002116840F67054C2F2000444F8A0
:106BD800316004EBC104656001F10101116070BD11
:106BE80070B505460C461646032801D9FAF726F86B
:106BF80040F6A453C2F2000353F8350008B1FAF77F
:106C08001DF840F6A451C2F2000141F8354001EBED
:106C1800C5056E6040F69C53C2F200031A6802F183
:106C280001021A60206930B1FDF700F804F104048C
:106C380020690028F8D170BD08B540F6CC23C2F20F
:106C48000003196881425AD040F6CC22C2F20002F1
:106C5800D36C834234D040F6CC21C2F20001D1F883
:106C6800982082422FD040F6CC23C2F20003D3F8FA
:106C7800E41081422AD040F6CC22C2F20002D2F8B7
:106C88003031834225D040F6CC21C2F20001D1F840
:106C98007C21824220D040F6CC23C2F20003D3F8F4
:106CA800C81181421BD040F6CC22C2F20002D2F8B1
:106CB8001432834216D0F9F7C1FF4FF0080013E0F1
:106CC8004FF0010010E04FF002000DE04FF003001C
:106CD8000AE04FF0040007E04FF0050004E04FF031
:106CE800060001E04FF0070040F6CC21C2F2000197
:106CF8004FF04C0202FB001090F8200008BD4FF046
:106D08000000F1E72DE9F04F8FB0089007910A9243
:106D18004FF0000309931360546813891B1B8B42BF
:106D280038BF07930799002900F04A81082C69D8D1
:106D380040F69C54C2F20004D4F800E040F6E45552
:106D4800C2F200052E680EEBCE0707EBC60404F16D
:106D580009044FF0000140F6A457C2F20007CB59CE
:106D68008BB1DD68641903F110051B695BB15E899D
:106D78000EB104F107049B890BB104F1070455F81F
:106D8800043F002BF3D101F108012029E7D140F697
:106D98009451C2F200010D682F7E6E7EEB8A03F1DA
:106DA8000103C3F347054FF000010C914FF00903AD
:106DB8008DF82C304FF002018DF82D10ADF82E40D3
:106DC8008DF830E04FF001018DF831104FF00001DF
:106DD80067F3451166F3861161F07F018DF8331072
:106DE8008DF834500093019007A8029002F1040036
:106DF800114609AA0BABFFF705FD079A002A00F018
:106E0800DD80E0E04FF009001060DCE05BF8364020
:106E1800002C00F0CE80059D286800284BD07A68A9
:106E2800B2420CD04FF0000310F0010F3ED1DFE06A
:106E380007EBC3025268B24240F0E38001E04FF032
:106E4800000357F83300D2B290F8048090F805C0D8
:106E580090F806E0C579016819B143F01000C3B293
:106E680001E04FF000034FF008008DF82C004FF0C0
:106E78000B018DF82D108DF82E208DF82F808DF8B0
:106E880030C08DF831E08DF832508DF833300A99E2
:106E98000090089A019207AB029301F1040009AA35
:106EA8000BABFFF7AFFC079828B987E003F10105A2
:106EB8002B468542BCD104F1100523697BB12946D4
:106EC8004FF00002588908B102F101029B890BB109
:106ED80002F1010251F8043F002BF3D101E04FF019
:106EE80000025FFA86FCD2B294F804E06079A179D6
:106EF80023681BB146F02003DBB201E04FF000032A
:106F08008DF82CA04FF004088DF82D808DF82EC038
:106F18004FF0000C8DF82FC08DF830208DF831E03F
:106F28008DF832008DF833108DF834300A99CDF889
:106F380000A0089A019207A8029001EB080009AA8C
:106F48000BABFFF75FFC0799002937D0A3686BB13B
:106F58000A99E26800920898019007AA029201EB48
:106F6800080009AAFFF74EFC079B3BB3246904B34A
:106F78004FF001084FF000092046FFF75DFE8DF83D
:106F88003500618939B10DF11C0C40462246FFF7E6
:106F980075FC079991B1A18939B10DF11C0C4846CE
:106FA8002246FFF76BFC079840B155F8044F002CB8
:106FB800E2D106F10106042E7FF428AF099814E007
:106FC8004FF0FF3011E04FF0000640F6A45BC2F22C
:106FD800000B40F6E454C2F2000405944FF0090A8D
:106FE80040F67057C2F2000710E70FB0BDE8F08F07
:106FF80003F1010307EBC3014A68B2427FF456AFBD
:107008001FE705F1010307EBC3014A68B2427FF4A9
:107018004DAF16E708B540F6C853C2F200031A5C34
:1070280040F6CC21C2F200014FF04C0000FB0210E8
:10703800436AD3F1010238BF002242634FF00001D6
:10704800C1630164416400F11000FDF79FF808BDB9
:107058002DE9F84F81468A4640F6C853C2F200032C
:107068001A5C40F6CC20C2F200004FF04C0404FB3E
:10707800020404F148064FF001084FF0000740F6FB
:107088008C2BC2F2000B354640463146F9F7DAFD43
:1070980030B14FF002003146F9F7D4FDBDE8F88F62
:1070A800BAF1000F05D148464146FCF755FC0328C4
:1070B80027D0256C75B15846A168E26BA8470546EC
:1070C800B0F1FF3F14D06064484659462A46FCF7A1
:1070D80083FC0EE0616CA5688D4228BF0D464846CA
:1070E800E16B2A46FCF778FCE36B5A19E26300E08F
:1070F8003D46606CA16888423CBFE7632764451B36
:10710800656438463146F9F79DFD0228BBD0BDE8D5
:10711800F88F00BFF8B505460E46174640F6C85327
:10712800C2F200031A5C40F6CC20C2F200004FF015
:107138004C0404FB02044FF00000FCF703FCE76377
:1071480026644FF00001616428464FF00101FFF703
:107158007FFF4FF00100FCF7F5FBF8BDF8B50546D9
:107168000F46164640F6C853C2F200031A5C40F6B2
:10717800CC20C2F200004FF04C0404FB0204A168CA
:10718800B1420DD245F6B043C2F200039F4207D385
:1071980046F2B042C2F20002974201D2F9F74EFD20
:1071A8004FF00000FCF7CEFBE7634FF000002064CF
:1071B800666428464FF00101FFF74AFF4FF00100CF
:1071C800FCF7C0FBF8BD00BF08B5FCF77DFC08BDA7
:1071D80070B586B005460C46164602A8FAF7F6FBC7
:1071E80001462EB102A82A46234600F0A5FD07E075
:1071F8004FF00103009302A82A46234600F04EFEF2
:1072080006B070BD70B58AB00378212B00F093806A
:1072180004D86BB1012B40F0D88186E0A12B00F097
:10722800A781C02B00F0B481802B40F0CE8195E07F
:107238004178052903D0092940F0CA8146E04088F1
:1072480040F6C452C2F200021378022B02D0032B7C
:1072580033D118E000F1FF318AB27E2A30D8C0B2AB
:1072680040F6D853C2F2000318704FF00201FCF741
:1072780055FE40F6C450C2F200004FF00301017001
:107288004FF00100C3E170B940F6D852C2F20002D3
:10729800107040F6C450C2F200004FF002030370B1
:1072A8004FF00100B3E17F280DD840F6D851C2F263
:1072B800000108704FF00100A9E14FF00200A6E1BB
:1072C8004FF00200A3E14FF00200A0E1827840F6FF
:1072D800C453C2F200031978022923D972B940F6BF
:1072E800C453C2F200034FF0030119704FF00100BC
:1072F8000146FFF7D1F94FF0010088E1012A18BFD4
:10730800022040F0848140F6C450C2F200004FF0E1
:10731800040202704FF000000146FFF7BDF94FF07C
:10732800010074E14FF0020071E140780B280CBFB6
:10733800012002206BE18388032B00F24C8140F688
:10734800A454C2F2000404EBC3035B68002B00F0F2
:1073580045819847002808BF022058E142781AB1B1
:10736800062A40F03E8121E0C18802291BD14FF056
:107378000000ADF8040040F69452C2F20002126810
:107388000346517E61F30003ADF80430127E62F3C8
:1073980041030AA921F8243D4FF00202FFF7DEFE5F
:1073A8004FF0030033E14FF0020030E18278C188EA
:1073B8008CB2C378022B2ED0032B3DD0012B40F08A
:1073C800D48040F63055C2F20005284649F62461BB
:1073D800C0F601014FF012020FF018FC40F694506D
:1073E800C2F2000001688A892A81CB896B81088AE8
:1073F800A8818A7C2A71CB7C6B71097DA9714FF0B9
:1074080000002946122C34BF22461222FFF7A6FE9E
:107418004FF00300FBE040F6E852C2F2000211818F
:107428004FF00000506046F60D51C0F60001FFF71E
:1074380071FE4FF00300EAE0D2B940F63054C2F2D0
:10744800000404F1020049F61061C0F601014FF092
:1074580002020FF0DBFB4FF0040222704FF003052D
:1074680065704FF000002146FFF778FE2846CEE011
:10747800012A06D140F69453C2F20003196809683C
:107488002FE0022A06D140F69452C2F20002106898
:10749800416826E0032A06D140F69453C2F200035D
:1074A800196889681DE002F00F0022F00F03102B05
:1074B80008D15A4B196888420EDA594A52F83000F6
:1074C80001680EE0202B07D1032805D8554951F84B
:1074D800300008B1016804E0EE2A04D04FF0020041
:1074E80095E009B93EE05049B1F1FF3F40F088808E
:1074F80001A84FF020014FF00102FFF769FE0AAD25
:107508002A184FF0000002F8240C01A978E000F1D5
:107518000206428003F10102134611F8015F5DB1D2
:1075280000F10400758002F1010311F8012F002A0F
:107538006FD101E04FF0000340F63051C2F2000174
:107548004FF003054D7003F101034FEA4303DAB22C
:107558000A704FF00000A24228BF2246FFF7FEFD46
:10756800284654E04FF0020051E04FF002004EE090
:107578008388032B38D840F6A454C2F2000404EBE5
:10758800C3035B689BB39847002808BF02203EE00E
:107598004378212B2ED1C18840F6E853C2F200036C
:1075A80019814FF000025A608088042825D11046BE
:1075B80046F6ED01C0F6000140F6E852C2F20002BC
:1075C800FFF7A8FD4FF0030021E04FF002001EE096
:1075D8004FF002001BE04FF0020018E04FF00200ED
:1075E80015E04FF0020012E04FF002000FE04FF0FC
:1075F80002000CE04FF0020009E04FF0020006E044
:107608000A78002A96D009484FF000037FE70AB0AD
:1076180070BD1E2B7FF47BAF8EE700BFE40D00200A
:10762800700D0020A40D0020849D0108300D00205D
:1076380010B50446436993B14FF00000606140F60D
:10764800C451C2F200010A78032A08D140F6D8537F
:10765800C2F2000318784FF00301FCF75FFC2069C1
:1076680058B34FF000002061E06040F6A051C2F22C
:107678000001087040F6DC51C2F200014FF0080228
:10768800FFF7A2FD082853D140F6DC52C2F20002EF
:10769800137813F0800F06D140F6DC50C2F20000D8
:1076A800C188002944D140F6DC50C2F200004FF0F6
:1076B80000010A46FFF7A6FD2DE0E168002937D052
:1076C8004FF00000E06040F6A052C2F200021378CA
:1076D80040F63051C2F20001C3F14002FFF774FDD9
:1076E800034628B340F6A050C2F2000001785A18A9
:1076F800D2B2027040F6DC53C2F20003D88890423E
:1077080016D140F6DC50C2F2000040F63051C2F209
:107718000001FFF777FD012804D0022808D1FCF703
:1077280039F910BD4FF0000001460246FFF716FD7B
:1077380010BD00BF08B540F6F453C2F200031B6940
:107748003BB14FF0000140F6F452C2F20002526918
:10775800984740F6F450C2F200004FF00001017063
:1077680041608160C1600161416108BD40F6F4502B
:10777800C2F20000816149F6E861C0F601018A5C45
:1077880042778377037F6FF3070303774FF0000196
:107798004162704730B583B040F6F454C2F2000439
:1077A8002070089D6560099DA5600A9DE5600B9D98
:1077B80025610C9D65619DF8184000949DF81C405A
:1077C8000194FFF7D3FF03B030BD00BF40F6F45378
:1077D800C2F200035B6AB3F1FF3F09D140F6F451EE
:1077E800C2F200014FF000034B624FF001007047F6
:1077F8003F2B0BD840F6F452C2F20002106AC15473
:1078080003F1010353624FF0010070474FF000008D
:10781800704700BF704700BF70B540F6F454C2F21D
:10782800000404F1180049F6A061C0F601014FF008
:1078380007020FF0EBF94FF0000049F6E061C0F6DF
:107848000101FFF7AFF947F69526C0F600064FF09D
:10785800000049F68861C0F601013246FFF7C0F919
:1078680049F6EC65C0F601054FF00100294632469D
:10787800FFF7B6F92869FFF7DFF984F8280040F622
:107888006060C2F200004FF0070147F6A502C0F69B
:1078980000024FF00003FCF759FC70BD38B540F604
:1078A8009463C2F200034FF001021A7040F6F454D8
:1078B800C2F2000494F828004FF000010A46FFF7CE
:1078C8004DFC606868B140F6F454C2F200044FF011
:1078D800FF3565626368207861699847616A0029A5
:1078E800F7D040F6F450C2F200004FF000024262B6
:1078F800836833B140F6F451C2F20001087849694F
:10790800984738BD2DE9F04F83B0804643680BB9DE
:10791800806828B14FF00001C8F80810FFF7BEFFD3
:10792800D8F80C20002A45D04FF00003C8F80C30D6
:10793800D8F8000040F62061C2F200014FF0400282
:10794800FFF742FC814640F6F450C2F20000C168DD
:1079580000292FD0B9F1000F2CD040F6F454C2F210
:10796800000440F62066C2F200064FF0000509F157
:10797800FF3B0BF0010B2078715D2A466369E768CD
:10798800B84705F1010AD14570D113E0207816F8FF
:107998000A102A466369E768B8470AF1010A20789D
:1079A80016F80A102A466369E768B8470AF1010A17
:1079B800D145EBD1D8F81420002A54D04FF0000458
:1079C80040F69463C2F200031C70C8F8144040F6F5
:1079D8007060C2F20000FEF747FD40F6F450C2F2B4
:1079E800000044624168002936D040F6F455C2F2DE
:1079F800000540F69864C2F200042C622C46656AC1
:107A08006268207861699047636A9D42F7D11DB327
:107A1800D8F8000040F69861C2F200012A46FFF744
:107A28009DFB4FF000000090019040F67060C2F29C
:107A380000004FF04B014FF0FF0247F6A503C0F6D8
:107A48000003FEF7B7FD0EE040F6F452C2F2000262
:107A580010785169984706E040F6F451C2F20001E7
:107A68008B68002BF0D103B0BDE8F08FBBF1000F9D
:107A78008CD0207816F80A102A466369E768B84758
:107A88000AF1010AD14581D194E700BF10B54478C5
:107A98000378212B02D0A12B1BD10EE0202C04D07F
:107AA800222C14BF0020012010BD072A14D10D4834
:107AB8000FF0ACF84FF0010010BD212C0FD14FF0A2
:107AC800000008494FF00702FFF748FB4FF003009A
:107AD80010BD4FF0000010BD4FF0020010BD4FF078
:107AE800000010BD0C0E002008B540F69463C2F2E9
:107AF8000003187870B940F6F451C2F200014A6ADE
:107B080072B940F6F453C2F2000393F82800FFF765
:107B180081FA08BD40F66060C2F20000FCF736FB4F
:107B280008BD00BF49F65860C0F60100704700BFA5
:107B380070B4037801298CBF4478002402298CBFD3
:107B480085780025DCF8000048B34FEA93064AF22E
:107B58001810C0F60100365C16704FEA031343EAAA
:107B6800141303F03F031B5C5370012907D94FEA34
:107B7800840444EA951303F03F04205C01E04FF0CD
:107B88003D009070022907D905F03F054AF2181305
:107B9800C0F60103E95C01E04FF03D01D17070BC13
:107BA800704700BF82B04FF009010CE00191019BC2
:107BB80003F1FF32019233B100BF019B03F1FF32A1
:107BC8000192002BF8D100F1FF30B0F1FF3FEDD169
:107BD80002B0704770B4C4B24FEA102049F6187664
:107BE800C0F601064AF21805C0F6010511F8013B76
:107BF8001AB94BB944EA00200BE06340F45C4440F6
:107C0800E85C013AF2D1F5E76340F45C4440E85C93
:107C1800ECE770BC704700BF10B444F6FB43C0F2F9
:107C2800861311F8014B02B9ACB380EA04404FEA5D
:107C3800400010F0807F18BF58404FEA400010F015
:107C4800807F18BF58404FEA400010F0807F18BF6F
:107C580058404FEA400010F0807F18BF58404FEA64
:107C6800400010F0807F18BF58404FEA400010F0E5
:107C7800807F18BF58404FEA400010F0807F18BF3F
:107C880058404FEA400010F0807F18BF5840002A43
:107C9800C7D0013AC5D120F07F4010BC704700BF63
:107CA80082B001909DF806304FF0000063F30700A2
:107CB8009DF8052062F30F209DF8042062F3174019
:107CC8009DF8072012F0800F14BF63F07F0103F0C6
:107CD8007F0161F307004FEA4201CAB262F31F60F5
:107CE80013F0800F18BF42F0010262F31F6002B068
:107CF800704700BF84B0C0F307438DF80C30C0F361
:107D080007228DF80D20C3B24FEA10604FEA5002E7
:107D180010F0010F14BF63F07F0103F07F018DF8AD
:107D28000E1013F0800F18BF62F07F028DF80F203D
:107D3800039804B0704700BF2DE9F04F83B00546A3
:107D48000F4614461E46019201F1FF3313F1050F49
:107D580044D8032E43D9A6F10400C0F380080DF1DE
:107D6800040C2846FFF7E4FE05F10305A7F103011B
:107D780004F10404A6F10406A7F1040717F1050F9E
:107D880067D92CE00DF1040C284639462246FFF746
:107D9800CFFE05F1030B5D46A7F1030104F1040AC8
:107DA8005446A6F104094E46A7F1040717F1050F3A
:107DB80015D80F460DF1040C58465246FFF7B8FE89
:107DC8000BF10305A7F103010AF10404A9F1040664
:107DD800A7F1040818F1050F59D900E0FFE799B396
:107DE80096B30DF1040C28466A46FFF7A1FE022E51
:107DF80011D0032E02D0012E26D11AE0019929B103
:107E08009DF8002022704FF0010301E04FF00003BD
:107E180004F1010401E04FF00003019830B102A918
:107E2800CA1812F8080C207003F1010304F10104C8
:107E380001E04FF00003019921B102AAD31813F809
:107E4800080C207004F101040199601A03B0BDE820
:107E5800F08F0F46032EC2D9B8F1000F92D00DF162
:107E6800040C28462246FFF763FE05F10305A7F137
:107E7800030104F10404A6F10406A7F1040717F1AD
:107E8800050FACD80F46032E3FF67CAFA7E7A7F146
:107E98000307032E3FF676AFA1E700BFF0B49DF8C5
:107EA8001040ECB14FEA41079F421CD2DD1B1DD0A8
:107EB80056194FF030046FEA0203F31803F0010378
:107EC80002F8014BB24240F0928007E0134603F8F3
:107ED800014B547003F10102B242F7D13B4607E06F
:107EE8004FF0000504E04FF0000501E04FF00005F9
:107EF80000293CD003F1FF34002B3AD000F10103F4
:107F080041182846521B04F1FF3515F0020F10D016
:107F180032E0A4F1020603F101031F46012C29D027
:107F28003446B44613F8016C4FEA1616092E42D9A6
:107F380044E01E4613F8015C4FEA1515092D8CBF65
:107F480037353035155414B900F1010012E013F833
:107F5800016C06F00F05092D8CBF37353035161822
:107F6800757000F1020528468B42D2D102E02846FE
:107F780000E02846F0BC70471E4613F8015C4FEA43
:107F88001515092D94BF303537351554002CDBD025
:107F980013F8016C06F00F05092D94BF30353735FD
:107FA8001618757000F102008B42E3D003F101034B
:107FB800A4F10204BDE706F1300601E006F1370638
:107FC8005655BCF1000FBFD013F8016C06F00F0630
:107FD800092E94BF303637361018467005F1020066
:107FE8008F42C7D003F10103A4F10204A1E7002BDB
:107FF8003FF46CAF02F8014BB2427FF467AF6DE714
:10800800DCF8143093F8452083F84420DCF8141089
:1080180091F8463081F84530DCF8141091F8472083
:1080280081F84620DCF8143083F84700704700BF19
:10803800DCF8143093F8470093F8462083F847207B
:10804800DCF8141091F8453081F84630DCF814104B
:1080580091F8442081F84520704700BF45F28042DE
:10806800C2F2000213684DF20001C0F60101C85CBB
:10807800C918497803F10203136041EA00207047E8
:10808800DCF80430DCF8082002EBD300CCF8080058
:1080980003F007014FF0010303FA01F2CCF80420C2
:1080A800704700BF2DE9F04F83B004468A469346D7
:1080B8001E46CDF804C04FF00007B846B9463DE06B
:1080C80025463046D047034600283DD0B9F1000F79
:1080D8000CD1202829D0092829D00A2829D00D28F0
:1080E80029D0022D4FF0010988BF0225A3F13002E3
:1080F800D1B2092910D9A3F14100C1B2052903D889
:10810800A3F13703D9B207E0A3F16102D0B2052881
:108118001AD8A3F15703D9B24FEA0717FCB241EABC
:10812800040708F101082C4606E02C4604E02C461A
:1081380002E02C4600E02C463046D847FF2CBFD042
:1081480004F1FF35002CBCD1DDF804C03846FFF738
:1081580057FF019B5A69D8F1010838BF4FF0000852
:1081680082F8508003B0BDE8F08F00BF42F6C40328
:10817800C2F200031B684B634BB19A68824209D074
:10818800DB684B631BB19A688242F9D102E04FF079
:108198001E0070474FF00000704700BF884204D8A7
:1081A800884234BF0220002070474FF0010070471A
:1081B800D0F80431D0F80021934214BFC05C0020ED
:1081C800704700BFD0F80431FF2B14BF01330023E0
:1081D800C0F80431704700BF10B4DCF81420D16C2B
:1081E8000B46044658B14FEA016343EA116301F4B0
:1081F8007F4043EA002301F47F0143EA1123DCF8BE
:10820800040030B199B24FEA134060F30F0361F3F1
:108218001F435CB94FEA036141EA136103F47F40ED
:1082280041EA002103F47F0341EA1323D36410BC1D
:10823800704700BFDCF80030B3F5805F05D240F628
:10824800DC62C2F20002D05C70474FF00000704759
:10825800DCF8003003F10103CCF80030DCF814003E
:1082680090F8512002F1010280F85120704700BFB8
:1082780070B404460846A1B199188C4211D2251849
:10828800AA420ED294423ABFC4EB0206F6B20026C6
:10829800A94205D20019821AD31AF118C8B200E00F
:1082A800304670BC704700BFF0B583B042F6CC03CF
:1082B800C2F200034FF008021A7042F6B400C2F28C
:1082C800000004683CB3154642F6CC07C2F200072A
:1082D8004FF0000621680B6873B10DF107000DF12E
:1082E800060198479DF807009DF8061032463B782E
:1082F800FFF7BEFF4519EDB26468002CEAD142F6DB
:10830800CC02C2F200021078A84204D242F6CC0194
:10831800C2F200010D7042F6CC03C2F200034FF026
:1083280007025A7042F6E404C2F2000424683CB31F
:10833800154642F6CC07C2F200074FF00006206847
:10834800036873B10DF107000DF1060198479DF818
:1083580007009DF8061032467B78FFF789FF45191C
:10836800EDB26468002CEAD142F6CC01C2F20001F9
:108378004A78AA4204D242F6CC00C2F20000457004
:1083880042F6CC03C2F200034FF00001997045F2A7
:108398007C44C2F20004246834B30D4642F6CC078C
:1083A800C2F200070E462268136873B10DF1070088
:1083B8000DF1060198479DF807009DF80610324612
:1083C800BB78FFF755FF4519EDB26468002CEAD178
:1083D80042F6CC00C2F200008178A94204D242F6EB
:1083E800CC02C2F20002957042F6CC03C2F200033E
:1083F8004FF00000D87045F28444C2F200042468AB
:1084080034B3054642F6CC07C2F200070646216897
:108418000A6872B10DF107000DF1060190479DF849
:1084280007009DF806103246FB78FFF721FF451933
:10843800EDB26468002CEAD142F6CC03C2F2000324
:10844800D878A84204D242F6CC01C2F20001CD701D
:1084580003B0F0BD45F27843C2F2000319684DF24B
:108468000000C0F60200401A704700BF034610B172
:1084780082688A4218D042F6C803C2F2000318681C
:1084880060B182688A4203D10BE083688B420AD0CC
:1084980040680028F9D14FF0000305E04FF00003D1
:1084A80002E0034600E003461846704710B541F65F
:1084B8001C74C2F200044FF4117303FB0044D4F897
:1084C8000811B1F1FF3F03D0D4F8042191420DD136
:1084D80023689A6A4FF0FF019047002834D0D4F8F7
:1084E800080100F10100C4F8080110BD91422BD821
:1084F8006318197942F65402C2F2000213787BB964
:10850800FD290FD923689A6A4FF0FE019047D8B128
:1085180042F65400C2F200004FF00101017010BD94
:108528006FEA01012268936AC9B2984760B1D4F82A
:10853800080100F10100C4F8080142F65401C2F232
:1085480000014FF000020A7010BD00BF70B506466A
:1085580041F61C75C2F200054FF4117404FB00F4D7
:108568002B194FF00101C3F80C112A599369984748
:108578002859016A3046884770BD00BF38B541F6B2
:108588001C71C2F200014FF4117202FB00F28C1848
:10859800D4F80831D4F80451AB420DD08958E31807
:1085A8008A6A1979904738B1D4F80801FF2814BFAE
:1085B80001300020C4F8080138BD00BF38B541F6C5
:1085C8001C74C2F200044FF4117202FB00F2A318EB
:1085D800D3F80451D3F808118D4206D14FF00001A9
:1085E800C3F80C11A2589369984738BD10B441F6E6
:1085F8001C73C2F200034FF4117202FB003000F545
:108608008870D0F80031FF2B14BF5A1C0022D0F814
:108618000441A2421CBFC154C0F8002110BC7047DD
:10862800F8B545F27844C2F2000424688568C76842
:10863800466807FB05604518611911D2CE180B482A
:10864800864210D8012B04D1635D13704FF00000EF
:10865800F8BD10461A460EF0D9FA4FF00000F8BDE2
:108668004FF01F00F8BD4FF01F00F8BD01D0020801
:1086780010B542F6B803C2F200031A8841F61C701E
:10868800C2F200004FF4117404FB0204F8F77EFBF9
:108698004FF0FF31C4F810124FF00003C4F818323D
:1086A80004F58874F8F77CFB10BD00BFF8B50646E2
:1086B8004FF0020303704CF20000C0F60100C28BB9
:1086C8004FF6FF718A4221D03F4C404BA34222D241
:1086D80003F110033E4DEF1A4FEA17124FF6FF75DC
:1086E80002F1010002F001071C46D98BA9424FD1C3
:1086F80015E01C46D98BA94211D002F1010203F101
:1087080010031C46D98BA94257D108E04CF200044B
:10871800C0F6010403E04CF20004C0F601044FF671
:10872800FF7021464FF00D02FFF754FA4FF6FF7322
:10873800984208BF0020E28982421BD0A4F11005AC
:108748004CF20000C0F6010085421AD34FF6FF70C4
:1087580029464FF00D02FFF73DFA4FF6FF718842A8
:1087680008BF002034F8024C84420AD12C464FF04E
:10877800010201E04FF00002607BFF2806D1327051
:1087880004E04FF0020333704FF000042046F8BDB8
:108798004FF0000202F1010203F110038242BED041
:1087A800002FA6D01C46D98BA942B8D002F10102ED
:1087B80003F1100382429CD1B1E702F1010203F1F7
:1087C8001003824295D1AAE700C8010800C0010839
:1087D8000FC8010870B5C0B005460E4620F0FF046A
:1087E800684621464FF04002F8F738FA00AB53FAD2
:1087F80085F031464FF010020EF008FA684621461F
:108808004FF48072F9F7D2FD40B070BD38B5054617
:1088180041F61C74C2F200044FF4117303FB0044C8
:10882800D4F81C02FDF72EFB42F6B800C2F2000095
:108838000188A94206D142F6B803C2F200034FF6F6
:10884800FF721A804FF00000C4F81C0238BD00BF48
:1088580010B54FF00000FBF7F1FC42F6B403C2F28A
:1088680000031C6834B12068016901B18847646855
:10887800002CF8D110BD00BF10B50446072822D837
:10888800032894BF4FF4FA73322303FB01F142F635
:108898007003C2F2000303EBC000416059B1FDF759
:1088A800BFFE002808BF012042F67003C2F2000391
:1088B80043F8340010BD42F67001C2F200014FF0D7
:1088C800000241F8342010BD38B5044607284BD8BB
:1088D80042F67003C2F2000303EBC00045680DB313
:1088E80042F67001C2F2000151F83420D2B1FDF70E
:1088F80097FE002808BF012042F67003C2F2000369
:1089080053F83410401A85420BD242F67003C2F273
:10891800000303EBC4024FF00005556043F83450E0
:1089280000E02D1A05F104054CF6CD41CCF6CC41FA
:10893800A1FB05204FEA9003032C0AD803F1630337
:1089480048F21F51C5F2EB11A1FB03324FEA521056
:1089580038BD03F109014CF6CD42CCF6CC42A2FB5E
:1089680001304FEAD00038BD4FF0000038BD00BFDD
:1089780070B506466446DCF814305D6AFDF750FEB3
:108988006169CA6A0AB9C86208E0801A05EB8505F8
:1089980006FB05F6B04224BF0020C8626369D96AA5
:1089A800D1F1010038BF002070BD00BF10B541F6FD
:1089B8001C73C2F200034FF4117404FB003303F577
:1089C8008873D3F80841002C5FD15AB14FF0FF31BA
:1089D800C3F8001142F66C03C2F200034FF0000026
:1089E800187010BDD3F80021B2F1FF3F06D1FF295E
:1089F8004BD14FF00002C3F8002110BDFF291ED152
:108A080042F66C01C2F200014FF000040C70012A1A
:108A180010D94FF00102C3F8082141F61C73C2F2C5
:108A280000034FF4117101FB0030D0F81C02FCF771
:108A3800E7FF10BD4FF00000C3F8000110BDFE298C
:108A480007D142F66C03C2F200034FF0010119701E
:108A580010BD42F66C00C2F20000007848B16FEA1F
:108A68000101C9B242F66C00C2F200004FF00004E6
:108A78000470FF2A05D8995402F10102C3F80021B5
:108A880010BD4FF0FF32C3F8002110BD08B541F604
:108A98001C73C2F200034FF4117202FB0030D0F8CD
:108AA8000811D0F8043100F1040099420AD94FF0B6
:108AB8000002C0F8002142F60010C2F2000040682F
:108AC800FCF79EFF08BD00BFF8B5654642F6F40303
:108AD800C2F200031A7802F00804E7B227B1DCF802
:108AE800146096F8516007E012F0110F06BFDCF829
:108AF800147097F85260002601EB800411F82030BA
:108B080003F0070302F02002D7B23FB111F820208A
:108B180002F00807FAB20AB14FEA430311F82070CD
:108B28004FEA9712012A08D0022A10D111F8200022
:108B3800C0F3011101FB06670BE06F6997F85170EC
:108B480011F82020C2F3011000FB077701E04FF075
:108B58000007042B50D8DFE813F0C60140003B00A3
:108B68002200050045F28041C2F200010B684DF277
:108B78000007C0F60107FA1892F802E0D0784FEA29
:108B8800006040EA0E40527840EA0220FF5C03F1A0
:108B980004030B603843FFF7ADF868602CE045F23A
:108BA8008042C2F2000213684DF20000C0F60100D4
:108BB800C11891F801C0C05C4FEA004040EA0C209F
:108BC8008978084303F1030313603F186F6013E0CB
:108BD800FFF744FAC2196A600EE045F28043C2F218
:108BE800000318684DF20001C0F601010A5CBF18C5
:108BF8006F6000F101001860637803F0070342F624
:108C0800F400C2F20000017801F02002D7B237B1B7
:108C1800607800F00801CAB20AB14FEA43036778E6
:108C28004FEA9710012807D002280ED16178C1F3C6
:108C3800011202FB06670AE06F6997F85100617834
:108C4800C1F3011202FB000701E04FF00007042BFB
:108C580050D8DFE813F0480140003B00220005002F
:108C680045F28041C2F200010B684DF20007C0F6E0
:108C78000107FA1892F802E0D0784FEA006040EA5B
:108C88000E40527840EA0220FF5C03F104030B60B7
:108C98003843FFF72FF8A8602CE045F28042C2F273
:108CA800000213684DF20000C0F60100C11891F8E7
:108CB80001C0C05C4FEA004040EA0C2089780843B4
:108CC80003F1030313603F18AF6013E0FFF7C6F921
:108CD800C219AA600EE045F28043C2F20003186888
:108CE8004DF20001C0F601010A5CBF18AF6000F147
:108CF80001001860A37803F0070342F6F400C2F2FB
:108D08000000017801F02002D7B237B1A07800F056
:108D18000801CAB20AB14FEA4303A7784FEA97108D
:108D2800012807D002280ED1A178C1F3011202FB55
:108D380006670AE06F6997F85100A178C1F301123C
:108D480002FB000701E04FF00007042B50D8DFE8D2
:108D580013F0CA0040003B002200050045F28041A4
:108D6800C2F200010B684DF20007C0F60107FA18BD
:108D780092F802E0D0784FEA006040EA0E4052785C
:108D880040EA0220FA5C03F104030B601043FEF78B
:108D9800B1FFE8602CE045F28042C2F2000213689D
:108DA8004DF20000C0F60100C11891F801C0C05C86
:108DB8004FEA004040EA0C208978084303F1030396
:108DC80013603F18EF6013E0FFF748F9C219EA6033
:108DD8000EE045F28043C2F2000318684DF200012C
:108DE800C0F601010A5CBF18EF6000F101001860CD
:108DF800E37803F0070342F6F400C2F200000178BA
:108E080001F02002D0B230B1E17801F00802D0B20E
:108E180008B14FEA4303E1784FEA9112012A02D0E0
:108E2800022A0FD108E06E6996F85100E278C2F381
:108E3800011101FB000607E0E078C0F3011101FB16
:108E4800066601E04FF00006042B4CD8DFE803F07B
:108E58004B031318300045F28043C2F20003186830
:108E68004DF20001C0F601010A5CB6182E6100F14E
:108E780001001860F8BDFFF7F1F882192A61F8BD02
:108E880045F28042C2F2000213684DF20000C0F6BB
:108E98000100C1184C78C05C4FEA004040EA042049
:108EA8008978084303F10303136036182E61F8BD6F
:108EB80045F28041C2F200010B684DF20004C0F691
:108EC8000104E2189678D0784FEA006040EA06403C
:108ED800527840EA0220E25C03F104030B6010437D
:108EE800FEF708FF2861F8BD08B503281ED8DFE89B
:108EF80000F0020910174BF24430C0F601000FF0E1
:108F080077FC08BD4BF24830C0F601000FF070FC4A
:108F180008BD4BF25C30C0F601000FF069FC08BDDB
:108F28004BF27430C0F601000FF062FC08BD00BFC0
:108F38002DE9F8430546884616461F4642F6B8030B
:108F4800C2F20003B3F8009045F6AC10C2F200007C
:108F5800016842F6B002C2F200021368994201D0D9
:108F6800FFF786FB072D6ED81F2E6CD841F61C74B0
:108F7800C2F200044FF4117000FB094442F60010DD
:108F8800C2F200004FF00001FCF7DAFA217965F32C
:108F98004711072D14BF00250125AA1962F3040102
:108FA8002171CBB22DB184F8058043444FF0020003
:108FB80001E04FF0010006F1FF3E5FFA8EFE46B376
:108FC80002463F1A0EF0010C3D5C04F104063554CC
:108FD8005B1902F101020EF1FF31C9B2FF2934D148
:108FE80014E0BD5C04F10406B5545B1902F10102FA
:108FF80001F1FF3101F0FF01BD5CB5545B1902F1CD
:10900800010201F1FF31C9B2FF29EAD100F10100E3
:1090180070442218137100F10100C4F804014FF0E4
:10902800FF33C4F8083121680B6A42F6B800C2F26F
:10903800000000789847FCF7B1FC42F60010C2F235
:109048000000FCF78BFBBDE8F8834FFA8CF5002D88
:10905800C7D0BD5C04F10406B5545B1902F10102E6
:1090680001F1FF31C9B2FF29BBD1CFE700B583B009
:109078004FF0040240F6D863C2F200031A704FF0B2
:1090880001008DF8040042F6E801C2F200010B88E5
:10909800ADF805304FF007004FF041010DEB02032A
:1090A800FFF746FF03B000BD08B540F6D863C2F22B
:1090B8000003197889B198B1042814D0042904D17F
:1090C800FFF7D4FF4FF0010008BD40F6D862C2F2A6
:1090D800000210704FF0000008BD4FF0000008BDFE
:1090E8004FF0000008BD4FF0000008BD38B5054638
:1090F80042F62C04C2F200042046FCF72FFBF8F7D6
:109108005FFD2846FCF712FE20464FF00001FCF7F1
:1091180017FA38BD10B586B00DF10700FFF7C6FA8B
:10912800044618B19DF8073023B90FE04CF200044B
:10913800C0F60104E2894FF6FF7082422BD04CF64C
:109148000001C0F601018C4209D32AE030482146CB
:109158004FF00D020DF004F9002848D0EAE74FF669
:10916800FF724CF60000C0F601006FEA0403C11854
:10917800C1F3001104F11004E389934239D10AE0E4
:1091880004F110031C46D989914204D003F110045C
:10919800E389934239D14CF60002C0F601029442A9
:1091A80007D34CF20004C0F6010420462146F9F723
:1091B80093F802A816494FF00D020DF027FD4FF065
:1091C800FF008DF815004FF6FF7002A94FF00D0251
:1091D800FEF700FD4FF6FF71884212BFADF816008A
:1091E8000021ADF81610204602A9FFF7F3FA06B0E1
:1091F80010BD8442D5D20029C2D004F11004E189FF
:109208009142C8D08442BBD3CBE78442B8D3C8E7E5
:10921800E20E00202DE9F04F85B0884691461D46A4
:10922800E2464FF0000426464FF0020B2DE00746B9
:109238002846C047034670B324B9202822D00928FD
:1092480002D11FE0012C05D12B2B0DD02D2B0DD0D9
:109258005C4601E0022C01D12E2B09D0A3F130028B
:10926800D0B2092817D805E05C4603E05C4601E067
:109278004FF003040E2E05D804A98A1902F8103CF1
:1092880006F101062846C8473846FF28CFD000F126
:10929800FF370028CCD1012C12D98EB104ACA61905
:1092A8004FF0000406F8104C684621460DF0B2F85D
:1092B800DAF81410C864DAF8142082F8504005E08F
:1092C800DAF814304FF0010083F8500005B0BDE81B
:1092D800F08F00BF10B586B04DF20000C0F6010057
:1092E8003449F8F7F9FF00284BD1334B334A9A42F7
:1092F8001DD24DF20001C0F601010B68B3F1FF3F2A
:1093080042D102F104032E4AD01A20F00302991820
:1093180012F0040F3FD118468B420CD003F104021F
:109328001B68B3F1FF3F3ED04FF0000031E04DF233
:109338000000C0F601004DF20003C0F60203984297
:1093480025D10DF10700FFF7B1F90446B0B19DF83A
:109358000710022912D002A821464FF010020DF082
:1093680055FC9DF815006FF307008DF81500204691
:1093780002A9FFF72FFA4FF001000AE04FF00100B1
:1093880007E04FF0000004E04FF0000001E04FF06C
:10939800000006B010BD184603F104030268B2F1DC
:1093A800FF3FB8D0C0E702F104031068B0F1FF3FF7
:1093B800B1D0B9E7FFCF020800D0020800D00108F9
:1093C80003D002082DE9F007034600284ED040F2EA
:1093D8000022C0F6000292F8469092F8470042F642
:1093E800CC04C2F2000494F8018092F848C02578B1
:1093F80042F6E802C2F200021468177A567AD2F8E6
:1094080004A04FF000021A7083F801909870DA7087
:109418004FF0FB0018714FF0060983F805909D7115
:1094280083F807804FF0040883F8088083F80980E0
:1094380083F80AC0DD721A734FEA14255D739C73B2
:10944800DF731E745A744FF01D029A744FF00202B3
:10945800DA744FF0FE021A755A754FEA1A229A7595
:1094680083F817A018764FF00F00587629B142F606
:10947800CC03C2F200031A680A60BDE8F00770471F
:10948800034628B142F6E802C2F2000210681860EA
:1094980042F6E801C2F20001087A704770B5054645
:1094A8000E4614464FF000002946FEF7DFFF08B1CC
:1094B800F7F7C4FB42F6C803C2F200031A686260F9
:1094C800A56026601C6070BD08B539B142F6B403CA
:1094D800C2F200031A68426018601EE042F6B40344
:1094E800C2F200031B6883420FD1586842F6B401E8
:1094F800C2F20001086010E042685A6041605A6890
:109508008242F9D013461BB907E033B14FF000018E
:109518005A688242F0D01346F5E7FEF7C5FE08BD4B
:1095280008B539B142F6E403C2F200031A68426092
:1095380018601EE042F6E403C2F200031B6883428F
:109548000FD1586842F6E401C2F20001086010E049
:1095580042685A6041605A688242F9D013461BB982
:1095680007E033B14FF000015A688242F0D0134649
:10957800F5E7FEF799FE08BD08B539B145F27C4319
:10958800C2F200031A68426018601EE045F27C438C
:10959800C2F200031B6883420FD1586845F27C4130
:1095A800C2F20001086010E042685A6041605A68DF
:1095B8008242F9D013461BB907E033B14FF00001DE
:1095C8005A688242F0D01346F5E7FEF76DFE08BDF3
:1095D80008B539B145F28443C2F200031A68426003
:1095E80018601EE045F28443C2F200031B68834200
:1095F8000FD1586845F28441C2F20001086010E0BA
:1096080042685A6041605A688242F9D013461BB9D1
:1096180007E033B14FF000015A688242F0D0134698
:10962800F5E7FEF741FE08BD01604360826042F63F
:10963800C403C2F200031A68C2601860704700BF12
:1096480070B582B006464FF000038DF807300D461E
:1096580001B10B7042F6B400C2F20000046874B1A4
:1096680021684B6843B130460DF107012A469847F7
:1096780010B19DF8070011E06468002CF0D1072EA6
:1096880003D83046FAF71EFE08E02DB14FF0050268
:109698002A704FF0000001E04FF0000002B070BDEA
:1096A80070B582B006464FF000038DF807300D46BE
:1096B80001B10B7042F6B400C2F20000046874B144
:1096C80021688B6843B130460DF107012A46984757
:1096D80010B19DF8070019E06468002CF0D1072E3E
:1096E8000BD83046FAF704FE8DF8070010B1304663
:1096F800FAF744FE9DF8070008E02DB14FF0050287
:109708002A704FF0000001E04FF0000002B070BD79
:1097180070B582B006464FF000038DF807300D464D
:1097280001B10B7042F6B400C2F20000046874B1D3
:109738002168CB6843B130460DF107012A469847A6
:1097480010B19DF8070011E06468002CF0D1072ED5
:1097580003D83046FAF79CFD08E02DB14FF005021A
:109768002A704FF0000001E04FF0000002B070BD19
:1097780070B582B006464FF000038DF807300D46ED
:1097880001B10B7042F6E400C2F2000004685CB15B
:1097980021688B682BB130460DF107012A4698479E
:1097A80058B96468002CF3D1062E0CDC082E0AD8B0
:1097B8003046F7F7F3FF8DF807009DF807000030F3
:1097C80018BF012008E02DB14FF006022A704FF0B3
:1097D800000001E04FF0000002B070BDF0B583B0AA
:1097E80005460E464FF000038DF8073042F6E400B8
:1097F800C2F200000468E4B14FF000072168CA68AB
:109808001AB1284631469047F0B923689B6833B1AE
:1098180028460DF106010DF10702984700E0384689
:109828009DF8071099B9646814B10028E6D004E0DF
:1098380018B9062D0DDC082D0ED82846314607F03C
:109848006FF84FF0000009E04FF0000006E008460E
:1098580004E04FF0060001E04FF0060003B0F0BD51
:1098680070B582B005460E464FF000038DF80730FC
:1098780012B11946FFF7B2FF42F6E400C2F2000047
:1098880004686CB121684B68284631460DF107021F
:10989800984710B19DF8070012E06468002CF1D1D8
:1098A800062D08DC082D09D828463146F7F798FF19
:1098B8004FF0000004E04FF0060001E04FF0060012
:1098C80002B070BD08B54FF0000001464FF001022C
:1098D800FFF7C6FF08BD00BF70B582B005460E464B
:1098E8004FF000038DF8073045F27C40C2F20000CB
:1098F8000468B4B121684B68284669460DF107022F
:10990800984728B10EB1009830609DF807000DE027
:1099180064684CB19DF80720002AEBD04FF00F0087
:1099280004E04FF00F0001E04FF00F0002B070BDEF
:1099380070B582B005460E464FF000038DF807302B
:1099480045F28440C2F2000004689CB121684B686B
:10995800284631460DF10702984710B19DF80700D7
:109968000DE064684CB19DF80720002AEED04FF056
:109978000E0004E04FF00E0001E04FF00E0002B0C0
:1099880070BD00BF70B582B005460E464FF00003AB
:109998008DF8073045F28440C2F200000468BCB17B
:1099A80021688B685BB1284669460DF10702984724
:1099B80028B10EB1009830609DF807000DE064688A
:1099C8004CB19DF80720002AEAD04FF0060004E0C9
:1099D8004FF0060001E04FF0060002B070BD00BF76
:1099E8002DE9F04F2DED048B8BB0834692469142C2
:1099F80064D289464FF000089FED379A9FED328B6D
:109A0800DFED369A32A7D7E900674FF000044FF030
:109A18000005C3F6E0758DED019ABBF1020F05D183
:109A28005FFA89F001A9FFF7ADFF04E05FFA89F05A
:109A380001A9FFF751FF08EB48030AAAD01800F85C
:109A4800209C01980BF046FF53EC182B0CF0BAFA47
:109A580008B1CDED019A01980BF03CFF32463B4628
:109A68000CF0D6F822462B460BF08EFF0BF0F8FED2
:109A780081B208EB48030AAAD31803F81E1C4FEA60
:109A8800112003F81F0C08F10108B8F10A0F06D0DD
:109A98000AF1FF3149450DD1B8F1000F0AD008EBA2
:109AA80048024FF007005946D2B202ABFFF740FA1E
:109AB8004FF0000809F10109CA45ACD80BB0BDEC5C
:109AC800048BBDE8F08F00BF9831CB64FE0F704067
:109AD8000000000000E06F4000000000F37F8043BA
:109AE8002DE9F04F9FB040F6C410FCF71FF94FF076
:109AF80002004FF0000142F6CC03C2F20003DA780C
:109B0800FFF76EFF4FF0010002904FF0000BDA46AE
:109B1800D94607464CF6CD41CCF6CC4103914FF0DF
:109B28007D00FCF703F98DF83790C8464E464C4641
:109B380013E045F0800504F10804E4B216A9725C4C
:109B4800AA4202D016ABF554B84606F101069DF8B4
:109B58003750002D50D1202E4ED020460DF1370120
:109B6800FFF76EFD051C18BF012504F10102D0B2F4
:109B78000DF13701FFF764FD10B145F00205EDB2B4
:109B880004F10203D8B20DF13701FFF759FD08B10E
:109B980045F0040504F10300C0B20DF13701FFF7E9
:109BA8004FFD08B145F0080504F10401C8B20DF1F4
:109BB8003701FFF745FD08B145F0100504F105022E
:109BC800D0B20DF13701FFF73BFD08B145F0200594
:109BD80004F10603D8B20DF13701FFF731FD08B1E2
:109BE80045F0400504F10700C0B20DF13701FFF759
:109BF80027FD00289DD19EE7B8F1000F02D1BAF1E8
:109C0800000F0CD14FF002004946F2B216ABFFF735
:109C18008FF94FF03200FCF789F8019701E0CDF891
:109C280004908DF83790C8464E464C4613E045F0F0
:109C3800800504F10804E4B20EA8315CA94202D000
:109C48000EAAB554B84606F101069DF83750002D06
:109C580050D1202E4ED020460DF13701FFF788FD58
:109C6800051C18BF012504F10100C0B20DF1370130
:109C7800FFF77EFD10B145F00201CDB204F10202FA
:109C8800D0B20DF13701FFF773FD08B145F00405B7
:109C980004F10303D8B20DF13701FFF769FD08B1EC
:109CA80045F0080504F10400C0B20DF13701FFF7D3
:109CB8005FFD08B145F0100504F10501C8B20DF1CA
:109CC8003701FFF755FD08B145F0200504F10602FC
:109CD800D0B20DF13701FFF74BFD08B145F0400553
:109CE80004F10703D8B20DF13701FFF741FD002851
:109CF8009DD19EE7B8F1000F02D1BAF1010F0AD148
:109D080048464946F2B20EABFFF712F94FF032005F
:109D1800FCF70CF8019742F6CC03C2F200039A78DC
:109D2800B2B1039EA6FB0A044FEA141000EB8001AF
:109D3800BAEB810F0CD138464946FFF751FE4FF078
:109D48003200FBF7F3FFBBF1000F40F0B88003E0EF
:109D5800BBF1000F40F09C8005A849464FF0200257
:109D68000CF078FF42F6CC06C2F20006B478ACB329
:109D78004D466FEA0900011901F0010209F00703D5
:109D880007FA03F69DF8140046EA00018DF814104E
:109D980005F10105A542C0F2B3801FE01EAB03EB3D
:109DA800D50605F0070007FA00F216F8641C42EA27
:109DB800010306F8643C05F101051EA800EBD50275
:109DC80005F0070107FA01F312F8646C43EA06008C
:109DD80002F8640C05F10105A542DFDB4FF007002E
:109DE8004FF011014FF01E0205ABFFF7A1F84FF03D
:109DF8003200FBF79BFF05A849464FF020020CF004
:109E080029FF42F6CC04C2F20004E578A5B34B461C
:109E18006FEA0902511901F0010609F0070007FA73
:109E280000F49DF8142044EA02018DF8141003F19F
:109E380001039D4250DC1FE01EAC04EBD30203F08B
:109E4800070007FA00F612F8641C46EA010402F853
:109E5800644C03F101031EAA02EBD30403F00700CC
:109E680007FA00F614F8641C46EA010204F8642CA8
:109E780003F101039D42DFDC4FF007004FF01201B0
:109E88004FF01E0205ABFFF753F84FF0060B16E034
:109E9800019AA2B9BBF1020F11D1029D7DB942F618
:109EA800CC03C2F20003DA784AB14FF00200494607
:109EB800FFF796FD4FF03200FBF738FF0297BAF133
:109EC800000F06D10BF1FF3BCDF808904FF0280AA0
:109ED80025E60AF1FF3A22E6002EADD01EAE06EBCB
:109EE800D30403F0070007FA00F214F8641C42EAEE
:109EF800010604F8646C03F101039D429CDCBBE796
:109F0800002A3FF44BAF1EAA02EBD50305F0070663
:109F180007FA06F013F8641C40EA010203F8642CFF
:109F280005F10105A542FFF639AF57E72DE9F04FD6
:109F38002DED028B87B008EE100A0C46174699469D
:109F4800129E1399B5EEC08AF1EE10FA54BF00259F
:109F58000125A84604F1FF33D8B2082807D8092AF2
:109F680005D8A24601F1FF32944205D808E001F174
:109F7800FF339C4240F2CD8001F1FF34E4B2C8E0E7
:109F880018EE100A0CF07AF848B930464FF03F0145
:109F980022460CF05FFE4FF000013155C4E018EE88
:109FA800100A0CF0D7F806EE900AF2EE047AF4EEF6
:109FB800E76AF1EE10FA0DDB4FF00100B0EE677AB8
:109FC80000F1010067EE877AF4EEE76AF1EE10FA25
:109FD800F6DA03E04FF00100F2EE047A2146431965
:109FE800A34200F39680C0EB040EC5EB0E0202F10B
:109FF800FF3E4AF2BC1AC0F6010ADFED9C4AF6EEB3
:10A00800003AB2EE044AC0EB040CC5EB0C0303F0B3
:10A01800010BBEF1000F00F38F808AE0BEF1000F44
:10A0280004DDBE45B4BF72463A4601E04FF0000277
:10A038005AF8223003EE103AB8EE430A20EE027ABC
:10A04800B4EEE47AF1EE10FA48BF37EE237ABDEEAB
:10A05800C73A13EE10CABCFBF3FB06EE10BAB8EE13
:10A06800C65AB4EEE75AF1EE10FA0DDB00F1010C16
:10A0780087EE006A67EE847A0EF1FF3E6046BEF115
:10A08800000200F3C380BEE013EE105AB5FBF3F4F0
:10A0980003FB14542CB916EE107A002F08BF4FF0AA
:10A0A8000008B9F1000F07D0C8EB0103181A002AFD
:10A0B80018BF0138831A01E04FF0000301F10101D4
:10A0C800B8F1000F04D04BF29837C0F6010703E04F
:10A0D80048F6E817C0F6010722B14BF29C30C0F6EB
:10A0E800010003E048F6E810C0F601004BF2B03575
:10A0F800C0F60105009501978DED026A0390049260
:10A10800059430464BF2A032C0F601020CF06CF90F
:10A118000AE03046002D0CBF2B212D2122460CF0E1
:10A1280099FD4FF00000305507B0BDEC028BBDE83B
:10A13800F08F4FF0000203E0BE45B4BF72463A46C6
:10A148005AF8223000EE103AB8EE405A65EE260A68
:10A15800F4EEE40AF1EE10FA48BF70EEA30ABDEE81
:10A16800E03A13EE10CABCFBF3FC06EE10CAF8EE98
:10A17800C65AF4EEE75AF1EE10FA85DB00F1010059
:10A1880080EE852A67EE847A0EF1FF3E42199142ED
:10A19800BFDBBBF1000F3FF441AFBEF1000F02DCA3
:10A1A8004FF0000203E0BE45B4BF72463A465AF883
:10A1B800223001EE103AF8EE411A21EE822AB4EE6E
:10A1C800E42AF1EE10FA48BF32EE232ABDEEC23A75
:10A1D80013EE10BABBFBF3FB06EE10BAF8EEC62A74
:10A1E800F4EEE72AF1EE10FAFFF64EAF00F10100A7
:10A1F80082EE212A67EE847A0EF1FF3E43199942D6
:10A20800BFF60CAF85E74FF0000202E0BA42A8BFE4
:10A218003A465AF8223006EE903AF8EE660A20EEF0
:10A22800861AB4EEE41AF1EE10FA48BF31EE231A9A
:10A23800BDEEC13A13EE10BABBFBF3FB06EE10BA43
:10A24800F8EEC65AF4EEE75AF1EE10FAFFF61CAF34
:10A258000CF1010081EE202A67EE847A0EF1FF3EB0
:10A2680042199142BFF6DAAE53E700BF0000004B37
:10A27800F8B505460F46F6F789FD064641F61C7205
:10A28800C2F200024FF4117303FB05F014181158C1
:10A2980011B18A682846904784F820724FF000056B
:10A2A800C4F81052C4F81452C4F80451C4F8085140
:10A2B8003046F6F775FD04F5097029464FF0080297
:10A2C800F6F71EFDF8BD00BF70B588B0054641F62B
:10A2D8001C74C2F200044FF4117303FB004494F899
:10A2E800200200284AD042F6B801C2F200010A88CA
:10A2F8004FF6FF76B24204D0D0B24FF00401FFF718
:10A30800B7FF28464FF00001FFF7B2FF42F6B80644
:10A31800C2F2000635804BF2BC30C0F601004FF0A7
:10A3280007014AF2F152C0F60002FBF7C1FCC4F87B
:10A338001C02246830784FF0010300934FF00002AC
:10A34800019248F2B541C0F60001029148F6952302
:10A35800C0F60003039348F6B511C0F60001049156
:10A3680048F61503C0F600030593069264684FF497
:10A3780016514FF00803A047FEF77AF908B070BDF0
:10A3880038B506F0C1FA42F6D003C2F200034FF026
:10A3980001021A704FF000042546E0B229462A4609
:10A3A800FFF75EFA60B904F10104E0B229462A46D3
:10A3B800FFF756FA00286BD002E04FF0000401E0E6
:10A3C8004FF000044FF00005E0B22946FFF7B0FA5D
:10A3D80010B904F10104F7E745F28441C2F2000123
:10A3E8000C6834B12368DA6802B190476468002CBD
:10A3F800F8D142F6C800C2F2000004683CB12168F6
:10A408000B680BB1A06898476468002CF7D1FAF77D
:10A418005BFBFEF71DFA41F61C72C2F2000292F8CD
:10A428002002042806D028B14FF000004FF00401A4
:10A43800FFF71EFF41F61C71C2F2000191F8643467
:10A44800042B06D02BB14FF001004FF00401FFF7A9
:10A458000FFF41F61C72C2F2000292F8A806042807
:10A4680006D028B14FF002004FF00401FFF700FFBB
:10A4780041F61C71C2F2000191F8EC38042B06D0A9
:10A488002BB14FF003004FF00401FFF7F1FE38BD88
:10A4980004F10104B4F5807F7FF47FAF8DE700BF3E
:10A4A80038B5054642F6B004C2F200042068FBF74E
:10A4B800E9FC4FF0000323608DB14BF2CC30C0F6BD
:10A4C80001004FF007014AF6C172C0F60002FBF71F
:10A4D800EFFB42F6BC02C2F20002106038BD42F641
:10A4E800BC04C2F200042068FBF7CCFC4FF000006B
:10A4F800206040F6D862C2F200021070FAF79EFEA1
:10A50800FFF73EFF0AF090FC42F6B801C2F20001E4
:10A5180008884FF6FF73984204D0C0B24FF0040188
:10A52800FFF7A6FE38BD00BF70B542F60010C2F2B4
:10A5380000004BF2DC31C0F60101FAF7E9FF42F600
:10A54800B803C2F200034FF6FF721A8041F61C747A
:10A55800C2F200044FF0040684F820624FF00005B0
:10A56800C4F81C522846FBF7BDF9206084F86464DF
:10A57800C4F860544FF00100FBF7B4F9C4F8440282
:10A5880084F8A866C4F8A4564FF00200FBF7AAF9AD
:10A59800C4F8880484F8EC68C4F8E8584FF003005D
:10A5A800FBF7A0F9C4F8CC0642F62C00C2F2000072
:10A5B8004BF2E831C0F60101FAF7AAFF42F6D400DF
:10A5C800C2F200004AF6F851C0F601012A462B46AD
:10A5D800FFF72AF8FDF768FE4FF00100FFF760FF6C
:10A5E80070BD00BF000000002DE9F04F2DED028B7B
:10A5F80091B04FF000020592904642F6BC07C2F2B5
:10A60800000742F6B003C2F20003049342F6B80B07
:10A61800C2F2000B41F61C76C2F200069FEDBC8B1D
:10A6280039684FF0FF3041B9F7F7CAFA386800289F
:10A638000CBFFA204FF0FF30FFE7FBF777FB28B19C
:10A64800B8F1320F09D808F1010806E0B8F1330F64
:10A658000CBF4FF034084FF000083C681CBBF7F7FC
:10A66800AFFAB8F1320F11D1049B1868FBF70AFC56
:10A678004FF0000104980160FAF7E0FD4FF0020086
:10A68800FEF732FC4FF0020405940CE0B8F1340FE9
:10A6980009D1059D012D06D04FF00100FEF724FCDD
:10A6A8004FF001020592BBF800504FF4117202FB03
:10A6B8000563D3F818120029B2D04FF4117000FBCB
:10A6C80005F505F5887406EB0409355DE02D0DD117
:10A6D80099F801200E2A09D14FF6FF704946D9F89A
:10A6E8000021FDF777FA10B300F03BBC335D03F0AF
:10A6F8001F0509EB05014A7805F0010019F8053036
:10A70800D21A05F1FF33002D40F048840BE019F808
:10A718000310501A03F1FF3519F80520821A05F1C4
:10A72800FF33002DF3D112F0FF0F40F01A84335D90
:10A738004FEA5311072900F20C84DFE811F00800F2
:10A748000A040A043500AB000A048F005901335D7E
:10A7580009F1010413F01F0000F0038409F1020954
:10A7680004F1020400F1FF3254FA82F503954FF028
:10A7780000054FF0010A15E019F8011CE8B2214064
:10A788005246FFF76DF8002840F0EB8305F101050C
:10A798004FEA4404FF2CEFD909F1010903998945CF
:10A7A80000F0DF835446E7E799F80150386898B11C
:10A7B800FBF768FB4FF00000386040F6D862C2F241
:10A7C80000021070FAF73AFDFFF7DAFD4FF00100CA
:10A7D800FEF78AFBF7F7F4F9049B196869B94BF29D
:10A7E800F030C0F601004FF0070149F6E922C0F643
:10A7F8000002FBF75DFA049C206007A84FF00001F7
:10A80800FEF7E0FD7DB9FBF70BFFC1B201F1FF33A5
:10A81800DCB2FD2C42F65500C2F2000092BF017076
:10A828000122027009E042F65500C2F200000278E7
:10A8380002FB05F505EB1525057042F65505C2F234
:10A848000005297810AB03F8241D4FF003004FF0E2
:10A8580000014FF01A02FEF76BFBE1E60DF11B0059
:10A86800FDF724FF01469DF81B408DF81C40012C84
:10A8780006D828B10DF11D004FF00D020CF0C6F9F5
:10A888004FF006004FF000014FF00E0207ABFEF745
:10A898004FFBC5E6BBF800304FF4117202FB03F41E
:10A8A80099F80100052800F2A080DFE800F00A35D9
:10A8B800485A037C40F6D863C2F200034FF0010205
:10A8C8001A704FF00100FFF7EBFD4FF0000510ABD9
:10A8D80003F8255D4FF0040029464FF00102FEF70A
:10A8E80027FB4FF0C800FDF75DF931599BF80000D0
:10A8F8004FF0010400940195D1F80CC04FF41651A3
:10A908002A464FF00803E047204627E3AFF30080CC
:10A918000000000000E06F404FF0000142F6E8033D
:10A92800C2F2000319724FF0010410AB03F8254D71
:10A938004FF004002246FEF7FBFA20460EE3FEF72E
:10A94800E9FB10AB4FF0020203F8252D4FF004008D
:10A958004FF000014FF00102FEF7EAFA4FF0010054
:10A96800FCE210AB4FF0120003F8250D4FF0040085
:10A978004FF000014FF00102FEF7DAFA4FF0C8007D
:10A98800FDF710F931599BF800004FF001040094CD
:10A998004FF000020192CD684FF416414FF00803C2
:10A9A800A8472046DAE210AB4FF0120103F8251D44
:10A9B8004FF004004FF000014FF00102FEF7B8FA23
:10A9C8004FF0C800FDF7EEF835599BF800004FF03E
:10A9D800010400944FF000020192ED684FF4E13158
:10A9E8004FF00803A8472046B8E24FF00000B5E250
:10A9F80099F802E099F8035005EB0E201FFA80FC45
:10AA080099F80130A3F10203412B00F2A582DFE897
:10AA180013F042009D00CF00A302A3020D0199018B
:10AA2800A302A302A302A302A3022502A302EB002E
:10AA3800A302A302B500A302A302A302A302A302D6
:10AA4800A302A302A302A302A302A302A302A302D6
:10AA5800A302A302A302A302A302A302A302A302C6
:10AA6800A302A302A302A302A302A302A302A302B6
:10AA7800A302A302A302A302A302A302A302A302A6
:10AA8800A302A302A302A302A302A302A302A30296
:10AA9800910296029B02325DC2F30405E8B20128D6
:10AAA80000F05F8209F1050409F1080E05EBC50104
:10AAB80005EB410303EBC30202F15402D5B205EBE7
:10AAC80045000EEB000AC4EB0A01A1F1030101F0F5
:10AAD800010599F8029014F8010C0AF03DFE53ECB8
:10AAE800182B0BF04BF90AF011FF01464846FEF708
:10AAF8001FFF04F10304544540F0378231E214F893
:10AB0800035C14F8010C0AF027FE53EC182B0BF029
:10AB180035F90AF0FBFE01462846FEF709FF04F165
:10AB2800030414F8035C14F8010C0AF015FE53EC46
:10AB3800182B0BF023F90AF0E9FE01462846FEF728
:10AB4800F7FE04F103045445D9D10AE2305DC0F39D
:10AB58000401A1F10201CAB209F103010EEB0203DB
:10AB6800FF2BC4BFCEF10002D2B240F6DC64C2F2C1
:10AB7800000404EB0E000CF049F8F2E1345DC4F374
:10AB88000402A2F10302D2B209F104010CEB02059E
:10AB980040F6FE708542C4BF6FEA0C02D2B240F69E
:10ABA800DC63C2F2000303EB0C000CF02FF837E56E
:10ABB80010AC04F824ED0DF11D0040F6DC62C2F281
:10ABC800000202EB0E01202D34BF2A4620220CF091
:10ABD8001DF805F101054FF007004FF00301EAB237
:10ABE8002346FEF7A5F91BE599F804504FEA1C2106
:10ABF80041EA0C2210AC24F8242D0DF11E0040F679
:10AC0800DC63C2F2000303EB0C011D2D34BF2A469E
:10AC18001D220BF0FBFF05F102054FF007004FF076
:10AC28001301EAB22346FEF783F9F9E44FF000096D
:10AC38008DF81B9007AD4C46CA4605F801AB204677
:10AC48000DF11B01FEF7FCFC28B115F8010C40F0D2
:10AC5800010205F8012C04F10101C8B20DF11B0134
:10AC6800FEF7EEFC28B115F8013C43F0020005F8A8
:10AC7800010C04F10202D0B20DF11B01FEF7E0FC59
:10AC880028B115F8011C41F0040305F8013C04F152
:10AC98000300C0B20DF11B01FEF7D2FC28B115F874
:10ACA800012C42F0080105F8011C04F10403D8B294
:10ACB8000DF11B01FEF7C4FC28B115F8010C40F09A
:10ACC800100205F8012C04F10501C8B20DF11B01B1
:10ACD800FEF7B6FC28B115F8013C43F0200005F852
:10ACE800010C04F10602D0B20DF11B01FEF7A8FC1D
:10ACF80028B115F8011C41F0400305F8013C04F1A6
:10AD08000700C0B20DF11B01FEF79AFC28B115F837
:10AD1800012C62F07F0105F8011C04F10804E4B27B
:10AD280009F101099DF81B3013B9B9F1200F84D13D
:10AD38004FF002004FF000015FFA89F207ABFEF70F
:10AD4800F7F86DE44FF000098DF81B9007AD4C46FD
:10AD5800CA4605F801AB20460DF11B01FEF708FDB8
:10AD680028B115F8010C40F0010205F8012C04F196
:10AD78000101C8B20DF11B01FEF7FAFC28B115F864
:10AD8800013C43F0020005F8010C04F10202D0B2C4
:10AD98000DF11B01FEF7ECFC28B115F8011C41F080
:10ADA800040305F8013C04F10300C0B20DF11B01D6
:10ADB800FEF7DEFC28B115F8012C42F0080105F871
:10ADC800011C04F10403D8B20DF11B01FEF7D0FCFD
:10ADD80028B115F8010C40F0100205F8012C04F117
:10ADE8000501C8B20DF11B01FEF7C2FC28B115F828
:10ADF800013C43F0200005F8010C04F10602D0B232
:10AE08000DF11B01FEF7B4FC28B115F8011C41F047
:10AE1800400305F8013C04F10700C0B20DF11B0125
:10AE2800FEF7A6FC28B115F8012C62F07F0105F8A1
:10AE3800011C04F10804E4B209F101099DF81B3072
:10AE480013B9B9F1200F84D14FF0000001465FFA21
:10AE580089F207ABFEF76CF8FFF7E2BBBEF1000F13
:10AE680016D1ADB909F0E0FF04980068FBF70AF8BD
:10AE78004FF00001049A1160FAF7E0F94BF2004034
:10AE8800C0F601000DF0B4FCFEF724FA002848D003
:10AE980099F8024099F803304BF21040C0F60100CF
:10AEA80043EA04210DF0A4FC99F80350494611F82F
:10AEB800020F4DF20002C0F6010202EB002440F638
:10AEC800DC6AC2F2000A0AEB050001F102014FF048
:10AED80080020BF09BFE4FF68071CFF6FF714B1B83
:10AEE800DDB20AEB050061194FF080020BF08EFE0F
:10AEF800504621464FF48072F7F758FAA0B95046E9
:10AF080021464FF480720BF02BFA80B94FF0010004
:10AF18004FF000010A460B46FEF70AF84FF0010011
:10AF28001CE04FF0000019E04FF0000016E04FF071
:10AF3800000013E04FF00300FEF7B6F80EE04FF004
:10AF48000100FEF7B1F809E04FF00200FEF7ACF897
:10AF580004E04FF0000001E04FF0000000287FF40B
:10AF68005FABFDF785FBFFF75BBB002D3FF4C7AD7B
:10AF780014F8035C14F8010C0AF0EEFB53EC182BE0
:10AF88000AF0FCFE0AF0C2FC01462846FEF7D0FC97
:10AF980004F1030454457FF4B2ADE2E700283FF41E
:10AFA800B6AB19F80350521B03F1FF33B3F1FF3F5F
:10AFB8007FF4ADABFFF7B7BB2DE9F04F2DED048B58
:10AFC800ABB01CAF26AC4AF2AC15C0F6010595E84B
:10AFD8000F0084E80F00A76048F23D23C0F6000385
:10AFE800E36020462AA9F7F749FF22AE95E80F004B
:10AFF80086E80F00B76048F25920C0F60000F060FC
:10B0080030462146F7F73AFF4FF000041B9442F60A
:10B018002C00C2F200002146FAF792FA42F6E80143
:10B02800C2F200010C72FFF7ABF909F0FDFE4FF018
:10B038000200FFF749F945F28042C2F200021568A2
:10B048000DBB0DF0C5FBF0B9F6F7BAFC10F0C20F56
:10B0580019D14FF00300FDF747FF4FF47A744FF012
:10B0680032052846FAF762FEF6F7AAFD04F1FF3426
:10B078002846FAF75BFEF6F7A3FD013CF1D14FF045
:10B088000000FDF731FF42F6F403C2F200034FF06F
:10B0980000041C604FF00100187042F62815C2F237
:10B0A80000052846214642F654220BF0D3FD40F60F
:10B0B800DC60C2F2000021464FF480520BF0CAFD5A
:10B0C80042F67000C2F2000021464FF040020BF039
:10B0D800C1FD45F27C30C2F2000021464FF0FC026F
:10B0E8000BF0B8FD21954FF00A0169622046294608
:10B0F800FDF73CF842F66802C2F20002146042F61C
:10B10800C003C2F200031C6045F28045C2F200058C
:10B118004FF030042C604DF20004C0F6010494F89E
:10B128002F0000F1010094F82E1000EB01221019F5
:10B1380045F27843C2F200031860FBF771FA0A90EF
:10B148002B68E15CFF2930D142F6E802C2F2000226
:10B158004FF00101117213602198026A1AB102F1CD
:10B16800010250F8223042F6E801C2F200014B60B9
:10B178004FF0FF00487242F6BC03C2F200034FF0E2
:10B1880000021A6042F6B801C2F20001088841F6CE
:10B198001C72C2F200024FF4117303FB0021D1F8B4
:10B1A8001C02FAF72DFC05F0F0B905F08BFB4FF007
:10B1B80000060996B246344601E04FF000042CB967
:10B1C8004FF00000FDF792FF4FF0640404F1FF34E4
:10B1D80040F6D867C2F200073D78032D27D14FF01B
:10B1E80000038DF8443045F28041C2F200010E8818
:10B1F800ADF845604FF007004FF041014FF00402F1
:10B2080011ABFDF795FE40F6D867C2F200073D780E
:10B21800032D15D14FF0000640F6D867C2F200079B
:10B228003046FDF763FF38780328F9D008E0022D8F
:10B2380006D140F6D860C2F200004FF00302027057
:10B2480042F6F403C2F200031A7802F0E7016FF342
:10B258004511197045F28045C2F200052E6808961E
:10B2680045F28046C2F200064DF20007C0F601071B
:10B2780042F6F408C2F200084AF64479C0F6010919
:10B2880030683D5C00F10100306098F8003013F040
:10B29800010F0ED10AF1010A40F2FF32924508D996
:10B2A80042F6E803C2F200034FF036021A7205F0C4
:10B2B80003B90DF1700C28464946FDF705FC4AF61E
:10B2C800B411C0F6010151F825304AF6640BC0F6F6
:10B2D800010B43F0010000473368FA5C0B9203F15D
:10B2E800010333600F2A05F2DF800DF1700C104660
:10B2F8005946FDF7E9FB4AF64461C0F601010B988F
:10B3080051F82030E5E73368FA5C0B9203F101034A
:10B318003360102A02D9154605F0C7B80DF1700C34
:10B328000B984AF6B451C0F60101FDF7CDFB4AF27D
:10B33800E861C0F601010B9851F82030C9E733687D
:10B34800FA5C0B9203F1010333600F2A02D9154608
:10B3580005F0ABB80DF1700C0B984AF60461C0F615
:10B368000101FDF7B1FB4AF2A861C0F601010B9893
:10B3780051F82030ADE73368FA5C0B9203F1010312
:10B3880033602F2A02D9154605F08FB80DF1700CDD
:10B398000B984AF68461C0F60101FDF795FB4AF265
:10B3A800F811C0F601010B9851F8203091E7336885
:10B3B800FA5C0B9203F1010333603B2A02D915466C
:10B3C80005F073B80DF1700C0B984AF2B851C0F63D
:10B3D8000101FDF779FB4AF2C841C0F601010B985B
:10B3E80051F8203075E73368FA5C0B9203F10103DA
:10B3F80033603F2A02D9154605F057B80DF1700C95
:10B408000B984AF26471C0F60101FDF75DFB4AF240
:10B41800C831C0F601010B9851F8203059E733685C
:10B42800FA5C0B9203F101033360432A02D91546F3
:10B4380005F03BB80DF1700C0B984AF6A401C0F664
:10B448000101FDF741FB4AF2B821C0F601010B9852
:10B4580051F820303DE7219F97F846500DF1700CC8
:10B46800FCF7E6FD219E291896F8502002F001000D
:10B478000B181C9386F84730FF2B94BF0023012339
:10B4880086F850309BE6219F97F846500DF1700CD6
:10B49800FCF7CEFD2E181C96219981F84760FF2EE7
:10B4A80094BF0026012681F8506088E60DF1700CE3
:10B4B800FCF7BEFD30B1219A92F84730181C18BF2E
:10B4C800012001E04FF00000219F87F8470076E651
:10B4D8000DF1700CFCF7ACFD219D95F847603040EC
:10B4E80085F847006BE61D99A1F1FB011C9119E154
:10B4F8001D98A0F1FB001C90A1E11D9AA2F1FB028E
:10B508001C92D2E11D9BA3F1FB031C936FE21D99D2
:10B51800A1F1FB011C914FF002001B9006E21D9A5D
:10B52800A2F1FB021C921E9B1B9330E21D99A1F114
:10B53800FB011C912AE11D98A0F1FB001C90ADE2D3
:10B548001D9AA2F1FB021C92E9E21D9FA7F1FB07DD
:10B558001C971E9E1B9626E31D9BA3F1FB031C93C1
:10B568001E991B914FF000008DF86A00DBE31D9ACD
:10B57800A2F1FB021C921E9B1B934FF001018DF858
:10B588006A10D0E31D98A0F1FB001C9000F068BC85
:10B598001D9DA5F1FB051C9500F0BDBC9DF8740030
:10B5A8004FF00101FEF71AF98DF86B0000283FF4FF
:10B5B80006AE42F6E804C2F20004207204F07CBF32
:10B5C8001D9E1C964FF001038DF86A301E46219A85
:10B5D80092F847100B4205D09DF870003146FEF7EF
:10B5E800FDF868B99DF86A304FEA43008DF86A00A3
:10B5F8001C9A02F101021C9210F0FE03E7D10CE044
:10B608009DF86A10012908D19DF86B4042F6E800C0
:10B61800C2F20000047204F04FBF0DF1700CFCF789
:10B6280007FDCCE59DF8740005F03EF9C7E50DF17E
:10B63800700CFCF7FDFC1C9045F28040C2F2000043
:10B6480002681C9B02EB43010160FCF707FD1C909C
:10B6580001F0D8BE42F6F402C2F20002137813F0E9
:10B66800280F06D01D99B1F5805F34BF0021012154
:10B6780004E01D99FA2994BF0021012141B142F645
:10B68800E804C2F200044FF01301217204F014BF61
:10B6980040F6DC60C2F200001D9A835C1C93CBE785
:10B6A800219890F852201C92C6E7219B93F85010DD
:10B6B8001C91C1E74FF0000A81E50DF1700CFCF711
:10B6C800B7FC1C90219F97F847101B91FCF766FD6B
:10B6D80087F8470073E5219D95F8470095F84610CF
:10B6E800FCF75CFD85F8500069E50DF1700CFCF77E
:10B6F800C7FC1E9E40F6DC62C2F20002905D1D9BF4
:10B7080020EA030191555AE545F27C30C2F2000067
:10B718004FF000014FF0FB020BF09CFA4FE54FF0A1
:10B7280000061C960DF1A80C1CF8386DFCF780FC7F
:10B738000146304607F06AFF8DF86B0000283FF499
:10B748003EAD42F6E804C2F20004207204F0B4BE32
:10B7580006F0E0FA33E506F0E5FA8DF86B0000280C
:10B768003FF42DAD42F6E802C2F20002107204F076
:10B77800A3BE45F27847C2F200073D681D98281815
:10B7880006F0BCFA1BE54FF000031C931C9841F629
:10B798001C72C2F200024FF4117101FB002393F8EE
:10B7A8002022032A3FD141F61C76C2F2000601FB93
:10B7B80000F000F58877F119331803F104034FF00E
:10B7C8000000D1F80021FE2A94BF551C0025D1F8AD
:10B7D8000461B54214BF0025012565F30000B2429B
:10B7E80014BF0022012262F34100D3F80051FE2D5C
:10B7F80094BF013500250DF1A80C4CF8385DD3F83D
:10B808000471BD4214BF0025012565F38200D3F8F9
:10B818000811D1F1010338BF002363F3C300C0B29C
:10B82800FCF7EEFBCBE442F6E804C2F200044FF06A
:10B838004800207204F040BE4FF000001C901C9B92
:10B8480041F61C72C2F200024FF4117101FB032091
:10B8580090F82022032A1CD141F61C76C2F2000679
:10B8680001FB0365D5F81072D5F81412781AB0F5F3
:10B87800807F88BF00F580701C901C9AFF2A84BFC7
:10B88800FF221C920DF1A80C1CF8380DFCF7B8FB30
:10B8980095E442F6E804C2F200044FF0480323722C
:10B8A80004F00ABE4FF000031C931C9841F61C726A
:10B8B800C2F200024FF4117101FB002393F8202219
:10B8C800032A24D141F61C76C2F2000601FB00656A
:10B8D80005F58877D7F80011D7F80431CA1AB2F5F8
:10B8E800807F88BF02F580721C920DF1700CFCF706
:10B8F8009FFB8DF86A001C9EB04238BF1C90D7F899
:10B9080004011C9D2918CBB2C7F8043157E442F64C
:10B91800E804C2F200044FF04800207204F0CCBDE5
:10B928004FF000021C924FF002001B901C9B41F646
:10B938001C72C2F200024FF4117101FB032090F84F
:10B948002022032A15D141F61C77C2F2000701FB19
:10B9580003760DF1700C1B9848F2B911C0F600017E
:10B9680048F2CD12C0F6000206F58873FCF79AFB80
:10B9780025E442F6E804C2F200044FF048032372BB
:10B9880004F09ABD4FF000011C911D981B901C9B60
:10B9980041F61C72C2F200024FF4117101FB032040
:10B9A80090F82022032A16D141F61C75C2F2000530
:10B9B80001FB03570DF1700C1B9848F2B911C0F642
:10B9C800000148F2CD12C0F6000207F58873FDF7B2
:10B9D80021FCFFF7F4BB42F6E804C2F200044FF082
:10B9E8004803237204F068BD4FF000011C911C98B5
:10B9F80041F61C72C2F200024FF4117303FB0021DE
:10BA080091F82022032A3DD141F61C76C2F20006A5
:10BA180003FB006505F588750DF1700CFCF708FB54
:10BA28008DF86A00D5F804111C914FF000071B9798
:10BA3800D5F800710B468F4207D06A5C824219D054
:10BA48004FF001024FF0000E0CE04FF0FF001B908A
:10BA580010E002F10106E95C814202D11C931B92BD
:10BA680008E03246FF2B14BF01337346BB42F0D1C6
:10BA78001C93EAE70DF1700C9DF86C00FCF7C0FA16
:10BA8800FFF79DBB42F6E804C2F200044FF04800FD
:10BA9800207204F011BD4FF000031C931C9841F66E
:10BAA8001C72C2F200024FF4117101FB002393F8DB
:10BAB8002022032A27D141F61C75C2F2000501FB9A
:10BAC800005707F58875D7F81462D7F810128E4218
:10BAD80012D00DF1700CFCF7ABFA8019C7B21C97A5
:10BAE8000DF1700CE85DFCF78BFA4FF00005219E14
:10BAF80086F85050FFF763BB4FF00102219B83F893
:10BB08005020FFF75CBB42F6E804C2F200044FF095
:10BB18004800207204F0D0BC4FF000011C911C9B1F
:10BB280041F61C72C2F200024FF4117000FB0321AF
:10BB380091F82022032A28D141F61C77C2F2000787
:10BB480000FB037505F58876D6F80401D6F80011D0
:10BB5800884213D00DF1700C305CFCF751FAD6F81E
:10BB68000471FF2F14BF01370027C6F804714FF086
:10BB78000005219E86F85050FFF721BB4FF00102C7
:10BB8800219B83F85020FFF71ABB42F6E804C2F263
:10BB980000044FF04803237204F08EBC4FF00000FD
:10BBA8001C901D991B9145F27842C2F20002D2F80E
:10BBB80000801B9F08EB07064DF20003C0F6020346
:10BBC8009E4208D942F6E804C2F200044FF01F0270
:10BBD800227204F071BC1C98032808D942F6E800C8
:10BBE800C2F200004FF03703037204F065BCF1782D
:10BBF8000D2908D942F6E804C2F200044FF03701D3
:10BC0800217204F059BC41F61C75C2F200054FF4CC
:10BC1800117202FB005393F8200238B118F807108C
:10BC280021B10FE04846FDF761FA05E04CF24F35C7
:10BC38004FF09609DDF828B0FAF7F2FCCBEB0002DA
:10BC4800AA42EFD918F80770032F5DD8DFE807F08C
:10BC580002080F169DF87000FEF736FBFFF7AFBA23
:10BC68009DF87000314607F0F3FCFFF7A8BA9DF87D
:10BC78007000314605F0AAFFFFF7A1BA9DF8705091
:10BC8800B77828464FF00301FEF7F2FA4FF4117324
:10BC980003FB05F041F61C71C2F2000108580028A8
:10BCA8003FF48DAA4AF2E413C0F6010307EB4707F5
:10BCB80003EB0708F6784AF22C72C0F6010252F834
:10BCC8002610DA5D98F8013098F8027000974FF066
:10BCD8000006019648F28557C0F60007029748F219
:10BCE800C557C0F60007039748F2F557C0F6000796
:10BCF800049748F61507C0F60007059706964668A4
:10BD08002846B047FFF75BBA9DF870004FF0040172
:10BD1800FEF7AEFAFFF753BA4FF000011C911D98D9
:10BD28001B908DF86A101C9841F61C73C2F2000330
:10BD38004FF4117101FB003292F82032032B79D1B4
:10BD480041F61C75C2F2000501FB005707F588791A
:10BD580045F27846C2F200063168219A936B01EBEE
:10BD6800030BCB5CFF2B5CD0D8464FF001054FF09E
:10BD7800000B0894CDF82CA0AA4698F8014004EBD3
:10BD8800032745F27846C2F200063268D319D9F87B
:10BD980004111C919DF86A0018B1D75D03F10103E5
:10BDA80000E05F4603F1FF349DF86A502DB177B982
:10BDB800089C5046DDF82CA005E066783EB9089C42
:10BDC8005046DDF82CA01C9AC9F804212BE01C9BD6
:10BDD800D9F800219A4218D014F8016F19F80350C5
:10BDE8001B9939B930460AF0A3FAC6B228460AF0B8
:10BDF8009FFAC5B2AE4208D11C98FF2814BF013083
:10BE080058461C9007F1FF37CEE70AF1010A18F8E7
:10BE1800023FFF2BB1D1089CDDF82CA04FF00000A9
:10BE280001E04FF000000DF1700CC0B2FCF7E8F82B
:10BE3800FFF7C5B942F6E804C2F200044FF0480023
:10BE4800207204F039BB4FF000031C931E9A1B921A
:10BE58004FF001018DF86A1065E74FF000011C9161
:10BE68001C9841F61C73C2F200034FF4117101FBD8
:10BE7800003292F82032032B31D141F61C76C2F2FF
:10BE8800000601FB006505F588770DF1700CFCF7DD
:10BE9800CFF88DF86A004FF000011C91D7F80431F3
:10BEA800D7F80051AB4212D0FA5C82420FD14FF062
:10BEB8000006FF2B14BF01333346AB4202D1C7F84B
:10BEC800043104E0F95C8142F3D0C7F804310DF184
:10BED800700C4FF00000FCF793F8FFF770B942F6CA
:10BEE800E804C2F200044FF04800207204F0E4BAFB
:10BEF800FAF796FB0A9FC01B0DF1700C4CF24F33FA
:10BF080098428CBF00200120FCF77AF8FFF757B958
:10BF18004FF000001C901C9D41F61C72C2F20002FA
:10BF28004FF4117606FB052191F82072032F7FF458
:10BF380046A941F61C73C2F2000306FB053000F166
:10BF48000405D0F80861D5F8002102F101029642F3
:10BF580038BF06F58076B11AFF2934BF0F46FF2790
:10BF68000DF1700CF8B2FCF74BF8FFF728B91D9BE0
:10BF780040F6DC60C2F20000C55C05F1FF36C6542D
:10BF8800FFF71DB942F6F402C2F20002117811F06F
:10BF9800280F06D01D9BB3F5805F34BF0023012313
:10BFA80004E01D9BFA2B94BF0023012343B142F602
:10BFB800E804C2F200044FF01302227204F07CBAC3
:10BFC8001D9840F6DC62C2F20002115C01F1FF33F9
:10BFD800D9B2115400293FF4F2A81E981C9001F020
:10BFE80011BA42F6F403C2F20003197811F0280FCF
:10BFF80006D01D98B0F5805F34BF0020012004E012
:10C008001D98FA2894BF0020012040B142F6E804A8
:10C01800C2F200044FF01302227204F04DBA1D9AC6
:10C0280040F6DC61C2F200018B5C03F1FF30C3B261
:10C038008B54002B42F0FD86FFF7C1B842F6F4019D
:10C04800C2F20001087810F0280F06D01D9BB3F546
:10C05800805F34BF0023012304E01D9BFA2B94BFAB
:10C068000023012343B142F6E804C2F200044FF072
:10C078001302227204F020BA1D9A40F6DC61C2F263
:10C088000001885C00F1FF33D8B28854002802F020
:10C09800D086FFF794B8219F97F8515005F1FF36E5
:10C0A80087F85160FFF78BB8219991F8473003F171
:10C0B800FF3081F84700FFF782B8219AD06C0AF068
:10C0C80049F8219FF864FFF77AB8219D95ED137A16
:10C0D800D5ED127A37EE270A85ED130A219AD06C2E
:10C0E80009F0ACFF30B14FF00202219B83F85020D9
:10C0F800FFF765B82198C06C09F0B0FF30B14FF078
:10C108000106219981F85060FFF759B84FF00007F0
:10C11800219D85F85070FFF752B89DF87400219959
:10C1280001F14C01FDF7D8FB8DF86B0000283FF4B6
:10C1380046A842F6E804C2F20004207204F0BCB932
:10C148009DF874002199C96CFDF7F2FB8DF86B001E
:10C1580000283FF434A842F6E803C2F2000318723C
:10C1680004F0AAB9219EF06C09F078FF20B9219853
:10C17800806C09F073FF30B14FF00306219880F806
:10C188005060FFF71CB8219AD2ED138A92ED128AFB
:10C1980078EEC80A10EE900A09F0DCFF09EE100AE2
:10C1A80018EE900A18EE101A09F06EFF01464FF0CB
:10C1B8007E5009F069FF9FEDCF1A01EE900A21EE3B
:10C1C800812AB4EEC29AF1EE10FA06D84FF00001B7
:10C1D800219B83F85010FEF7F2BF219FD7ED132A59
:10C1E80097ED123AF4EEC32AF1EE10FA05DD4FF09E
:10C1F800010587F85050FEF7E2BFF4EEC32AF1EECE
:10C2080010FA4CBF0222032287F85020FEF7D7BF4E
:10C21800219AD2ED133AB7EE004A73EEC44AC2ED42
:10C22800134A2198C06C09F019FF30B14FF003058B
:10C23800219F87F85050FEF7C2BF219BD3ED138A88
:10C248009FEDAD8A38EEC89A19EE100A09F082FF00
:10C2580009EE100A18EE900A18EE101A09F014FFE9
:10C2680001464FF07E5009F00FFFDFEDA23A04EED1
:10C27800100A64EE234AB4EEE49AF1EE10FA22D9D9
:10C28800219E96ED138ADFED9C8A38EE285A15EE2A
:10C29800100A09F05FFF08EE900A18EE100A6FF016
:10C2A800525109F0F1FE01464FF07E5009F0ECFEC4
:10C2B800DFED905A06EE100A66EE256AF4EEE68A7D
:10C2C800F1EE10FA06D84FF00406219981F8506073
:10C2D800FEF775BF2199CD6C284609F03BFF08EEA3
:10C2E800100A28464FF0000109F0CEFE01464FF033
:10C2F8007E5009F0C9FEDFED7F7A07EE100A27EEBF
:10C30800270AB4EEC08AF1EE10FA06D84FF0000002
:10C31800219B83F85000FEF752BF219FD7ED130AE7
:10C32800F5EEC00AF1EE10FA05DD4FF0010287F8CC
:10C338005020FEF744BFF5EEC00AF1EE10FA4CBFEC
:10C348000222032287F85020FEF739BF219F97ED7C
:10C35800125AD7ED135A85EE256A87ED136ABDE6A2
:10C368002199C86C09F066FE002841F04980FEF763
:10C3780026BF219BDE6C304609F0ECFE08EE100A61
:10C3880030464FF0000109F07FFE01464FF07E5025
:10C3980009F07AFEDFED576A07EE100A67EE267A93
:10C3A800B4EEE78AF1EE10FA01F32A80FEF707BF30
:10C3B8002198C06C09F03EFE002801F02180FEF7AC
:10C3C800FEBE219A92ED130AD2ED120AB4EEE00AEB
:10C3D800F1EE10FA81F21480FEF7F1BE219991ED89
:10C3E800131AD1ED121AB4EEE11AF1EE10FA01F3B4
:10C3F8000780FEF7E4BE219B93ED132AD3ED122AA2
:10C40800B4EEE22AF1EE10FA40F2FA87FEF7D7BE50
:10C41800219890ED133AD0ED123AB4EEE33AF1EEEA
:10C4280010FA00F1ED87FEF7CABE219EF66C304681
:10C4380009F090FE08EE100A30464FF0000109F0AE
:10C4480023FE01464FF07E5009F01EFE9FED294A5B
:10C4580004EE900A24EE845AB4EEC58AF1EE10FA7E
:10C4680040F2CE87FEF7ABBE219DE86CFBF718FCC7
:10C47800E8640DF1700C4FF00000FBF7ADFEFEF71D
:10C488009EBE1D9AF62A08D942F6E804C2F20004B4
:10C498004FF01202227204F00FB8219FF86C09F0D5
:10C4A800C9FD38B9219B93ED136AF6EE006A36EEA2
:10C4B800268A06E0219991ED138AF6EE005A38EEA5
:10C4C800658A18EE100A09F0B5FDF8B99FED0B7AE8
:10C4D800B4EEC78AF1EE10FA04DC18EE100A09F07F
:10C4E800ADFD98B14FF00100219E86F850006FF025
:10C4F80000403AE000000034FFFF7F4BFEFFFF4A98
:10C50800FEFFFFCA00008043000080C318EE100A37
:10C5180009F090FD98B15FED067AB4EEE78AF1EE86
:10C5280010FA04D418EE100A09F088FD38B14FF05B
:10C538000101219B83F850104FF0004015E018EEE0
:10C54800100A09F08BFD38B14FF00202219F87F8DD
:10C5580050204FF0000008E0BDEEC88A18EE100A1F
:10C568004FF00006219D85F850604FEA006545EAC6
:10C57800106200F47F4742EA072100F47F0341EA92
:10C58800132045F27C36C2F200061D9D7051FEF75D
:10C5980016BE1D99F62908D942F6E804C2F200042D
:10C5A8004FF01201217203F087BF45F27C37C2F2C7
:10C5B800000778584FEA006343EA106600F47F45A5
:10C5C80046EA052100F47F0241EA122700EE107ABC
:10C5D800F8EEC00A2198C0ED130A1FED381AF4EEE0
:10C5E800C10AF1EE10FA06DC5FED3B1AF4EEE10A3F
:10C5F800F1EE10FA05D54FF0010680F85060FEF70D
:10C60800DEBD4FF0000380F85030FEF7D8BD0DF1C5
:10C61800700C4FF00100FBF7DFFD219DE86CFBF784
:10C6280069FB219AD064FEF7CABD219F97ED132AB2
:10C63800F7EE002A32EE223A87ED133AF1E5219A15
:10C64800D06C09F00BFD50B1219D4FF0000785F823
:10C6580047704FF0040285F85020FEF7B0BD2198CE
:10C6680090ED131AB5EEC01AF1EE10FA23DB1FEDA8
:10C678005B3AB4EEC31AF1EE10FA0FD5FCEEC13AEC
:10C6880013EE906A0DF1700CF0B2FBF7B9FC4FF0A5
:10C698000001219B83F85010FEF791BD0DF1700C3D
:10C6A8004FF0FF00FBF7ACFC4FF00202219880F836
:10C6B8005020FEF784BDB5EEC01AF1EE10FA7EF5F3
:10C6C8007EAD5FED6F1AB4EEE11AF1EE10FA11DDEE
:10C6D800B1EE412AFCEEC22A12EE901A0DF1700C4E
:10C6E800C8B2FBF78DFC4FF00105219F87F8505029
:10C6F800FEF765BD0DF1700C4FF0FF00FBF780FCF5
:10C708004FF00306219B83F85060FEF758BD42F6B0
:10C71800F400C2F20000017811F0280F08D01D9B28
:10C7280003F10103B3F5805F34BF0023012306E062
:10C738001D9B03F10103FA2B94BF0023012343B18E
:10C7480042F6E804C2F200044FF01302227203F02A
:10C75800B3BE219E96ED134AFDEEC44A14EE905ADC
:10C768002FB21C97BAB2C5F3072040EA022140F65F
:10C77800DC66C2F200061D9BF152FEF720BD42F6B0
:10C78800F400C2F20000017811F0280F08D01D9BB8
:10C7980003F10103B3F5805F34BF0023012306E0F2
:10C7A8001D9B03F10103FA2B94BF0023012343B11E
:10C7B80042F6E804C2F200044FF01302227203F0BA
:10C7C8007BBE219D95ED135AFCEEC55A15EE907A65
:10C7D800BEB21C964FEA162242EA062040F6DC61F9
:10C7E800C2F200011D9BC852FEF7E9BC1D9D219FA6
:10C7F800BD64FEF7E4BC1D9E2198C664FEF7DFBC4D
:10C808000DF1700CFBF714FC06EE100AF8EE466A00
:10C818002199C1ED136AFEF7D2BC42F6F403C2F2C5
:10C8280000031A7812F0280F08D01D9800F10100B3
:10C83800B0F5805F34BF0020012006E01D9800F1AC
:10C848000100FA2894BF0020012040B142F6E80414
:10C85800C2F200044FF01301217203F02DBE40F61E
:10C86800DC65C2F200051D9FEE5B4FEA162141EA26
:10C8780006239AB207EE902AB8EE670A219880ED4F
:10C88800130A9FEDC97AB4EEC70AF1EE10FAFEF664
:10C8980096ACDFEDC60A30EE601A80ED131AFEF78B
:10C8A8008EBC42F6F403C2F200031A7812F0280F85
:10C8B80008D01D9800F10100B0F5805F34BF00205A
:10C8C800012006E01D9800F10100FA2894BF00201D
:10C8D800012040B142F6E804C2F200044FF013010F
:10C8E800217203F0E9BD40F6DC65C2F200051D9F28
:10C8F800EE5B4FEA162141EA06239AB201EE902A2E
:10C90800B8EE612A219880ED132AFEF758BC1D98CD
:10C91800072808D942F6E803C2F200034FF00802DC
:10C928001A7203F0C9BDFBF7CFFF02EE900AB8EE0A
:10C93800623A219D85ED133AFEF741BC219FD7ED60
:10C94800133A97ED124A63EE844AC7ED134AFFF78C
:10C95800C5BB219E96ED135AF1EE455AC6ED135A02
:10C96800FEF72DBC4FF000004FF001010A46FCF71E
:10C9780077FF219890ED136AF1EE046A66EE267A45
:10C988004FF000010091019145F28840C2F2000089
:10C99800BCEEE70A10EE101A4FF0FF0249F6CD037D
:10C9A800C0F60003F9F706FEFEF709BC42F6F403E9
:10C9B800C2F200031A7812F0280F08D01D9800F16F
:10C9C8000300B0F5805F34BF0020012006E01D9809
:10C9D80000F10300FA2894BF0020012040B142F67C
:10C9E800E804C2F200044FF01301217203F064BDA1
:10C9F80040F6DC65C2F200051D9FE859FBF77AF99D
:10CA0800219EB064FEF7DBBB42F6F403C2F20003DA
:10CA18001A7812F0280F08D01D9800F10300B0F51D
:10CA2800805F34BF0020012006E01D9800F103005C
:10CA3800FA2894BF0020012040B142F6E804C2F26F
:10CA480000044FF01301217203F036BD40F6DC6597
:10CA5800C2F200051D9FE859FBF74CF9219EF064CE
:10CA6800FEF7ADBB1D9B072B08D942F6E804C2F2BE
:10CA780000044FF00800207203F01EBD2198D0ED8D
:10CA8800130AF5EEC00AF1EE10FA0FDB9FED487AB3
:10CA9800F4EEC70AF1EE10FA08D8FCEEE01ACDED74
:10CAA8001C1A4FF0000580F8505021E09FED401A05
:10CAB800F4EEC10AF1EE10FA07DD6FF07F431C9324
:10CAC8004FF0010280F8502012E04FF000021C9253
:10CAD80010EE900A09F0AEFA28B14FF0020621993B
:10CAE80081F8506004E04FF00305219F87F850500B
:10CAF8001D981C99FBF7C0FEFEF761BB219FF86CDF
:10CB080009F0ACFA00287EF45AAB219E96ED132A60
:10CB1800B5EEC02AF1EE10FA04DD4FF07E53F3644F
:10CB2800FEF74DBBB5EEC02AF1EE10FA7EF547AB25
:10CB38004FF00001CBF68071F164FEF740BB219DF8
:10CB4800AA6ACAB1F9F76CFD219FBE6AC6F1040151
:10CB58000B184CF6CD45CCF6CC45A5FB03124FEA95
:10CB680092007E6AB0FBF6F102EE901AB8EE623AD5
:10CB780087ED133AFEF723BB4FF6FF70C7F67F70B9
:10CB8800E864FEF71CBB42F6F403C2F200031A780D
:10CB980012F0280F10D01D9800F10300B0F5805F47
:10CBA80034BF002001200EE000000047000080474D
:10CBB800FFFF7F4B000000341D9800F10300FA28A6
:10CBC80094BF0020012040B142F6E804C2F20004FC
:10CBD8004FF01301217203F06FBC1D9F219DE86C7B
:10CBE800FBF75EF840F6DC66C2F20006F051FEF78D
:10CBF800E6BA219BD3ED123A93ED134A73EEC44A79
:10CC0800C3ED134AFFF76ABA2198C76C1C97856C65
:10CC1800C5648764FEF7D3BA219EF06C09F01EFA4A
:10CC280030B14FF00307219B83F85070FEF7C7BA65
:10CC38002199C86C09F002FA30B14FF00401219A29
:10CC480082F85010FEF7BBBA219AD76C384609F023
:10CC580081FA08EE100A38464FF0000109F014FA7C
:10CC680001464FF07E5009F00FFA1FED2E5A05EEDF
:10CC7800900A25EE856AB4EEC68AF1EE10FA06D857
:10CC88004FF00005219E86F85050FEF798BA219B78
:10CC9800D3ED136AF5EEC06AF1EE10FA05DD4FF038
:10CCA800010083F85000FEF78ABAF5EEC06AF1EE8B
:10CCB80010FA4CBF0222032283F85020FEF77FBAF5
:10CCC8002198D0ED138A90ED128A38EEC89A19EEA1
:10CCD800100A09F03FFA09EE100A18EE900A18EE49
:10CCE800101A09F0D1F901464FF07E5009F0CCF93D
:10CCF8005FED507A00EE100A60EE270AB4EEE09A73
:10CD0800F1EE10FA0DF1700C8CBF00200120FBF73A
:10CD180077F9FEF754BA219DEE6C304609F01AFAFD
:10CD280008EE100A30464FF0000109F0ADF901464F
:10CD38004FF07E5009F0A8F91FED621A07EE100AAD
:10CD480067EE011AB4EEE18AF1EE10FA0DF1700CFB
:10CD58008CBF00200120FBF753F9FEF730BA219968
:10CD680091ED132AD1ED122AB4EEE22AF1EE10FA6F
:10CD78000DF1700CB4BF00200120FBF741F9FEF75C
:10CD88001EBA219A92ED133AB5EEC03AF1EE10FAB6
:10CD98000DF1700CB4BF00200120FBF731F9FEF74C
:10CDA8000EBA219FD7ED133A97ED124AF4EEC43A22
:10CDB800F1EE10FA0DF1700CD4BF00200120FBF742
:10CDC8001FF9FEF7FCB9219BD3ED134A93ED125AD4
:10CDD800F4EEC54AF1EE10FA0DF1700C8CBF00208C
:10CDE8000120FBF70DF9FEF7EAB92198D0ED135AA7
:10CDF80090ED126AF4EEC65AF1EE10FA0DF1700CCD
:10CE080054BF00200120FBF7FBF8FEF7D8B9219D9D
:10CE1800D5ED136AF5EEC06AF1EE10FA0DF1700C5B
:10CE280054BF00200120FBF7EBF8FEF7C8B9219E9C
:10CE3800D6ED138A96ED128A38EEC89A19EE100AC2
:10CE480009F088F909EE100A18EE900A18EE101A7F
:10CE580009F01AF901464FF07E5009F015F95FED17
:10CE6800AB7A00EE100A60EE270AB4EEE09AF1EE13
:10CE780010FA0DF1700CD4BF00200120FBF7C0F8A8
:10CE8800FEF79DB92199CF6C384609F063F908EE91
:10CE9800100A38464FF0000109F0F6F801464FF045
:10CEA8007E5009F0F1F81FEDBD1A07EE100A67EE83
:10CEB800011AB4EEE18AF1EE10FA0DF1700CD4BF4C
:10CEC80000200120FBF79CF8FEF779B942F6F4023E
:10CED800C2F20002137813F0280F08D01D9800F151
:10CEE8000200B0F5805F34BF0020012006E01D98E5
:10CEF80000F10200FA2894BF0020012040B142F658
:10CF0800E804C2F200044FF01300207203F0D4BA10
:10CF1800F9F786FB219F00F104004CF6CD45CCF6CD
:10CF2800CC45A5FB00164FEA96017A6AB1FBF2F3ED
:10CF38001D9D40F6DC60C2F2000041194E78425D4A
:10CF48004FEA024545EA0620897840EA01061B9621
:10CF58009B1B23F07F421C9202EE102AF8EE422A15
:10CF6800C7ED132AFEF72BB9219FFD6CBD64FEF7B0
:10CF780026B9219991F85130002B40F04182FEF7F3
:10CF88001EB9219A92F85100002800F03982FEF764
:10CF980016B942F6F401C2F200010B7813F0280F1B
:10CFA80006D01D9AB2F5805F34BF0022012204E04A
:10CFB8001D9AFA2A94BF0022012242B142F6E804DF
:10CFC800C2F200044FF01300207203F075BA40F665
:10CFD800DC60C2F200001D99435C002B7EF4EFA8D0
:10CFE8001E9A1C920EE242F6F401C2F200010B787E
:10CFF80013F0280F06D01D9AB2F5805F34BF0022C7
:10D00800012204E01D9AFA2A94BF0022012242B1AB
:10D0180042F6E804C2F200044FF01300207203F055
:10D028004BBA40F6DC60C2F200001D99435C002B4D
:10D038003EF4C5A81E9A1C92E4E142F6E801C2F249
:10D0480000014FF001030B7203F036BA1D98F9285E
:10D0580008D942F6E804C2F200044FF01202227224
:10D0680003F02ABA45F27C32C2F20002115C1E9B20
:10D0780019427EF4A4A81F981C90C3E11D99F929B0
:10D0880008D942F6E804C2F200044FF012032372F2
:10D0980003F012BA45F27C33C2F20003585C1E9AC0
:10D0A80010423EF48CA81F991C91ABE142F6F400A3
:10D0B800C2F20000027812F0280F06D01D99B1F5CF
:10D0C800805F34BF0021012104E01D99FA2994BF33
:10D0D8000021012141B142F6E804C2F200044FF0F8
:10D0E8001300207203F0E8B940F6DC60C2F20000D9
:10D0F8001D9BC25C002A7EF462A81E991C91B2E1B5
:10D1080042F6F403C2F200031A7812F0280F06D090
:10D118001D99B1F5805F34BF0021012104E01D99FC
:10D12800FA2994BF0021012141B142F6E804C2F274
:10D1380000044FF01300207203F0BEB940F6DC6023
:10D14800C2F200001D9BC25C002A3EF438A81E995A
:10D158001C9188E142F6F403C2F200031A7812F037
:10D16800280F06D01D99B1F5805F34BF0021012139
:10D1780004E01D99FA2994BF0021012141B142F62A
:10D18800E804C2F200044FF01303237203F094B9C9
:10D1980040F6DC60C2F200001D9BC25C1E998A4208
:10D1A8007EF60DA81F981C902CE142F6F402C2F2FC
:10D1B8000002117811F0280F06D01D98B0F5805F95
:10D1C80034BF0020012004E01D98FA2894BF0020F5
:10D1D800012040B142F6E804C2F200044FF0130304
:10D1E800237203F069B940F6DC62C2F200021D9BAB
:10D1F800D15C1E988142FDF4E2AF1F9A1C9201E1B6
:10D2080042F6F401C2F20001087810F0280F06D0A7
:10D218001D9AB2F5805F34BF0022012204E01D9AF6
:10D22800FA2A94BF0022012242B142F6E804C2F26F
:10D2380000044FF01303237203F03EB940F6DC619B
:10D24800C2F200011D9BC85C1E9A90427DF4B7AFE4
:10D258001F991C91D6E042F6F400C2F20000027851
:10D2680012F0280F06D01D99B1F5805F34BF002158
:10D27800012104E01D99FA2994BF0021012141B13F
:10D2880042F6E804C2F200044FF01303237203F0DD
:10D2980013B940F6DC60C2F200001D9BC25C1E9907
:10D2A8008A423DF48CAF1F981C90ABE042F6F40222
:10D2B800C2F20002117811F0280F06D01D98B0F5BF
:10D2C800805F34BF0020012004E01D98FA2894BF35
:10D2D8000020012040B142F6E804C2F200044FF0F9
:10D2E8001303237203F0E8B840F6DC62C2F20002CE
:10D2F8001D9BD15C1E9881423DF661AF1F9A1C921E
:10D3080080E042F6F401C2F20001087810F0280F1C
:10D3180006D01D9AB2F5805F34BF0022012204E0D6
:10D328001D9AFA2A94BF0022012242B142F6E8046B
:10D33800C2F200044FF01303237203F0BDB840F6A5
:10D34800DC61C2F200011D9BC85C1E9A9042BDF4CC
:10D3580036AF1F991C9155E0219890F847201D99E8
:10D368008A427DF42CAF1E9B1C937CE0219890F898
:10D3780047201D998A423DF422AF1E9B1C9372E000
:10D38800219890F847201D998A427DF618AF1E9B78
:10D398001C9368E0219890F847201D998A42FDF473
:10D3A8000EAF1E9B1C935EE0219890F847201D99B4
:10D3B8008A42BDF404AF1E9B1C9354E0219890F858
:10D3C80047201D998A423DF6FAAE1E9B1C934AE0FF
:10D3D8009DF874000DF16B01FCF762F98DF86A0095
:10D3E8009DF86B1031B142F6E804C2F200042172D4
:10D3F80003F062B800283DF4E2AE1E981C9001E0EC
:10D408001D9A1C921C984DF20003C0F6010393F874
:10D418002E1093F82F2042EA0123834208D242F6C5
:10D42800E804C2F200044FF00900207203F044B887
:10D4380045F28045C2F200052860FDF7C0BE0DF137
:10D44800700CFAF7F5FD1C900028D9D0FDF7B7BE8F
:10D458000DF1700CFAF7ECFD1C900028D0D1FDF707
:10D46800AEBE1D9B1C93219A136A052B08D942F660
:10D47800E804C2F200044FF00A03237203F01CB858
:10D4880003F1020045F28041C2F20001096842F846
:10D49800201003F10103219A1362B3E70DF1700C18
:10D4A800FAF7C6FD1C900028DBD0FDF788BE0DF109
:10D4B800700CFAF7BDFD1C900028D2D1FDF77FBE95
:10D4C8000DF1700CFAF7B4FD1C901D9988427DF49B
:10D4D80076AE1E981C9095E70DF1700CFAF7A8FD32
:10D4E8001C901D9A90423DF46AAE1E9B1C9389E7DE
:10D4F8000DF1700CFAF79CFD1C901D9988427DF681
:10D508005EAE1E981C907DE70DF1700CFAF790FD49
:10D518001C901D9A9042FDF452AE1E9B1C9371E71D
:10D528000DF1700CFAF784FD1C901D998842BDF42A
:10D5380046AE1E981C9065E70DF1700CFAF778FD61
:10D548001C901D9A90423DF63AAE1E9B1C9359E7DB
:10D558009DF874000DF16B01FCF772F88DF86A0004
:10D568009DF86B1031B142F6E804C2F20004217252
:10D5780002F0A2BF00283DF422AE1E981C9041E79D
:10D588009DF874000DF16B01FCF75AF88DF86A00EC
:10D598009DF86B3033B142F6E801C2F200010B721C
:10D5A80002F08ABF00287DF40AAE1E9A1C9229E771
:10D5B8000DF1700CFAF764FD40F6DC60C2F2000071
:10D5C8001E9BC25C1D990A423DF4F9AD1F981C9040
:10D5D80018E70DF1700CFAF753FD40F6DC62C2F261
:10D5E80000021E9BD15C1D9801427DF4E8AD1F9A94
:10D5F8001C9207E70DF1700CFAF742FD40F6DC616A
:10D60800C2F200011E9BC85C1D9A10427DF4D7AD82
:10D618001F991C9127E70DF1700CFAF731FD40F6C0
:10D62800DC60C2F200001E9BC25C1D990A423DF4F8
:10D63800C6AD1F981C9016E798F8005045F00800F2
:10D6480088F80000FDF71CBE0DF1700CFAF7F0FC2D
:10D658008DF86A00219991F851201D9BD1181C91D1
:10D6680042F6F402C2F20002137813F0280F09D030
:10D678001E9A02F1FF335918B1F5805F34BF0021BB
:10D68800012107E01E9A02F1FF335918FA2994BFC5
:10D698000021012141B142F6E804C2F200044FF032
:10D6A8001303237202F008BF4FF000061B961E9F5B
:10D6B800DFB11C9D40F6DC61C2F200014A5D824286
:10D6C80034D007F1FF3240F6DC63C2F200035B1985
:10D6D80040F6DC66C2F20006C6F10101C5EB010E98
:10D6E80012F0010F1AD002F073BF4FF0FF001B9029
:10D6F8001CE013F8019F02F1FF36484504D11C9540
:10D70800CDF86CC01E9211E03246CD180EEB030C1A
:10D7180013F8017FB84242F06887F0E7CD180EEBA6
:10D72800030C002AE5D11C951E92DEE70DF1700C62
:10D738009DF86C00FAF764FCFDF741BD0DF1700C23
:10D74800FAF776FC42F6580BC2F2000B8BF8000091
:10D758004FF001011C91CDF830B0BBE0219A92F84E
:10D7680051001D9BC1181C9142F6F402C2F200023E
:10D77800107810F0280F07D001F10101B1F5805F92
:10D7880034BF0021012105E001F10101FA2994BF0C
:10D798000021012141B142F6E804C2F200044FF031
:10D7A8001303237202F088BE1E981B900DF1700CB3
:10D7B80026AD45F0010122AE46F001024FF000030C
:10D7C800FAF770FCFDF7FBBC219991F851201D98E0
:10D7D80013181C9342F6F401C2F200010A7812F001
:10D7E800280F05D0B3F5805F34BF0023012303E081
:10D7F800FA2B94BF0023012343B142F6E804C2F296
:10D8080000044FF01300207202F056BE1F9F1E98AE
:10D81800B84228BF38461B900DF1700C26AD45F074
:10D82800010122AE46F001024FF00003FBF7F2FCC3
:10D83800FDF7C5BC0DF1700CFAF7FAFB034642F68A
:10D84800580BC2F2000B58464FF010014BF21C4225
:10D85800C0F6010208F0C8FD1C90CDF830B039E0E0
:10D868001E9B1C931F991B914FF000020C9231E0F4
:10D878004FF0FF301C900C902CE0219EF06C9DF82E
:10D8880078109DF87C2042F65806C2F200060096F1
:10D898004FF0100301934FF00103FCF747FB4FF0E3
:10D8A800FF311C910C9615E0219AD06C9DF87810E8
:10D8B8009DF87C2042F65806C2F2000600964FF00A
:10D8C800100301934FF00003FCF730FB4FF0FF30DB
:10D8D8001C900C961D9BA3F1FB0291B20B91A3F136
:10D8E800FB00032823D841F61C73C2F200034FF44F
:10D8F80011720B9902FB013090F82032032B08D0EB
:10D9080042F6E801C2F200014FF04800087202F046
:10D91800D3BD41F61C76C2F200064FF411770B9A7C
:10D9280007FB026707F104074FF0000605E0219F97
:10D9380097F85160F6184FF00007DDF870B0BBF1AA
:10D94800FF3F11D14FF0FF0B4FF00009C84642F6D8
:10D95800F401C2F200010D9140F6DC60C2F2000051
:10D968000E900F950C9D05E0BBF1000FECD14FF028
:10D9780000096FE01D9BA3F1FB03032B10D8D7F818
:10D988000061FF2E14BF01364646D7F8042196429F
:10D9980006D14046FBF7AAFBD7F804118E42F8D00F
:10D9A800B5F1FF3F15D1219850F8342F1168D1F8FF
:10D9B80000C0494610AA4FF00103E0478DF86B00FC
:10D9C80080B10F9D42F6E804C2F20004207202F012
:10D9D80073BD25B115F809308DF8403002E01B9869
:10D9E8008DF840001C98B0F1FF3F02D19DF84030FF
:10D9F80083B31D9AA2F1FB02032A07D8D7F80001C6
:10DA08009DF840303B54C7F800611FE00D99087835
:10DA180010F0280F05D0B6F5805F34BF0020012034
:10DA280003E0FA2E94BF0020012048B10F9D42F672
:10DA3800E804C2F200044FF01301217202F03CBD69
:10DA48009DF840300E9A935506F1010609F1010937
:10DA5800D9458FD31D9EA6F1FB06032E05D80B9A38
:10DA6800D0B2FAF773FDFDF7AABB219F97F8515082
:10DA780009EB050E87F851E0FDF7A1BB1D9AA2F14D
:10DA8800FB01032958D88FB241F61C71C2F200017C
:10DA98004FF4117202FB071393F82002032808D0F1
:10DAA80042F6E804C2F200044FF04803237202F081
:10DAB80003BD41F61C76C2F200064FF4117505FB52
:10DAC800076505F104051E9901F1FF321E9271B335
:10DAD8004FF0000845F28049C2F200094DF20003F8
:10DAE8009B46C0F6010BD5F80061FF2E14BF013626
:10DAF8004646D5F80401864206D14046FBF7F6FAB9
:10DB0800D5F804118E42F8D0D9F80030D5F80021A4
:10DB18001BF80300A85403F10103C9F80030C5F845
:10DB280000611E9E06F1FF311E91002EDBD1F8B276
:10DB3800FAF70CFDFDF743BB1E9B1C93219991F846
:10DB4800510082181B9242F6F406C2F2000636789B
:10DB580016F0280F08D003F1FF36B218B2F5805F2F
:10DB680034BF0022012206E003F1FF36B218FA2A78
:10DB780094BF0022012242B142F6E804C2F2000436
:10DB88004FF01300207202F097BCC71881F851704B
:10DB98001C9A02F1FF351C95002A3DF410AB45F2A2
:10DBA8008043C2F200031E681B9F40F6DC61C2F28C
:10DBB8000001C9194DF20000C0F6010030184FF0FD
:10DBC800000305F0010E10F803C001F803C003F1CB
:10DBD8000103934242F0ED840DE010F8038001F850
:10DBE800038003F1010310F803E001F803E003F1F7
:10DBF80001039342F1D1E819A91901F1010145F294
:10DC08008042C2F2000211604FF0FF331C9300F112
:10DC180001001B90FDF7D3BA4FF000028DF86A207F
:10DC2800219991F851201D9BD3181C931E9A1B9281
:10DC380042F6F400C2F20000007810F0280F08D075
:10DC480002F1FF32D018B0F5805F34BF0020012008
:10DC580006E002F1FF32D018FA2894BF0020012014
:10DC680040B142F6E804C2F200044FF013002072FB
:10DC780002F022BC40F6DC67C2F2000707EB03099A
:10DC88009DF87CB045F27845C2F200052E688B6B92
:10DC9800F118F75CFF2F52D088464FF00102089226
:10DCA8000B9498F8014004EB072745F27845C2F237
:10DCB80000052E68F3194FF000011C919DF86A00C9
:10DCC800002802F04984F75D03F1010302F046BC25
:10DCD8009DF86A2012B15FB90B9C02E065783DB9E6
:10DCE8000B9C219E96F851209D1886F8515029E0EA
:10DCF80014F8015F19F803B046B9284608F018FB74
:10DD0800C5B2584608F014FB5FFA80FB5D4508D1A0
:10DD18001C9B03F101031C9307F1FF371B999942E0
:10DD2800D6D2B346089800F10100089018F8027F8F
:10DD3800FF2FB6D10B9C4FF00003089302E04FF081
:10DD4800000008900DF1700C0899C8B2FAF758F95C
:10DD5800FDF735BA4FF001008DF86A0060E70DF164
:10DD6800700CFAF765F9034642F6580BC2F2000B3D
:10DD780058464FF010014BF22442C0F6010208F059
:10DD880033FB1C90CDF830B0A4E50DF1700CFAF718
:10DD98004FF9034642F6580BC2F2000B58464FF0B3
:10DDA80010014BF22C42C0F6010208F01DFB1C903A
:10DDB800CDF830B08EE50DF1700CFAF739F903465D
:10DDC80042F6580BC2F2000B58464FF010014BF2C6
:10DDD8003042C0F6010208F007FB1C90CDF830B0C5
:10DDE80078E50DF1700CFAF723F9034642F6580B63
:10DDF800C2F2000B58464FF010014BF23842C0F601
:10DE0800010208F0F1FA1C90CDF830B062E5219BD0
:10DE180093F8516006F1010683F85160FDF7CFB918
:10DE28001D9F40F6DC65C2F20005EA5D02F10102C1
:10DE3800EA55FDF7C4B9219991F8470000F10100AE
:10DE480081F84700FDF7BBB99DF874000DF16B012F
:10DE5800FBF7F6FB0DF1700CFAF7D2F89DF86B3072
:10DE6800002B3DF4ACA942F6E804C2F20004237288
:10DE780002F022BB9DF874000DF16B01FBF748FC22
:10DE88000DF1700CFAF7BCF89DF86B1000293DF401
:10DE980096A942F6E802C2F20002117202F00CBB27
:10DEA8001D981C904FF000031B934FF001018DF853
:10DEB8006A109DF870000DF16B01FBF7C1FB9DF82E
:10DEC8006B309BB920B19DF86A201B9810431B90BA
:10DED8009DF86A104FEA41038DF86A301C9A02F1E6
:10DEE80001021C9213F0FE0FE3D10AE09DF86A00CC
:10DEF800012806D142F6E804C2F20004237202F0B7
:10DF0800DBBA0DF1700C9DF86C00FAF779F8FDF7A3
:10DF180056B91D991C914FF000031B934FF0010255
:10DF28008DF86A209DF870000DF16B01FBF7F0FB8E
:10DF38009DF86B1099B920B19DF86A001B9B0343AB
:10DF48001B939DF86A204FEA42018DF86A101C98CD
:10DF580000F101001C9011F0FE0FE3D10AE09DF8DA
:10DF68006A30012B06D142F6E804C2F2000421729D
:10DF780002F0A2BA0DF1700C9DF86C00FAF740F8A7
:10DF8800FDF71DB99DF874000DF16B01FBF788FBD7
:10DF98008DF86A009DF86B1031B142F6E802C2F2C2
:10DFA8000002117202F088BA0DF1700CFAF728F825
:10DFB800FDF705B91D981C904FF000031B934FF017
:10DFC80001038DF86A30219991F8472013420ED049
:10DFD8009DF870000DF16B01FBF762FB9DF86B304B
:10DFE8009BB920B19DF86A001B9901431B919DF8CC
:10DFF8006A204FEA42038DF86A301C9800F101004C
:10E008001C9013F0FE03DED10AE09DF86A10012986
:10E0180006D142F6E804C2F20004237202F04CBAB8
:10E028001B9E219F87F84760FDF7C9B89DF87400CB
:10E038000DF16B01FBF79CFB0DF1700CF9F7E0FF9C
:10E048009DF86B0000283DF4BAA842F6E802C2F237
:10E058000002107202F030BA1D9B1C93D8B20DF169
:10E068006B01FBF785FB1B909DF86B1031B142F6F5
:10E07800E804C2F20004217202F01EBA4FF0010552
:10E088008DF86A501C9E70191C90C0B20DF16B017E
:10E09800FBF76EFB9DF86A7000FA07F01B9A0243C3
:10E0A8001B9207F101078DF86A701C9800F10100B6
:10E0B8001C90FBB2072BE8D90DF1700C9DF86C0091
:10E0C800F9F79EFFFDF77BB80DF1700C219991F8D7
:10E0D8005100F9F795FFFDF772B8FDF770B842F6F1
:10E0E800D005C2F200054FF001062E70FDF767B8A3
:10E0F80042F6D007C2F200074FF000023A70FDF76F
:10E108005EB821984FF000014FF0540208F0A2FDCC
:10E118004FF00000219042F66803C2F200031C6829
:10E1280004F1FF31196002F021B942F66803C2F226
:10E13800000319687F2908D942F6E804C2F20004EE
:10E148004FF03002227202F0B7B94FF001051C956A
:10E1580042F62816C2F20006B76D002F42F0098277
:10E1680005E0D2F8AC10002949D11C9301E04FF02A
:10E1780001031D9F42F62815C2F200054FF0540610
:10E1880006FB03F3EA18EF5057601E9882F8520016
:10E198004FF00A015162104600F13400219901F153
:10E1A80034014FF0100208F031FD1C9B06FB0350B0
:10E1B80000F14400219901F144014FF0040208F0F4
:10E1C80025FD1C9F06FB075000F14800219901F12D
:10E1D80048014FF0080208F019FD219A92F8510001
:10E1E8001C9906FB015585F8510042F66806C2F2F3
:10E1F8000006336803F101033360FCF7E0BF03F165
:10E2080001052B4602F15402D2F8AC60002E42F010
:10E21800C781AAE71C93FCF7D2BF219A92F8520053
:10E228001E9082E70DF1700CF9F702FF1E907CE753
:10E238001D9F219880F85170FCF7C1BF0DF1700C3B
:10E248009DF87400F9F7DCFEFCF7B9BF21998B6AD9
:10E25800002B3CF4B4AFF8F7E3F921998A6A801AE5
:10E26800496A1D9B01FB03F303EB83029042BCF454
:10E27800A6AF1E981C90FFF7C5B8F8F7D1F9219DF5
:10E28800A862FCF79CBF45F27C31C2F2000191F80C
:10E29800FB201E9BD018FB2808D942F6E803C2F2DF
:10E2A80000034FF01200187202F006B942F6F401AA
:10E2B800C2F20001087810F0280F09D01D98111833
:10E2C80001F1FF31B1F5805FB4BF0021012107E002
:10E2D8001D99501800F1FF31FA29D4BF00210121FE
:10E2E80041B142F6E804C2F200044FF01302227270
:10E2F80002F0E2B845F27C36C2F20006F01840F6A9
:10E30800DC67C2F200071D9D791908F07FFCFCF755
:10E3180056BF98F8001041F0100588F80050FCF737
:10E32800AFBF219E96F84770002F0CBFFF22002236
:10E3380086F84720FCF743BF219B93F847006FEA14
:10E34800000183F84710FCF73ABF0DF1700CF9F79C
:10E3580097FE1E9D40F6DC66C2F20006775D1D9AA8
:10E368007A407255FCF72BBF219B986B1D990A18B0
:10E378001C92BDE1219BD86B996B42181C92B7E1A6
:10E38800219B186C40B942F6E804C2F200044FF031
:10E398002001217202F090B800F1FF351D64FCF7EE
:10E3A8000EBF219A136C03F101031364002B7CF454
:10E3B80006AF42F6E800C2F200004FF020040472F3
:10E3C80002F07AB821994A6B1368586840B942F646
:10E3D800E803C2F200034FF01E021A7202F06CB892
:10E3E8000DF1700CF9F724FE1C90219850F8346F49
:10E3F80031684E681D991CAA4FF00103B0478DF88B
:10E408006B0000283CF4DBAE42F6E804C2F20004DC
:10E41800207202F051B80DF1700CF9F709FE1C904A
:10E4280054E10DF1700CF9F703FE219FF863FCF736
:10E43800C6BE0DF1700CF9F7FBFD219D2864FCF7B1
:10E44800BEBE219850F8346F31680E681D991CAA19
:10E458004FF00103B0478DF86B0030B142F6E80485
:10E46800C2F20004207202F027B80DF1A80C1CF8C3
:10E47800380DF9F7C5FDFCF7A2BE2198436B0DF1E5
:10E48800700C187AF9F7BCFDFCF799BE0DF1700C09
:10E49800219A92F83C00F9F7B3FDFCF790BE219958
:10E4A800086CFF2808D942F6E804C2F200044FF0CD
:10E4B8002003237202F000B80DF1700CC0B2F9F716
:10E4C8009FFDFCF77CBE219850F8347F3D68AE680C
:10E4D800B04703EE100AF8EE433A219AC2ED133A18
:10E4E800FCF76DBE219991ED0E4AF8EE444AC1ED54
:10E4F800134AFCF764BE219890ED105AF8EE455A7D
:10E50800C0ED135AFCF75BBE219B93ED136AFCEE3A
:10E51800C66ACDED1C6AEBE0219AD2ED137A9FED25
:10E52800B40AF4EEC07AF1EE10FA08DB42F6E80419
:10E53800C2F200044FF02001217201F0BDBFFCEED1
:10E54800E70AC2ED100AFCF73ABE219850F8346F7A
:10E5580033681E681D991CAA4FF00403B0478DF854
:10E568006B0030B142F6E802C2F20002107201F00C
:10E57800A3BF1C98F9F7BEFB219FB864FCF71FBE28
:10E58800219850F8341F0E6836681D991CAA4FF060
:10E598000403B0478DF86B0030B142F6E804C2F2CC
:10E5A8000004207201F088BF1C98F9F7A3FB219D95
:10E5B800E864FCF704BE2198436B1A68516841B9B6
:10E5C80042F6E800C2F200004FF01E02027201F0AB
:10E5D80073BFC06CF9F764FB1C90219850F8346F36
:10E5E80033685E681D991CAA4FF00403B0478DF884
:10E5F8006B0000283CF4E3AD42F6E804C2F20004E4
:10E60800207201F059BF42F6F401C2F200010B7802
:10E6180013F0280F0BD0219AD16B1D9B581800F1CD
:10E62800FF30B0F5805F34BF0020012009E0219859
:10E63800C26B1D998B1803F1FF30FA2894BF002094
:10E64800012040B142F6E801C2F200014FF0130088
:10E65800087201F031BF219B184650F8347F3E689C
:10E6680036684FF0000140F6DC67C2F200071D9AD9
:10E67800BA18DB6BB0478DF86B0000283CF49FADEF
:10E6880042F6E804C2F20004207201F015BF219896
:10E6980050F8343F1E6836681D991BAA4FF00403D2
:10E6A800B0478DF86B0030B142F6E804C2F20004BE
:10E6B800207201F001BF1B998AB2C1F3072040EA1A
:10E6C800022399B21C9113E01D9A1C921C9821995F
:10E6D800F9F74CFD8DF86B0000283CF470AD42F65C
:10E6E800E803C2F20003187201F0E6BE1D981C9000
:10E6F8001C98B0F5803F08D342F6E804C2F2000443
:10E708004FF01F02227201F0D7BE219DA863FCF7CB
:10E7180056BD1D9D219FFD63FCF751BD1D9E21998E
:10E728000E64FCF74CBD219A906B1D9BC11A1C917D
:10E73800DEE71E9A219BD96B8818FB2808D942F678
:10E74800E803C2F200034FF012021A7201F0B4BEDD
:10E7580045F27C37C2F2000787F8FB10184650F8DC
:10E76800346F31680E681D99BA18DB6BB0478DF8A5
:10E778006B0000283CF423AD42F6E804C2F2000422
:10E78800207201F099BE219B586B0668766846B9DD
:10E7980042F6E800C2F200004FF01E02027201F0D9
:10E7A8008BBE42F6F401C2F200010A7812F0280F7B
:10E7B8000AD0DA6B1D99881800F1FF30B0F5805F38
:10E7C80034BF0020012008E0D86B1D990A1802F117
:10E7D800FF30FA2894BF0020012058B142F6E80320
:10E7E800C2F200034FF01301197201F065BE00BFB9
:10E7F8000000804703F134004FF0000140F6DC6769
:10E80800C2F200071D9ABA18DB6BB0478DF86B008F
:10E8180000283CF4D4AC42F6E804C2F200042072AA
:10E8280001F04ABEF6F75EFA00287CF4C8AC1D9BDE
:10E838001C93FEF7E7BDF6F755FA00283CF4BFAC89
:10E848001D991C91FEF7DEBD1D98072808D942F6D0
:10E85800E804C2F200044FF00502227201F02CBE57
:10E86800C0B24FF00001F6F7FBF901EE100AB8EE5E
:10E87800417A219F87ED137AFCF7A1BC1D9B072BDA
:10E8880008D942F6E801C2F200014FF0050008720B
:10E8980001F012BED8B24FF00101F6F7E1F901EE2E
:10E8A800900AB8EE612A219D85ED132AFCF787BCF2
:10E8B8001D9A072A08D942F6E804C2F200044FF06C
:10E8C8000503237201F0F8BDD0B24FF00001F6F74E
:10E8D80037F9FCF774BC1D99072908D942F6E800F6
:10E8E800C2F200004FF00502027201F0E5BDC8B2A5
:10E8F8004FF00101F6F724F9FCF761BC1D9B072BCB
:10E9080008D942F6E804C2F200044FF0050121726A
:10E9180001F0D2BDD8B24FF00001F6F761F9FCF76B
:10E928004EBC1D98072808D942F6E803C2F2000336
:10E938004FF005021A7201F0BFBDC0B24FF00101DD
:10E94800F6F74EF9FCF73BBC9DF87400F2F760FF50
:10E9580000287CF434AC42F6E804C2F200044FF01C
:10E968002801217201F0A8BD9DF87400219901F1D8
:10E978004C01F2F76DFF00287CF421AC42F6E80068
:10E98800C2F200004FF02803037201F095BD219AEE
:10E99800D2ED132A9DF87400BCEEE23A13EE101A79
:10E9A800F2F788FF00287CF40AAC42F6E804C2F2C9
:10E9B80000044FF02801217201F07EBDFCF7FFBB77
:10E9C8000DF1700CF9F734FB30B9219E96F84770B9
:10E9D8003D1C18BF012501E04FF00105219880F882
:10E9E8004750FCF7ECBB9DF874600DF1700CF9F71B
:10E9F8001FFB014630464FF00102FAF731FF8DF850
:10EA08006B0000283CF4DBAB42F6E803C2F20003DB
:10EA1800187201F051BD0DF1700CF9F709FB0146B0
:10EA28008DF86A009DF87400FAF7D8FE8DF86B002F
:10EA380000283CF4C4AB42F6E802C2F200021072AD
:10EA480001F03ABD1D991C914FF001038DF86A3011
:10EA58001E46219890F8472013420AD090F8461095
:10EA68009DF8700019403246FAF7FAFE8DF86B00EF
:10EA780068B99DF86A304FEA43018DF86A101C980E
:10EA880000F101001C9011F0FE03E2D10AE09DF8AC
:10EA98006A20012A06D142F6E804C2F20004207274
:10EAA80001F00ABD4FF000068DF86B600DF1700C97
:10EAB800F9F7BEFA0DF1700CF9F7BAFAFCF77FBB5B
:10EAC8009DF874004FF001010A46FAF7C9FE8DF867
:10EAD8006B0000283CF473AB42F6E801C2F2000177
:10EAE800087201F0E9BC9DF874004FF000014FF086
:10EAF8000102FAF7B5FE8DF86B0000283CF45FAB15
:10EB080042F6E803C2F20003187201F0D5BC0DF119
:10EB1800700CF9F78DFA219F97F84750284387F82A
:10EB28004700FCF74CBB1D980DF1A80C4CF8380DAC
:10EB3800F9F71EFF00287CF442AB45F28040C2F290
:10EB48000000089A026001F028BC10A8F9F7AEFD91
:10EB5800014640B19DF84060022E04D0C2484FF0F3
:10EB68000D0208F053F80DF1700C9DF84000F9F70C
:10EB780047FAFCF724BBFAF7CDFAFCF720BB0DF1F6
:10EB8800700CF9F755FAFCF71ABB1D9EFA2E08D936
:10EB980042F6E804C2F200044FF01203237201F0B7
:10EBA8008BBC0DF1700CF9F743FA45F27C31C2F2D7
:10EBB80000018855FCF703BB0DF1700CF9F738FA22
:10EBC80045F27C37C2F2000787F8FB00FCF7F7BA7A
:10EBD8000DF1700C219D95F84700F9F711FAFCF733
:10EBE800EEBA1D98FA2808D942F6E801C2F20001E7
:10EBF8004FF012040C7201F05FBC0DF1700C45F27D
:10EC08007C32C2F20002105CF9F7FAF9FCF7D7BAC5
:10EC18000DF1700C45F27C36C2F2000696F8FB0046
:10EC2800F9F7EEF9FCF7CBBA1D9EF62E08D942F695
:10EC3800E800C2F200004FF01202027201F03CBC80
:10EC4800219B986CF9F72CF845F27C37C2F2000743
:10EC5800B851FCF7B4BA42F6F401C2F200010B78DD
:10EC680013F0280F06D01D98B0F5805F34BF002040
:10EC7800012004E01D98FA2894BF0020012040B12B
:10EC880042F6E804C2F200044FF01302227201F0C7
:10EC980013BC0DF1700C40F6DC65C2F200051D9E38
:10ECA800A85DF9F7ADF9FCF78ABA0DF1700CF9F720
:10ECB800E7F940F6DC67C2F200071E99785C1D9BF5
:10ECC80018420DF1700C0CBF0020FF20F9F798F9DD
:10ECD800FCF775BA42F6F402C2F20002117811F09C
:10ECE800280F08D01D9800F10100B0F5805F34BFEF
:10ECF8000020012006E01D9800F10100FA2894BFC9
:10ED08000020012040B142F6E801C2F200014FF0B4
:10ED180013020A7201F0D0BB1D9B40F6DC62C2F2FE
:10ED28000002D15CD018437843EA01221C92002AE1
:10ED38003CF445AAFEF766BB42F6F403C2F20003B0
:10ED4800187810F0280F06D01D99B1F5805F34BFF0
:10ED58000021012104E01D99FA2994BF0021012115
:10ED680041B142F6E804C2F200044FF013012172E7
:10ED780001F0A2BB40F6DC62C2F200021D9BD05C2F
:10ED8800002856D1FCF71BBA42F6F402C2F2000280
:10ED9800137813F0280F06D01D98B0F5805F34BFA4
:10EDA8000020012004E01D98FA2894BF00200120CB
:10EDB80040B142F6E804C2F200044FF0130020729A
:10EDC80001F07ABB40F6DC61C2F200011D9A8B5C4F
:10EDD8007BB3FCF7F4B90DF1700CF9F729F91C9025
:10EDE80038BBFCF7ECB90DF1700CF9F749F940F6AE
:10EDF800DC61C2F200011E9A885C1D9B184218D083
:10EE0800FCF7DDB90DF1700CF9F73AF940F6DC6161
:10EE1800C2F200011E9A885C1D9B184209D1FCF7BA
:10EE2800CEB90DF1700CF9F703F91C9000287CF4A9
:10EE3800C6A9219B186A40B942F6E804C2F2000448
:10EE48004FF00301217201F037BB00F1FF351D625D
:10EE580000F1010053F8207045F28046C2F2000626
:10EE68003760FCF7ACB900BFE20E002098F80050FC
:10EE780045F0200188F80010FCF702BA219E96F8A8
:10EE880047704FEAD71242EA470086F84700FCF776
:10EE980096B9219B93F847504FEA550141EAC516A8
:10EEA80083F84760FCF78BB9F9F7D2FCFCF787B910
:10EEB80042F6F807C2F20007FA784FF0010000FAAC
:10EEC80002F03B7923EA00033B71FCF778B942F67C
:10EED800E804C2F200044FF00101217201F0ECBA1B
:10EEE80042F6F805C2F20005EE7846B942F6F80097
:10EEF800C2F200004FF00603C370FCF760B906F1D8
:10EF0800FF3742F6F802C2F20002D770FCF757B991
:10EF180042F6F801C2F200010D7805F1FF36F7B2AA
:10EF28000F700A79FF2A0BD1632F7CF648A942F6A5
:10EF3800F801C2F200014FF063050D70FCF73FB90C
:10EF4800172F7CF63CA942F6F800C2F200004FF0F9
:10EF580017030370FCF733B942F6F806C2F200064D
:10EF6800777807F1FF32D0B270703379FF2B0BD16D
:10EF780000287CF424A942F6F806C2F200064FF0F5
:10EF88000C077770FCF71BB93B287CF618A942F6EA
:10EF9800F801C2F200014FF03B054D70FCF70FB9C4
:10EFA80042F6E804C2F200044FF00102227201F0B6
:10EFB80083BA42F6E800C2F200004FF00103037280
:10EFC80001F07ABA42F6E801C2F200014FF00104FA
:10EFD8000C7201F071BA42F6E800C2F200004FF07C
:10EFE8000102027201F068BA42F6F805C2F20005A1
:10EFF800EE78052E08D942F6F803C2F200034FF066
:10F008000001D970FCF7DBB806F1010642F6F807F3
:10F01800C2F20007FE70FCF7D2B842F6F800C2F25E
:10F028000000027802F10102D5B205700679FF2EC0
:10F038000BD1632D7CF6C3A842F6F801C2F2000199
:10F048004FF000000870FCF7BAB8172D7CF6B7A887
:10F0580042F6F807C2F200074FF000033B70FCF7D6
:10F06800AEB842F6F802C2F20002557805F1010581
:10F07800EEB256701779FF2F0BD10C2E7CF69FA895
:10F0880042F6F800C2F200004FF001024270FCF7AD
:10F0980096B83B2E7CF693A842F6F803C2F200031A
:10F0A8004FF000015970FCF78AB842F6E804C2F242
:10F0B80000044FF00103237201F0FEB942F6F8058F
:10F0C800C2F20005EE784FF0010707FA06F7297932
:10F0D80087EA01002871FCF772B80DF1700CF8F797
:10F0E800A7FF42F6F802C2F200021071FCF767B8F7
:10F0F8000DF1700CF8F79CFF062842F6F803C2F2EF
:10F10800000392BFD8700025DD70FCF758B80DF1E8
:10F11800700CF8F78DFF42F6F806C2F20006307060
:10F12800FCF74DB80DF1700CF8F782FF42F6F807BE
:10F13800C2F200077870FCF742B80DF1700CF8F7CE
:10F1480077FF42F6F801C2F200018870FCF737B881
:10F158000DF1700C42F6F800C2F200000079F8F7E1
:10F168004FFFFCF72CB80DF1700C42F6F802C2F212
:10F178000002D078F8F744FFFCF721B80DF1700CC5
:10F1880042F6F803C2F200031878F8F739FFFCF7E3
:10F1980016B80DF1700C42F6F805C2F20005687851
:10F1A800F8F72EFFFCF70BB80DF1700C42F6F806D5
:10F1B800C2F20006B078F8F723FFFCF700B842F671
:10F1C800E804C2F200044FF00101217201F074B9A1
:10F1D8001D9A0F2A08D942F6E804C2F200044FF03B
:10F1E8002700207201F068B941F6DC67C2F2000717
:10F1F80007EB820042F6F803C2F2000317F8225028
:10F208001D7046785E704FF000019970D970827851
:10F218001A71FBF7D4BF42F6E803C2F200034FF0BD
:10F228000101197201F048B942F6F807C2F2000765
:10F23800FD784FF0010606FA05F63A7946EA02002B
:10F248003871FBF7BCBF42F6E804C2F200044FF085
:10F258000103237201F030B942F6E801C2F200015D
:10F268004FF001020A7201F027B94FF00007139717
:10F2780012971197199742F6F805C2F200052E78F1
:10F2880006F164061696687800F1FF331593A9789D
:10F29800149111A807F0E0FA179A1AB102F1FF3594
:10F2A800EFB201E04FF0060742F6F806C2F2000698
:10F2B800F770FBF784BF1D9A0F2A08D942F6E804B5
:10F2C800C2F200044FF02702227201F0F5B841F6AD
:10F2D800DC60C2F2000000EB820142F6F803C2F2E1
:10F2E80000031F7800F822705D784D701E798E70CB
:10F2F800FBF765BF42F6E800C2F200004FF00101DB
:10F30800017201F0D9B80DF1700C219B93F85000EF
:10F31800F8F776FEFBF753BF42F6F404C2F2000496
:10F32800227812F0010F08D142F6E800C2F200007C
:10F338004FF03001017201F0BFB842F66800C2F226
:10F348000000016841B942F6E804C2F200044FF037
:10F358003102227201F0B0B842F6F403C2F200039F
:10F368001C7804F0FE0242F00400187042F6C00156
:10F37800C2F200014FF000030B6000F0F7BF42F645
:10F38800F403C2F200031C7814F0010F08D142F60E
:10F39800E800C2F200004FF03002027201F08CB8AF
:10F3A80042F66802C2F20002106840B942F6E80369
:10F3B800C2F200034FF034041C7201F07DB842F62B
:10F3C800F401C2F200010B7803F0FE0444F00202DB
:10F3D8000A7042F6C000C2F200004FF0000101605E
:10F3E80000F0C4BF219F97F846500DF1700CF8F754
:10F3F8001FFE219E291A96F8503003F001000A1AC0
:10F408001C9286F84720FF2A94BF0022012286F822
:10F418005020FBF7D4BE42F6F401C2F200010B788B
:10F4280013F0280F06D01D98B0F5805F34BF002078
:10F43800012004E01D98FA2894BF0020012040B163
:10F4480042F6E804C2F200044FF01302227201F0FF
:10F4580033B840F6DC67C2F200071E9D1D9EBD55FD
:10F46800FBF7ADBE4FF000011C911AE04FF001030D
:10F478001C9316E04FF002001C9012E04FF00307B7
:10F488001C970EE04FF004051C950AE04FF00506A6
:10F498001C9606E04FF006021C9202E04FF00701AE
:10F4A8001C911D991B911C98F9F7E6F9FBF787BE8B
:10F4B8000DF1700CF8F7E4FD1E9B40F6DC67C2F214
:10F4C8000007F85C1D9D0543FD54FBF778BE1D9BA6
:10F4D800F92B08D942F6E804C2F200044FF01201F1
:10F4E800217200F0E9BF45F27C36C2F200061E9A8E
:10F4F800F254FBF764BE45F27C37C2F200071D9850
:10F5080087F8FB00FBF75BBE45F24473C2F20003C9
:10F518001A6842B942F6E800C2F200004FF0010151
:10F52800017200F0C9BF56681D981E994FF001027C
:10F538000DF16A03B0478DF86B009DF86A10D1F1A0
:10F54800010238BF0022219B83F8502000283BF499
:10F5580036AE42F6E804C2F20004207200F0ACBFF6
:10F5680045F24472C2F20002136843B942F6E80059
:10F57800C2F200004FF00101017200F09DBF1A684D
:10F588001D981E9990478DF86B0000283BF417AE24
:10F5980042F6E804C2F20004207200F08DBF45F282
:10F5A8004473C2F200031A6842B942F6E800C2F294
:10F5B80000004FF00101017200F07EBF56681D98EF
:10F5C8001E994FF000020DF16A03B0478DF86B00E9
:10F5D8009DF86A10D1F1010238BF0022219B83F8FF
:10F5E800502000283BF4EBAD42F6E804C2F20004D8
:10F5F800207200F061BF09981E99F8F737FF09904B
:10F6080040B942F6E803C2F200034FF0170018723F
:10F6180000F052BF099A13689B6A43B942F6E801A1
:10F62800C2F200014FF015020A7200F045BF0998B6
:10F6380080689DF8741045F27C32C2F20002984747
:10F648008DF86B0000283BF4BAAD42F6E804C2F22C
:10F658000004207200F030BF09981E99F8F706FFE1
:10F66800099040B942F6E803C2F200034FF01700D0
:10F67800187200F021BF09990A68536943B942F624
:10F68800E801C2F200014FF015020A7200F014BF3F
:10F69800099880689DF8741045F27C32C2F2000225
:10F6A80098478DF86B0000283BF489AD42F6E804D2
:10F6B800C2F20004207200F0FFBE09981E99F8F704
:10F6C800D5FE099040B942F6E803C2F200034FF0B4
:10F6D80017021A7200F0F0BE099F39688F6947B99E
:10F6E80042F6E800C2F200004FF01501017200F086
:10F6F800E3BE45F27C36C2F20006099A90689DF88E
:10F70800741032460DF16A03B8478DF86B009DF806
:10F718006A30337000283BF452AD42F6E804C2F276
:10F728000004207200F0C8BE09981E99F8F79EFEE2
:10F7380009901D997F2909D1051C18BF012545F29B
:10F748007C36C2F200063570FBF739BD099840B91E
:10F7580042F6E803C2F200034FF01700187200F0F7
:10F76800ABBE099B1A68536843B942F6E801C2F276
:10F7780000014FF015020A7200F09EBE09988068D9
:10F78800C9B245F27C32C2F2000298478DF86B008C
:10F7980000283BF414AD42F6E804C2F200042072DB
:10F7A80000F08ABE09981E99F8F760FE099040B9E2
:10F7B80042F6E803C2F200034FF017021A7200F093
:10F7C8007BBE099F39688F6847B942F6E800C2F2E4
:10F7D80000004FF01501017200F06EBE45F27C3654
:10F7E800C2F20006099A90689DF8741032780DF1FB
:10F7F8006A03B8478DF86B009DF86A3033700028AB
:10F808003BF4DDAC42F6E804C2F20004207200F0DA
:10F8180053BE09981E99F8F729FE099040B942F697
:10F82800E801C2F200014FF017030B7200F044BE6A
:10F83800099F3868C76847B942F6E800C2F2000075
:10F848004FF01502027200F037BE45F27C36C2F264
:10F858000006099988689DF8741032460DF16A030C
:10F86800B8478DF86B009DF86A30337000283BF478
:10F87800A6AC42F6E804C2F20004207200F01CBEF6
:10F8880009981E99F8F7F2FD099040B942F6E80088
:10F89800C2F200004FF01702027200F00DBE099F7D
:10F8A8003868076947B942F6E801C2F200014FF02B
:10F8B80015030B7200F000BE099ED6F808809DF86B
:10F8C800749045F27C36C2F200063068F8F712FAF6
:10F8D8000246404649460DF16A03B8478DF86B0069
:10F8E8009DF86A20327000283BF469AC42F6E804BF
:10F8F800C2F20004207200F0DFBD09984FF0000149
:10F90800F8F7B4FD099040B942F6E803C2F20003E3
:10F918004FF01700187200F0CFBD09990B68DB6A29
:10F9280043B942F6E801C2F200014FF015020A722B
:10F9380000F0C2BD099880689DF8741098478DF84A
:10F948006B0000283BF43BAC42F6E804C2F200042A
:10F95800207200F0B1BD09981E99F8F787FD09904B
:10F9680040B942F6E803C2F200034FF017001872DC
:10F9780000F0A2BD09990A68D36943B942F6E801C3
:10F98800C2F200014FF015020A7200F095BD099805
:10F9980080689DF8741045F27C32C2F200029847E4
:10F9A8008DF86B0000283BF40AAC42F6E804C2F27A
:10F9B8000004207200F080BD09981E99F8F756FDE2
:10F9C800099040B942F6E803C2F200034FF017006D
:10F9D800187200F071BD09990A68136A43B942F6B2
:10F9E800E801C2F200014FF015020A7200F064BD8E
:10F9F800099880689DF8741045F27C32C2F20002C2
:10FA080098478DF86B0000283BF4D9AB42F6E80420
:10FA1800C2F20004207200F04FBD09981E99F8F751
:10FA280025FD099040B942F6E801C2F200014FF005
:10FA380017030B7200F040BD09990A68536A43B96D
:10FA480042F6E800C2F200004FF01502027200F020
:10FA580033BD099880689DF8741010AA98478DF8EE
:10FA68006B001098F8F71CF945F27C31C2F20001DE
:10FA780008609DF86B30002B3BF4A1AB42F6E8041C
:10FA8800C2F20004237200F017BD09984FF000017C
:10FA9800F8F7ECFC099040B942F6E803C2F200031B
:10FAA8004FF01701197200F007BD09980268136B2F
:10FAB80043B942F6E800C2F200004FF015020272A4
:10FAC80000F0FABC099988689DF8741045F27C32F8
:10FAD800C2F2000298478DF86B0000283BF46FAB28
:10FAE80042F6E804C2F20004207200F0E5BC1D985A
:10FAF800072808D942F6E804C2F200044FF00803C8
:10FB0800237200F0D9BC42F67005C2F2000555F820
:10FB18003070002F7BF453ABF6F782FD002808BF46
:10FB2800012042F67006C2F200061D9A46F832001D
:10FB3800FBF745BB1D99072908D942F6E804C2F22C
:10FB480000044FF00801217200F0B6BC42F67000C4
:10FB5800C2F2000050F83150002D3BF430ABF6F7FC
:10FB68005FFD1D9F42F67006C2F2000656F8372068
:10FB7800831A1C9306EBC701486883428CBF002098
:10FB8800C3EB00001B9042F67005C2F2000505EBBE
:10FB9800C7061B9A72604FF0000345F83730FBF731
:10FBA8000EBB42F6F400C2F20000027812F0280FF1
:10FBB80006D01D9BB3F5805F34BF0023012304E00A
:10FBC8001D9BFA2B94BF0023012343B142F6E8049E
:10FBD800C2F200044FF01301217200F06DBC1D9FAA
:10FBE8000DF1700CF8F724FA40F6DC65C2F2000556
:10FBF800E855FBF7E4BA0DF1700CF8F741FA0DF18E
:10FC0800700CF8F715FA1C9050B11E9D40F6DC6692
:10FC1800C2F20006725D1D9911437155FBF7CFBA08
:10FC28001E9E40F6DC62C2F20002905D1D9B20EA37
:10FC380003079755FBF7C3BA1D9B1E9AD018C1B28C
:10FC480045F27C30C2F2000080F8FB10FA2908D98E
:10FC580042F6E804C2F200044FF01203237200F0E7
:10FC68002BBC45F28047C2F200073D6845F27C365E
:10FC7800C2F20006F0184DF20003C0F60103E918BD
:10FC880006F0C4FF3A681E9950183860FBF797BA17
:10FC980042F6F402C2F20002117811F0280F08D0DF
:10FCA8001D9800F10200B0F5805F34BF00200120EC
:10FCB80006E01D9800F10200FA2894BF00200120F8
:10FCC80038B142F6E804C2F200044FF0130222727F
:10FCD800F2E3F6F7A5FC00F104004CF6CD47CCF6AC
:10FCE800CC47A7FB00154FEA9506219B5A6AB6FB3D
:10FCF800F2F71C971D9D40F6DC61C2F200014FEA45
:10FD0800174048554E194FEA17237370B770FBF721
:10FD180056BA42F6F401C2F20001087810F0280F32
:10FD280008D01D9B03F10203B3F5805F34BF0023A5
:10FD3800012306E01D9B03F10203FA2B94BF002365
:10FD480001233BB142F6E804C2F200044FF013026B
:10FD58002272B1E3F6F764FC00F104004CF6CD47DB
:10FD6800CCF6CC47A7FB00254FEA9506219A516AA5
:10FD7800B6FBF1F01D9B40F6DC67C2F20007FE18E7
:10FD88007578FA5C4FEA024141EA0527B37847EAF9
:10FD980003061B96801B20F07F451C950DF1700C07
:10FDA8001E9885422CBF00200120F8F729F9FBF79F
:10FDB80006BA219991F846700DF1700CF8F738F9E8
:10FDC8003E1A1C96219B83F84760FF2E94BF00269D
:10FDD800012683F85060FBF7F2B942F6F400C2F24C
:10FDE8000000027812F0280F08D01D9901F10101D6
:10FDF800B1F5805F34BF0021012106E01D9901F1B2
:10FE08000101FA2994BF0021012139B142F6E80322
:10FE1800C2F200034FF013021A724DE31D9A45F225
:10FE28008043C2F200031B6840F6DC61C2F20001A5
:10FE38004FEA132088548A185370FEF7FABF2198A6
:10FE480090F847501C9590F8467080F8477080F8F5
:10FE58004650FBF7B4B91D98072807D942F6E804BD
:10FE6800C2F200044FF00801217225E3F8F72CFDD7
:10FE78000DF1A80C4CF8380D003018BF0120F8F728
:10FE8800BFF8FBF79CB9219E96F8470096F84630D4
:10FE98000DF1700C984214BF00200120F8F7B0F85B
:10FEA800FBF78DB9219A92F8470092F846500DF168
:10FEB800700C401B18BF0120F8F7A2F8FBF77FB9B8
:10FEC800219F97F8470097F846100DF1700C88426B
:10FED8002CBF00200120F8F793F8FBF770B9219E9A
:10FEE80096F8470096F846300DF1700C984294BF8A
:10FEF80000200120F8F784F8FBF761B9219A92F8FD
:10FF0800470092F846500DF1700CA8428CBF0020B3
:10FF18000120F8F775F8FBF752B9219F97F84700C9
:10FF280097F846100DF1700C884234BF002001206C
:10FF3800F8F766F8FBF743B91D98F62807D942F693
:10FF4800E804C2F200044FF012022272B4E245F251
:10FF58007C36C2F200063058F7F7CCFE219BD864F5
:10FF6800FBF72DB91D99F62907D942F6E800C2F228
:10FF780000004FF0120303729EE245F27C35C2F294
:10FF880000056858F7F7B6FE219FB864FBF717B964
:10FF980045F27C32C2F2000292F8FB201D9BD11878
:10FFA800FB2907D942F6E803C2F200034FF0120119
:10FFB800197281E242F6F400C2F20000017811F0F1
:10FFC800280F09D01E99501800F1FF30B0F5805F56
:10FFD800B4BF0020012007E01E98111801F1FF307E
:10FFE800FA28D4BF0020012038B142F6E804C2F252
:08FFF80000044FF01302227215
:020000040801F1
:100000005EE240F6DC66C2F200061E9D701945F203
:100010007C37C2F20007F91806F0FCFDFBF7D3B8F5
:100020002198466B326856683EB942F6E803C2F240
:1000300000034FF01E01197242E21E9A45F27C3312
:10004000C2F2000393F8FB309918FB2907D942F656
:10005000E800C2F200004FF01202027230E200F13A
:1000600034001D9945F27C37C2F20007BA18B04738
:100070008DF86B0000283BF4A6A842F6E804C2F213
:10008000000420721CE242F6E804C2F200044FF0C1
:100090000100207214E20DF1700CF7F7F5FF40F645
:1000A000DC65C2F200051E9FEE5D1D9A16423BF410
:1000B0008AA845F28043C2F200030899196070E1F2
:1000C0000DF1700CF7F7E0FF40F6DC60C2F20000C3
:1000D0001E9D475D1D9E37427BF475A845F2804406
:1000E000C2F20004089A22605BE19DF874000DF1F1
:1000F0006B01F9F7A9FA8DF86A009DF86B302BB106
:1001000042F6E804C2F200042372D9E100283BF46D
:100110005AA845F28040C2F200000899016040E10F
:100120009DF874000DF16B01F9F78EFAD0F1010220
:1001300038BF00228DF86A209DF86B1029B142F675
:10014000E802C2F200021172BAE1219DEF6A17B90A
:100150008DF86A7002E09DF86A6066B90DF1700C66
:100160001E98F8F709FC30B945F28044C2F2000449
:100170000898206015E10DF1700C9DF86A00F7F702
:1001800043FF4FF00002219BDA62FBF71CB89DF899
:1001900074000DF16B01F9F757FA8DF86A009DF8BC
:1001A0006B302BB142F6E800C2F20000037287E127
:1001B00000287BF408A845F28045C2F20005089F9C
:1001C0002F60EEE09DF874000DF16B01F9F76CFA09
:1001D0008DF86A009DF86B1029B142F6E802C2F270
:1001E000000211726CE100287AF4EDAF45F280460E
:1001F000C2F20006089C3460D3E09DF874000DF153
:100200006B01F9F751FA031C18BF01238DF86A300E
:1002100092E79DF874000DF16B01F9F715FA0030C3
:1002200018BF01208DF86A0086E71D9EF62E07D9BB
:1002300042F6E803C2F200034FF012041C723FE1E1
:100240002199C86CF7F730FD45F27C35C2F2000504
:10025000A851FAF7B8BF0DF1700CF7F7EDFE219F2A
:1002600097F84760D6F1010238BF0022002814BF7A
:10027000104682F0010087F84700FAF7A4BF0DF19D
:10028000700CF7F7D9FE219991F84750684081F832
:100290004700FAF798BF0DF1700CF7F7CDFE219BE0
:1002A00083F85100FAF78FBF05F046FA0DF1A80C5C
:1002B0004CF8380DFF2828BFFF20C0B2F7F7A4FE86
:1002C000FAF781BF05F02EFA0DF1A80C4CF8380DA5
:1002D000FF2828BFFF20C0B2F7F796FEFAF773BFDA
:1002E00005F034FA0DF1A80C4CF8380DFF2828BFA2
:1002F000FF20C0B2F7F788FEFAF765BF05F008FAED
:100300000DF1700C00280CBFFF200020F7F77CFED9
:10031000FAF759BF45F27842C2F2000210681D99FF
:10032000401804F057FD8DF86B0000283AF44BAFED
:1003300042F6E804C2F200042072C1E01D9804F005
:1003400007FDFAF740BF0DF1700CF7F775FE04F0EA
:10035000F9FCFAF738BF45F27847C2F200073E6869
:100360001D9D701904F010FDFAF72DBF04F0F4FC88
:10037000FAF729BF42F66803C2F200031A6882B98D
:1003800042F6F400C2F20000017801F00204E3B288
:100390003BB142F6E804C2F200044FF03503237289
:1003A0008EE042F6F407C2F200073E7816F0010F25
:1003B0007AF407AF219D2DB145F28042C2F20002CE
:1003C0001068686042F6C001C2F200010C687F2C20
:1003D00000F2CF8004F101041B941C9414B94FF077
:1003E00001071B9742F62816C2F200064FF054058B
:1003F00042F6F404C2F2000442F66807C2F20007B3
:100400001C9B05FB036221929BB9217801F004003B
:10041000C1B209B9386840B9217841F001006FF3E1
:1004200082002070506840B115E04FF001021C922C
:10043000E6E7506878B9802B02D003F1010301E0B0
:100440004FF000031C931B9A9342D9D14FF0000048
:10045000F8F750FED4E742F6C006C2F20006336059
:1004600045F28045C2F2000528604FF0000A54466C
:10047000FAF7A9BE219F396A41F000403863FAF7C4
:10048000A2BE4FF00006219D2E63FAF79CBE40F6F7
:10049000D862C2F200021378002B3AF494AE40F610
:1004A000D867C2F200074FF003013970FAF78BBE2C
:1004B0000B9D42F6E804C2F200044FF001002072E6
:1004C00042F6E804C2F20004089921602198036A08
:1004D00023B103F1010350F82320089242F6E80407
:1004E000C2F20004089961606572F1F76DFBF1F7E3
:1004F0006BFB219D286A78B14FF000031C93219A71
:10050000146A4CB1F1F760FB1C9901F101011C91D7
:10051000219D286A8842F5D840F6D863C2F20003CC
:100520001A782AB94FF00000F8F7E4FDFAF77FBD1A
:10053000F8F7A0FD40F6D864C2F20004217804293F
:100540007AF475AD4FF0000540F6D864C2F20004AD
:100550002846F8F7CFFD20780428F9D0FAF767BDD0
:100560004FF0000703F1FF344FF000035E46FDF744
:10057000B3BB4FF000031C9331E74FF002031C9311
:1005800042F62812C2F20002D2F8AC0030B9FDF7F0
:10059000F0BD2BB0BDEC048BBDE8F08F03F101037F
:1005A00002F15402FDF7E1BD05F1010302F154022D
:1005B000812B7DF4DAADFDF731BEBEF1000F3DF4C5
:1005C00010AB10F8039001F8039003F1010393427C
:1005D0007DF407ABFDF713BBCD180EEB030C13F83E
:1005E000017F02F1FF36B8423DF48DA83246FDF797
:1005F00099B806F1FF32FDF795B800BF704700BF0C
:10060000704700BF42F6C403C2F200031B684B638D
:100610004BB19A68824209D0DB684B631BB19A6880
:100620008242F9D102E04FF01E0070474FF0000007
:10063000704700BF45F2AD43C2F200031A78027062
:1006400045F2AC40C2F2000003780B70704700BF67
:1006500045F2AD43C2F200031B78834225D845F230
:10066000AC42C2F2000212789A18904220DAC01A04
:100670004FEA50034FF0010202FA03F310F0010FAA
:1006800009D045F2B840C2F20000026813400B7076
:100690004FF00100704745F2B040C2F2000002681E
:1006A00013400B704FF0010070474FF0000070478F
:1006B0004FF00000704700BF10B545F2AD43C2F2E5
:1006C00000031B7883427AD845F2AC42C2F20002A2
:1006D00012789A18904275DAC31A03F0FE0445F2B4
:1006E000BC40C2F200000278A418E4B24FEA530200
:1006F0004FF0010000FA02F213F0010F12D041B1E5
:1007000045F2B840C2F20000016842EA010303600A
:100710001AE045F2B840C2F20000036823EA02037F
:10072000036011E041B145F2B040C2F2000003683D
:1007300042EA0301016007E045F2B043C2F2000360
:10074000196821EA0201196045F2B040C2F20000C6
:1007500001680A4224D045F2B843C2F20003186887
:1007600002420ED020464FF00001F1F73DF804F1AF
:100770000102D0B24FF00101F1F736F84FF001005D
:1007800010BD20464FF00101F1F72EF804F10101F0
:10079000C8B24FF00001F1F727F84FF0010010BD8B
:1007A00020464FF00001F1F71FF804F10102D0B22A
:1007B0004FF00001F1F718F84FF0010010BD4FF0B5
:1007C000000010BD4FF0000010BD00BF08B545F29D
:1007D000BC43C2F20003187045F2B443C2F20003F6
:1007E000197045F2AD43C2F200031A70091A01F103
:1007F0000101C8B245F2AC42C2F2000210704128B9
:1008000001D9F0F71FFA40F2F410C2F200004FF0E5
:100810000101F8F789FE08BD2DE9F84345F2BD4313
:10082000C2F2000318784FEA400111F0FF0405D02E
:1008300045F2BD42C2F20002147006E045F2BD4529
:10084000C2F200054FF001062E7045F2E047C2F2F9
:100850000007387845F2BD43C2F200031978084218
:100860000CBF4FF000094FF001094FF000052C4676
:100870004FF0010745F2C046C2F20006A84604F058
:100880001F0207FA02F0AB59184204D0204649462D
:100890004246F8F7E9FF04F10104E4B214F01F0F37
:1008A000EDD105F10405202DE9D1BDE8F88300BFA5
:1008B00045F2E043C2F20003187045F2BD40C2F2B7
:1008C00000004FF001020270704700BF00B583B016
:1008D00045F2C040C2F200004FF000014FF00802A4
:1008E000F0F712FA4FF0000300934FF0010001906F
:1008F00045F2E440C2F200004FF47A714FF0060274
:1009000040F61903C0F60103F5F758FE03B000BD29
:1009100008B545F2E440C2F20000F5F7A9FD4FF03A
:10092000CC00FFF7C5FF08BD89B14FEA501245F270
:10093000C043C2F2000300F01F004FF0010101FAB2
:1009400000F053F82210084343F8220011E04FEA68
:10095000501245F2C043C2F2000300F01F004FF0F6
:10096000010101FA00F053F8221021EA000143F8D6
:1009700022104FF00000704748F65813C0F60103EC
:10098000597A48F2A062C0F2010202FB01F0A0F520
:100990009202997A42F2107000FB0122A2F5EA213C
:1009A000A1F582411B78A3F14E00C2B2012A04D9FD
:1009B000442B14BF0022012201E04FF001024FF44A
:1009C0007A7000FB02124A2B10D148F65811C0F67B
:1009D0000101497861292AD148F65810C0F6010072
:1009E00081786E2923D14FF064036DE0462B5DD0F2
:1009F0004D2B10D148F65811C0F6010148786128F6
:100A000017D148F65811C0F601018978722910D122
:100A10004FF4967358E0412B09D148F65810C0F6B0
:100A200001004178702928D14FF4C8734CE04D2B58
:100A300010D148F65811C0F60101497861292AD130
:100A400048F65810C0F601008178792923D14FF477
:100A5000FA7339E04A2B10D148F65813C0F6010357
:100A6000587875281FD148F65813C0F601039878B6
:100A70006E2878D14FF4167326E0412B0BD148F63F
:100A80005811C0F60101497840F2DC53752908BFBE
:100A90004FF4487318E0532B0BD04F2B0CD04E2B38
:100AA0000DD0442B0ED040F2DC530DE04FF0C803C4
:100AB0000AE04FF4617307E04FF0000304E04FF0E9
:100AC000640301E04FF0C803D21848F65810C0F68E
:100AD000010003792F2B83BF03EB83035900A1F59A
:100AE000F0710021501848F65811C0F601014A79FA
:100AF000A2F13002831845F26470C2F20000036074
:100B000048F64C13C0F60103197848F2A062C0F20F
:100B1000010202FB01F0A0F592015A7842F2107036
:100B200000FB0211A1F5EA22D9784FF47A7000FB9C
:100B30000122A2F53B41A1F583401A794FF06401EF
:100B400001FB02009A7902EB820100EB4100A0F563
:100B5000A552DB79A3F13003D11845F26070C2F2DF
:100B600000000160704748F65813C0F601039878FA
:100B70006C2898D14FF42F73A6E700BF08B54FF447
:100B800040404BF25041C0F6010145F20852C2F21A
:100B90000002F8F787FC08BD10B584B0144649BBC5
:100BA0000DF10D0300930DF10E0001904FF00000C8
:100BB00001460DF10A020DF10B03F4F7EFF94FF0C6
:100BC00000018DF80C109DF80B201AB14FF00103B5
:100BD0008DF80C309DF80A0028B19DF80C1041F0FA
:100BE00002028DF80C204FF000008DF80F00039BDF
:100BF000236001E04FF0140004B010BD70B514463E
:100C00008AB199B94FF0000001460246F4F73EFA66
:100C100006462578F4F71EFB85420AD2735D2370E1
:100C20004FF0000070BD4FF0160070BD4FF0140083
:100C300070BD4FF0160070BDF8B515461F464FF059
:100C400000033B70A9B992F8FB0060B14FF00004BB
:100C50002646285D3146F4F70DF904F1010495F8B4
:100C6000FB20A242F5D84FF0010139704FF000008F
:100C7000F8BD4FF01400F8BD10B586B04FF0010478
:100C80001C70F1B945F21453C2F20003197845F211
:100C90001550C2F20000037802AC00944FF010002F
:100CA000019010461A464FF00103F9F743F94BF251
:100CB0004C40C0F60100214607F09EFD4FF00000B9
:100CC00004E04FF000021A704FF0140006B010BD9F
:100CD0002DE9F04115461C464FF00103237004290D
:100CE0007CD8DFE801F0030B7B1B6400687829786F
:100CF000F4F7BCF94FF00000BDE8F081287845F228
:100D00001451C2F2000108706A7845F21553C2F21C
:100D100000031A704FF00000BDE8F0812C786D7868
:100D200005F1040546F26761C6F2666181FB0523A1
:100D30004FEA630202EB820010F0FF0555D04FF03E
:100D40000007A5F1050808F00108042C94BF264609
:100D5000052630463946F4F78DF8A41BE4B2A5F118
:100D6000050515F0FF0544D11DE0042C94BF26466F
:100D7000052630463946F4F77DF8A31BA5F1050595
:100D800005F0FF0503F0FF04042C94BF264605265A
:100D900030463946F4F76EF8A21BD4B2A5F105052A
:100DA00015F0FF05E1D14FF00000BDE8F0812E788D
:100DB000F4F750FA864206D34FF0000020704FF04F
:100DC0001600BDE8F081304605F101014FF0010247
:100DD000F4F778F94FF00000BDE8F0814FF0000023
:100DE00020704FF01400BDE8F0814FF00000BDE826
:100DF000F0814FFA88F6002EB7D0042C94BF264617
:100E0000052630463946F4F735F8A11BCCB2A5F1DA
:100E1000050515F0FF05A8D1C5E700BF10B51C46B4
:100E20004FF001032370052941D8DFE801F0030EDC
:100E300018222C361046F4F7E1F800283DD14FF087
:100E4000000020704FF0160010BD4BF23840C0F685
:100E50000100114607F0D0FC4FF0000010BD4BF22E
:100E60003040C0F60100114607F0C6FC4FF000000C
:100E700010BD4BF22C40C0F60100114607F0BCFC3F
:100E80004FF0000010BD4BF22440C0F601001146A7
:100E900007F0B2FC4FF0000010BD4BF21C40C0F652
:100EA0000100114607F0A8FC4FF0000010BD4FF004
:100EB000000121704FF0140010BD4FF0000010BD74
:100EC00008B5012805D0022814BF002201221146CE
:100ED00003E04FF000024FF001014FF00100F4F782
:100EE00097F908BD08B54FF00103137001F1FF3108
:100EF000032921D8DFE801F0020B12194BF244302C
:100F0000C0F6010007F078FC4FF0000008BD4FF07C
:100F10000000FFF7D5FF4FF0000008BD4FF00100C3
:100F2000FFF7CEFF4FF0000008BD4FF00200FFF7C3
:100F3000C7FF4FF0000008BD4FF0000010704FF0E9
:100F4000140008BD08B5F4F77DF94FF001004FF02B
:100F500000010A46F4F75CF9F4F780F94FF00C0051
:100F60004FF00001F3F786FFF4F76CF908BD00BFFE
:100F7000037B13B9437B13B90EE0994208D301F107
:100F8000FF318A18437B9A428CBF0020012001E088
:100F90004FF00000C0B270474FF00100704700BF33
:100FA00070B4447A24B14FF0320606FB04F610E028
:100FB000C5784AF22C74C0F6010454F82550B5F5F2
:100FC000964F9DBF49F26466B6FBF5F606EB8606C2
:100FD0000826847A24B14FF0320505FB04F501E0C0
:100FE00041F28835C07A18B1FF2808BF012001E01E
:100FF0004FF0010001B10E6002B1156003B118603D
:1010000070BC704741F61C73C2F200034FF41172BA
:1010100002FB00304FF00001C0F810124FF6FF73D2
:10102000C0F82C32C0F81812704700BFF8B505465A
:101030000E4641F61C74C2F200044FF4117303FB18
:101040000044D4F8240200EB5007F5F7EDFAD4F889
:101050002812421A974202D9B81AF4F76BFE236895
:101060009A6928464FF00101904741F61C70C2F280
:1010700000004FF4117101FB05014FF6FF7001F103
:1010800004013246F6F7AAFDA31918714FEA10229F
:101090005A7106F10206C4F804614FF00000C4F86A
:1010A000080121680B6A28469847F4F77BFC28461C
:1010B000FFF7A8FFF8BD00BF30B583B041F61C7440
:1010C000C2F200044FF4117505FB0040D0F8300265
:1010D000B1F57A7F1BD3A1F57A7163B1837B13B924
:1010E000C37B13B907E0994224D38A1802F1FF3277
:1010F000C07B824221D8C8B20DF10701F8F73CFB52
:101100009DF80710D1F1010038BF00201AE04FEA26
:10111000D10402F107024FEAD20523B121462A4643
:10112000FFF726FF60B12819B0F5805F2CBF0020C3
:10113000012007E04FF0000004E04FF0000001E064
:101140004FF0000003B030BD08B5B0F57A7F21D272
:1011500079B14FEAD00340F6DC62C2F2000200F03F
:1011600007004FF0010101FA00F0D15C0843D054B0
:1011700008BD4FEAD00340F6DC62C2F2000200F084
:1011800007004FF0010101FA00F0D15C21EA0000F4
:10119000D05408BD00F11800C0B24FF00102F8F7BA
:1011A00063FB08BD10B541F61C74C2F200044FF495
:1011B000117303FB0044D4F81C02F4F767FE4FF0F0
:1011C0000000C4F81C0210BD38B54FF4117101FBCA
:1011D00000F141F61C72C2F200028C18D4F80831FA
:1011E000D4F80451AB420BD08958E3188A6A1979B4
:1011F000904728B1D4F8080100F10100C4F80801B3
:1012000038BD00BF08B541F61C73C2F200034FF4AD
:10121000117202FB0031D1F8082101F10401D1F86B
:1012200000319A420BD141F61C71C2F200014FF419
:10123000117202FB0010D0F81C02F4F7E5FB08BDA8
:1012400070B582B005468DF8071041F61C74C2F2E5
:1012500000044FF4117303FB0044D4F81802002873
:1012600050D11AB12846FFF7CDFE4BE0F5F7DCF977
:10127000D4F82812431AC4F82802D4F81002D4F87B
:101280002422934204D800F10103B3F5807F04D1F6
:101290002846FFF7B7FE4FF00103D4F8101262188A
:1012A00002A911F8010D82F81001C4F81032B4F847
:1012B0002C024FF00102F6F791FCC4F82C0208BB97
:1012C00004F5887694F82032012B03D1304602F0E1
:1012D00033FA38B994F82012022913D1304600F0BD
:1012E00041FD78B14FF00102C4F8182241F61C709C
:1012F000C2F200004FF4117303FB0505D5F81C0280
:10130000F4F782FB02B070BD836B45F21C52C2F24F
:1013100000021360016C45F21853C2F20003196019
:10132000C16B40F2FC12C2F2000211604FF00003E8
:1013300083630364C363704745F21C53C2F2000326
:101340001968816345F21852C2F2000213680364FF
:1013500040F2FC11C2F200010A68C263704700BF8C
:101360002DE9F041804617461E4642F62814C2F287
:101370000004656BAD6808462146FFF743F9002875
:1013800040D1606B0468002C31D0616800292ED0F8
:1013900042F62814C2F200042046FFF7B5FF2046AB
:1013A00050F8342F13685C6841463A463346A047EC
:1013B00070B142F62814C2F200042046FFF7BCFFC9
:1013C00028462146FFF71EF94FF00000BDE8F081E6
:1013D00042F62814C2F200042046FFF7ADFF28466B
:1013E0002146FFF70FF94FF00100BDE8F0812846D4
:1013F00042F62811C2F20001FFF704F94FF0000095
:10140000BDE8F0814FF00000BDE8F081F0B583B099
:101410000D461E46ADF8062041F61C72C2F20002CF
:101420004FF4117101FB0020D0F83002037BFF2B39
:1014300003D1427BFF2A00F0B5802C68B4F57A7F97
:1014400018D221464FF00202FFF792FD002800F06B
:10145000AC80002E40F0AC8040F6DC61C2F20001AE
:10146000BDF806206252286800F1020028604FF0A3
:101470000100AEE0A4F57A77B7F57A7F1AD2394643
:101480004FF00102FFF774FD002800F09480002E59
:1014900040F09480BDF806204FEA122140F6DC604F
:1014A000C2F20000C1552B6803F101032B604FF01D
:1014B00001008EE0A4F6B831B1F5FA6F1CD204F148
:1014C0000044A4F6B8344FEA44014FF00202FFF79B
:1014D0004FFD002875D0002E76D140F6DC61C2F2B7
:1014E0000001BDF8060021F814002B6803F1010388
:1014F0002B604FF001006CE0A4F5BB50A0F1100090
:10150000B0F57A7F0FD24EF69003C7F6FF73E2185C
:101510004FEA42004FF001010DF106024FF00203C5
:10152000FFF71EFF55E0A4F5DA53A3F11803B3F556
:101530007A7F0ED24EF2A841C7F6FF7160184FEACB
:1015400040004FF002010DF106020B46FFF708FFC5
:101550003FE0A4F5FA52B2F57A7F0CD24FEA44028A
:10156000A2F57A504FF003010DF106024FF002038D
:10157000FFF7F6FE2DE0A4F50C51A1F12801B1F51D
:101580007A7F24D24DF6D840C7F6FF7023184FEA71
:1015900043004FF004010DF106024FF00203FFF784
:1015A000DFFE16E04FF0000013E04FF0000010E007
:1015B0004FF001000DE04FF000000AE04FF0010095
:1015C00007E04FF0000004E04FF0010001E04FF0B1
:1015D000000003B0F0BD00BF2DE9F04182B08046AD
:1015E00017461D464FF00003ADF8063042F62814AA
:1015F000C2F20004606B866808462146FFF702F8D5
:1016000038B1002D42D04FF001032B704FF0000095
:101610003EE042F62811C2F200014A6B13683BB368
:10162000186828B342F62814C2F200042046FFF7D7
:101630006BFE204650F8342F13681C6841460DF1AC
:1016400006024FF00203A04718B115B14FF0010098
:101650002870012F05D19DF806104FEA0122ADF840
:10166000062042F62810C2F20000FFF765FE03E0F4
:1016700015B14FF001012970304642F62811C2F22F
:101680000001FEF7BFFFBDF8060001E04FF00000CB
:1016900002B0BDE8F08100BF10B504460B4611B1A1
:1016A0004FF000020A702268B2F57A7F08D240F645
:1016B000DC60C2F20000105A02F10202226010BD8A
:1016C000A2F57A71B1F57A7F0AD240F6DC63C2F2F4
:1016D0000003595C4FEA012002F10102226010BDB3
:1016E000A2F5FA60262811D84FF000000146024604
:1016F000F3F7CCFC2368A3F5FA6281184978805C83
:1017000040EA012003F10203236010BDA2F6B831C4
:10171000B1F5FA6F0DD202F10041A1F6B83040F6F2
:10172000DC63C2F2000333F8100002F10102226010
:1017300010BDA2F59C50A0F10800B0F57A7F11D23F
:101740004EF67841C7F6FF7150184FEA40004FF04F
:1017500000014FF00202FFF73FFF236803F101038E
:10176000236010BDA2F5BB51A1F11001B1F57A7F44
:1017700011D24EF69001C7F6FF7150184FEA4000A3
:101780004FF001014FF00202FFF726FF226802F13D
:101790000102226010BDA2F5DA50A0F11800B0F5E8
:1017A0007A7F10D24EF2A840C7F6FF7012184FEAA7
:1017B00042004FF002010A46FFF70EFF236803F1D3
:1017C0000103236010BDA2F5FA51B1F57A7F0ED264
:1017D0004FEA4202A2F57A504FF003014FF00202A5
:1017E000FFF7FAFE216801F10101216010BDA2F5A9
:1017F0000C50A0F12800B0F57A7F11D24DF6D841F7
:10180000C7F6FF7150184FEA40004FF004014FF047
:101810000202FFF7E1FE236803F10103236010BD1C
:101820002BB14FF001021A704FF0000010BD4FF0C5
:10183000000010BD30B583B004460D4602A840F844
:10184000084D68460DF10701FFF726FF9DF80730A8
:1018500083B904F1FF34651902A941F8085D6846AF
:101860000DF10701FFF718FF9DF80720101C18BFA6
:10187000012001E04FF0010003B030BDF0B583B0AE
:1018800004464FF000038DF80730B0F5805F07D2B3
:1018900040F6DC62C2F20002135C8DF807303CE0D7
:1018A000A0F5FA60262806D80B19A3F5FA6001788E
:1018B0008DF8071031E045F22151C2F200010A789B
:1018C0005AB342F62815C2F200056E6BB6684FF0A7
:1018D00002002946FEF796FE6B6B1868B0B10168EE
:1018E000A1B142F62815C2F200052846FFF70CFD0B
:1018F000284650F8347F3A68176821460DF10702F0
:101900004FF00103B8472846FFF716FD304642F670
:101910002811C2F20001FEF775FE9DF8070003B022
:10192000F0BD00BFF0B583B004464FF00003ADF842
:101930000630B0F5805F07D240F6DC63C2F20003E8
:10194000C05AADF806003EE0A0F5FA60262808D897
:1019500004460B185878095D41EA0022ADF80620CC
:1019600031E045F22151C2F200010A785AB342F641
:101970002815C2F200056E6BB6684FF002002946CA
:10198000FEF740FE6B6B1868B0B10168A1B142F67A
:101990002815C2F200052846FFF7B6FC284650F885
:1019A000347F3A68176821460DF106024FF00203B2
:1019B000B8472846FFF7C0FC304642F62811C2F26D
:1019C0000001FEF71FFEBDF8060003B0F0BD00BF2A
:1019D000F0B583B004468DF80710B0F5805F08D2EB
:1019E000CAB240F6DC63C2F200031A544FF001049D
:1019F0003DE045F22153C2F200031878002834D0AC
:101A000042F62815C2F20005696B8E684FF002009D
:101A10002946FEF7F7FD6A6B1368CBB15868D0B161
:101A200042F62815C2F200052846FFF76DFC28464D
:101A300050F8347F39684F6821460DF107024FF0A6
:101A40000103B8472846FFF777FC4FF0010404E094
:101A50004FF0000401E04FF00004304642F6281138
:101A6000C2F20001FEF7CEFD01E04FF00004204677
:101A700003B0F0BDF0B583B00446ADF80610B0F584
:101A8000805F08D240F6DC63C2F200038AB2C25221
:101A90004FF001043DE045F22153C2F200031878F3
:101AA000002834D042F62815C2F20005696B8E6812
:101AB0004FF002002946FEF7A5FD6A6B1368CBB113
:101AC0005868D0B142F62815C2F200052846FFF743
:101AD0001BFC284650F8347F39684F6821460DF1C9
:101AE00006024FF00203B8472846FFF725FC4FF0E7
:101AF000010404E04FF0000401E04FF00004304620
:101B000042F62811C2F20001FEF77CFD01E04FF021
:101B10000004204603B0F0BD10B545F22253C2F2D6
:101B200000031B78032B47D841F61C72C2F2000257
:101B30004FF4117101FB032340F2D072C2F2000294
:101B400052E8001F01F1010142E80014012CF7D016
:101B500018B14FF00100C3F83C0245F22054C2F224
:101B600000044FF001012170D3F840221AB1D3F8DC
:101B70001C02F3F749FF40F2D073C2F2000353E8AE
:101B8000002FA2F1010243E80024012CF7D053E812
:101B9000002FB2F1004F0DD14FF0000243E80024B6
:101BA000012CF4D04EF60450CEF20000016841F052
:101BB00080510160BFF32F8F10BD00BF10B545F2FB
:101BC0002253C2F200034FF004041C70FFF7EAFA3C
:101BD00010BD00BF2DE9F04F8BB005460E4691F8C1
:101BE000029009EB49094AF2E418C0F6010809EB32
:101BF000080308934FF4117B0BFB00FB41F61C7AA2
:101C0000C2F2000A0BEB0A0442F62817C2F20007E0
:101C1000796B8A6809924FF00201F8F72DFB45F2C3
:101C20002250C2F200000570C4F83062304604F55C
:101C3000097104F50D7204F50E73FFF7B1F928462A
:101C4000FFF7E0F9F4F7F0FCC4F828024FF00103C5
:101C500000934BF28440C0F601004FF0040141F6BE
:101C6000C972C0F601022B46F4F71AF8C4F81C0238
